:020000040801F1
:100000000080012045ED0508000000000000000010
:10001000F9EE0508F9EE0508F9EE05080000000004
:100020000000000000000000000000009D02010828
:10003000F9EE05080000000085040108D904010854
:10004000F9EE0508F9EE0508F9EE0508F9EE0508E0
:10005000F9EE0508F9EE0508F9EE0508F9EE0508D0
:10006000F9EE050855770508590E0508F9EE05085B
:10007000C1730508F9EE0508399C0508F9EE050875
:10008000F9EE0508F9EE0508F9EE0508F9EE0508A0
:10009000BDA90508F9EE0508F9EE0508A90E050841
:1000A00089170508F9EE0508F9EE0508F9EE0508C7
:1000B000F9EE0508F9EE0508AD9D0208F9EE050810
:1000C000F9EE0508F9EE0508F9EE0508F9EE050860
:1000D000F9EE0508095C0508596205085568050828
:1000E000F9EE0508F9EE0508F9EE0508F9EE050840
:1000F000F9EE0508F9EE0508F9EE0508F9EE050830
:10010000F9EE0508F1210608F9EE0508F9EE0508F3
:10011000F9EE0508416E0508F9EE0508F9EE050847
:10012000F9EE0508F9EE0508F9EE0508F9EE0508FF
:1001300000000000000000000000000000000000BF
:1001400000000000000000000000000000000000AF
:10015000000000000000000000000000000000009F
:10016000000000000000000000000000000000008F
:10017000000000000000000000000000000000007F
:10018000000000000000000000000000000000006F
:10019000000000000000000000000000000000005F
:1001A000000000000000000000000000000000004F
:1001B000000000000000000000000000000000003F
:1001C000000000000000000000000000000000002F
:1001D0000000000000000000000000005FF8E0F1F7
:1001E000DFF854040068006880F308880B4B196836
:1001F000086801F10401DFF84424B1E8F00FA2E837
:10020000F00FB0E8F80F83F3148880F309884FF0FB
:10021000000080F31188DFF828E470470400002014
:1002200030B44FF0807500E922000446012B14BF62
:1002300003230223002140F80C1C40F8202C44F832
:10024000443D204630BC704708B5836913F8020C62
:10025000012811D004D3022816D00F4B984708BDAF
:100260004EF61C53CEF200031A6842F07F421A6029
:10027000BDE80840FFF7B4BF4EF60453CEF20003CA
:100280004FF080521A6008BDEFF3148121F0010194
:1002900081F3148808BD00BF519F05081EF0040FAC
:1002A0000CBFEFF30880EFF30980FFF7CDBF00200C
:1002B000FFF7CABF4EF62053CEF20003196830B4E0
:1002C00041F47F01196019684EF6905241F07F4168
:1002D000CEF2000219601368B3F5006F15D04EF22C
:1002E000140241F63F11CEF20002C0F201014EF2BB
:1002F00010031160CEF2000307221A605A4B00224D
:100300001A6000DF002030BC7047584958484EF64C
:100310009C53401A41F01002CEF2000320281A60CC
:1003200040F29A804023052203E001321F2A00F0A8
:10033000838098424FEA4303F7D8012302FA03F27D
:10034000C0F2076313434B4D41F011044EF6A05029
:100350004EF69C52691ACEF20000CEF2000220291D
:100360000360146074D94023052202E001321F2A81
:1003700066D099424FEA4303F8D8012302FA03F208
:10038000C0F2075313433C493C4D41F012044EF672
:10039000A0504EF69C52691ACEF20000CEF2000236
:1003A0002029036014605BD94023052202E001325A
:1003B0001F2A49D099424FEA4303F8D8540044F029
:1003C000837444F001144EF6A0524EF69C53132051
:1003D000CEF20002CEF20003C4F200004FF6FE712E
:1003E0001460C1F6FF7118604022052301E08A42C3
:1003F0001CD8013352001F2BF9D13F21C1F200312B
:100400004EF6A053CEF200034EF624521960CEF2FF
:10041000000211684EF6945341F480311160CEF21F
:1004200000031A6842F005021A6058E7590041F0CB
:10043000985141F00101E3E73F23C0F2076382E7EF
:100440003F23C0F207539EE73F24C0F20714BAE7E8
:100450000923C0F2075396E70923C0F2076372E746
:100460000924C0F20714AEE7040D002000000108C3
:1004700000001008004001080000002000020020D9
:10048000704700BFEFF30980124B1A68EFF3148135
:1004900020E9F20F10602DE908404FF0BF0080F313
:1004A000118801F07DFA4FF0000080F31188BDE85B
:1004B00008401968086801F10401604AB1E8F00FCA
:1004C000A2E8F00FB0E8F80F83F3148880F30988EE
:1004D000704700BF0400002008B54FF0BF0080F354
:1004E000118841F29563C0F6010398474FF0000070
:1004F00080F3118808BD00BF30B4002945D0002B1F
:1005000027D105254C68ECB10B6845F01002134368
:10051000202C83607AD94023052202E001321F2A71
:1005200015D09C424FEA4303F8D852008B6843F041
:1005300001031343C36001350C310830082DE1D1AC
:1005400030BC704745F010038360C460F3E73E227F
:10055000ECE79B0042F01402202B026058D94022A5
:10056000052402E001341F2C0BD093424FEA4202D3
:10057000F8D8012304FA03F4C0F20733234343609D
:10058000BFE73F23C0F20733F9E7274B274943F082
:100590001402C91A2029026042D94023052202E030
:1005A00001321F2A2AD099424FEA4303F8D8012387
:1005B00002FA03F2C0F2073313431D4A1D4942F009
:1005C0001504891A20294360846025D94023052217
:1005D00002E001321F2A15D08B424FEA4303F8D3C1
:1005E000520042F0837242F00112C26016220023D0
:1005F0000261172243618261C361A1E73F23C0F218
:100600000733DAE73F22C0F20712EEE708228DE750
:100610000923C0F20733B2E70922C0F20712E4E768
:100620000923C0F20733C8E7000000200080012042
:10063000000000200002002008ED00E09CED00E03A
:10064000FDFFFFFF2DE9F84306460F4638B34C2067
:10065000174DA847044610B306FB07F808F1010040
:10066000A84705462060E8B1721E07FB020200EBB6
:1006700008014FF0FF336160002104F11000DFF842
:100680003890A163E2606364A364A560E6632764B5
:10069000C84704F12400C8472046BDE8F88300207D
:1006A000BDE8F8832046034B98472846BDE8F88309
:1006B000611C0108A51C010801A505082DE9F04FE2
:1006C000824687B0A14F039202930191B847DAF8AE
:1006D0003820DAF83C3000259A42DFF88482DFF8CF
:1006E00084B29B4CC0F09780039E002E00F01B81CB
:1006F000002D00F0088104ADC047D847B847DAF8AC
:100700004430013300F00B81DAF84830013300F057
:100710000281C04741F6F523284603A9C0F601032C
:100720009847002840F00481B847DAF83860DAF8D2
:100730003C5049F68973C0F605039847AE4240F035
:100740008C800AF1100528460399824B984749F698
:100750005573C0F605039847DAF84830002B1DDDC5
:10076000DAF82430D3B10AF12406DFF8EC9109E07D
:10077000DAF84830013B002BCAF848300EDDDAF8D1
:1007800024305BB13046A0470028F1D0C847DAF8E2
:100790004830013B002BCAF84830F0DC4FF0FF3303
:1007A000CAF84830C047B847DAF84430002B1ADDA1
:1007B000DAF81030BBB1684E09E0DAF84430013B9A
:1007C000002BCAF844300EDDDAF810305BB1284651
:1007D000A0470028F1D0B047DAF84430013B002BA5
:1007E000CAF84430F0DC4FF0FF33CAF84430C04759
:1007F0005A4B984730B94EF60453CEF200034FF0EF
:1008000080521A600125B847DAF83820DAF83C300F
:100810009A42BFF469AFDAF84020002A40F0EB803A
:10082000DAF80040002C00F01581DAF83830013396
:10083000CAF83830DAF8243063B1454B0AF12400A5
:100840009847012801BF4EF60453CEF200034FF043
:1008500080521A60C047012067E049F65573C0F620
:1008600005039847DAF84830002B1CDDDAF824300D
:10087000CBB10AF12406384D09E0DAF84830013BE3
:10088000002BCAF848300EDDDAF824305BB1304670
:10089000A0470028F1D0A847DAF84830013B002BE8
:1008A000CAF84830F0DC4FF0FF33CAF84830C04790
:1008B000B847DAF84430002B1CDDDAF81030CBB141
:1008C0000AF11005244E09E0DAF84430013B002B10
:1008D000CAF844300EDDDAF810305BB12846A04784
:1008E0000028F1D0B047DAF84430013B002BCAF8B9
:1008F0004430F0DC4FF0FF33CAF84430C047174BA8
:10090000984701257FE704AD41F6DD232846C0F670
:1009100001039847F0E60023CAF84830F9E60023BF
:10092000CAF84430F0E6C047304607B0BDE8F08F63
:10093000B847DAF84830002B2CDDDAF824304BB316
:100940000AF12405024C044E18E000BF559F05082B
:10095000711A0108011A0108611B0108AD1701088D
:10096000899F05082D160108DAF84830013B002B55
:10097000CAF848300EDDDAF824305BB12846A047CB
:100980000028F1D0B047DAF84830013B002BCAF814
:100990004830F0DC4FF0FF33CAF84830C047B84762
:1009A000DAF84430002B1DDDDAF81030D3B12D4CCD
:1009B0000AF110052C4E09E0DAF84430013B002B17
:1009C000CAF844300EDDDAF810305BB12846A04793
:1009D0000028F1D0B047DAF84430013B002BCAF8C8
:1009E0004430F0DC4FF0FF33CAF84430C0471F4BAF
:1009F0009847002099E7029BABB901991C4BDAF8A4
:100A000008009847DAF80810DAF84030DAF80420DD
:100A1000CB189342CAF80830FFF407AFDAF8003079
:100A2000CAF8083001E70199114BDAF80C00984731
:100A3000DAF84030DAF80C205B42DAF80010D2180D
:100A40008A42CAF80C203EBFDAF80420D318CAF84C
:100A50000C30EAE6DAF80400064B9847CAF804407E
:100A6000E3E600BF711A0108611B0108AD17010818
:100A7000755F01080D1C010838B50A4B456804462E
:100A80009847854201D0002038BDE1680139E16016
:100A900009B1012038BD20460A460B46FFF70EFE7D
:100AA000012038BD951B010870B54C200F4B9847AD
:100AB0000446C8B100254FF0FF330122E2636364AE
:100AC000A36400F110000A4E65602560A560E56032
:100AD000A5632564B04704F12400B04720462946A9
:100AE0002A462B46FFF7EAFD204670BD611C01082F
:100AF00001A5050870B5044616464FF0BF0080F307
:100B00001188A56BE06B854206D300234FF00000EF
:100B100080F31188184670BD226C62B92568002DDB
:100B200032D0A26BA36C0132A2635A1C11D00133E4
:100B3000A3640123EAE7C3B9164BA0689847A168EC
:100B4000236C6268CB189342A360EAD32368A36046
:100B5000E7E7636A002BECD004F124000E4B9847C2
:100B60000028E6D001233360D0E70A4BE0689847BD
:100B7000226CE368524221689B188B42E3603EBFBF
:100B800063689B18E360CCE76068044B9847656036
:100B9000C7E700BF755F0108711A01080D1C010845
:100BA0002DE9F04F814687B0A74E0193A74F0291E0
:100BB0000392B047D9F838300025DFF8A8A2B8462C
:100BC000A34C002B40F091800398002800F0368160
:100BD000002D00F0C08004ADB847D047B047D9F829
:100BE0004430013300F01B81D9F84830013300F064
:100BF0001281B84741F6F523284603A9C0F6010340
:100C00009847002840F03281B047D9F83850C047A3
:100C1000002D40F0A880D9F80030002B00F00381AF
:100C200009F124058B4B284603999847B047D9F81A
:100C30004830002B1BDDD9F82430C3B1DFF828B2CF
:100C400009E0D9F84830013B002BC9F848300EDDE7
:100C5000D9F824305BB12846A0470028F1D0D84706
:100C6000D9F84830013B002BC9F84830F0DC4FF090
:100C7000FF33C9F84830B847B047D9F84430002BA3
:100C80001DDDD9F81030D3B109F11005DFF8D8B166
:100C900009E0D9F84430013B002BC9F844300EDD9F
:100CA000D9F810305BB12846A0470028F1D0D847CA
:100CB000D9F84430013B002BC9F84430F0DC4FF048
:100CC000FF33C9F84430B847634B984730B94EF604
:100CD0000453CEF200034FF080521A600125B04752
:100CE000D9F83830002B3FF46FAFD9F80030D9F87D
:100CF0000C4073B1D9F84020D9F80400A118814202
:100D0000C9F80C10029824BFC9F80C301946534B8F
:100D10009847019B002B40F0FE80D9F83820D9F885
:100D20000030013AC9F83820002B00F00481D9F8CE
:100D30001030002B00F0F48009F11000444B98476C
:100D4000012840F0ED804EF60453CEF200034FF040
:100D500080521A60E4E004AD41F6DD232846C0F677
:100D60000103984738E749F65573C0F605039847DD
:100D7000D9F84830002B1DDDD9F82430D3B109F162
:100D80002405DFF8E4B009E0D9F84830013B002B36
:100D9000C9F848300EDDD9F824305BB12846A047A9
:100DA0000028F1D0D847D9F84830013B002BC9F8CA
:100DB0004830F0DC4FF0FF33C9F84830B847B0474F
:100DC000D9F84430002B1DDDD9F81030D3B109F12A
:100DD0001005DFF894B009E0D9F84430013B002B4E
:100DE000C9F844300EDDD9F810305BB12846A04771
:100DF0000028F1D0D847D9F84430013B002BC9F87E
:100E00004430F0DC4FF0FF33C9F84430B847124BA0
:100E10009847012563E70023C9F84830E9E6002335
:100E2000C9F84430E0E649F65573C0F60503984723
:100E3000D9F804000A4B9847C047F1E60090B8473C
:100E4000009807B0BDE8F08F559F0508899F0508F9
:100E5000711A0108011A0108AD170108755F010830
:100E6000A11B01082D160108611B0108B047D9F824
:100E70004830002B1EDDD9F82430DBB1304C09F1AD
:100E80002405DFF8C08009E0D9F84830013B002B89
:100E9000C9F848300EDDD9F824305BB12846A047A8
:100EA0000028F1D0C047D9F84830013B002BC9F8E1
:100EB0004830F0DC4FF0FF33C9F84830B847B0474E
:100EC000D9F84430002B1DDDD9F81030D3B109F129
:100ED00010051B4C1B4E09E0D9F84430013B002B98
:100EE000C9F844300EDDD9F810305BB12846A04770
:100EF0000028F1D0B047D9F84430013B002BC9F8A5
:100F00004430F0DC4FF0FF33C9F84430B8470E4BA3
:100F10009847002095E7D9F82430C9F80C4013B958
:100F2000B84701208DE709F12400054B98470028B8
:100F30007FF409AFF4E7054B9847C9F80400F6E6DB
:100F4000711A0108611B0108AD170108951B010802
:100F500070B50C4B456804460E46984785420CD048
:100F60000021204632460B46FFF71AFE012800D02A
:100F700070BDE3680133E36070BDE36801201B18B6
:100F8000E36070BD951B010870B5044616464FF02E
:100F9000BF0080F31188A36B2BB94FF0000080F3E2
:100FA0001188184670BD206860B1E368226C6568DE
:100FB0009B18AB42E36024BF0346E0600846194635
:100FC0000B4B9847A26B636C013A591CA26303D088
:100FD000013363640123E0E72369002BFAD004F1B5
:100FE0001000044B98470028F4D001233360D4E765
:100FF000755F0108711A010849F6557310B5C0F6FE
:10100000050304469847A46B49F68973C0F60503A7
:101010009847204610BD00BF806B704738B541F639
:10102000A5440546C0F601040068A0472846A0472D
:1010300038BD00BF806BD0F1010038BF0020704781
:10104000826BC06BB2EB000CDCF1000050EB0C00CB
:10105000704700BF2DE9F04F814683B0684F68208C
:101060008B4616469A460E9DB8470446002800F067
:10107000C380002D00F0B3800565B200A52128468D
:10108000604B9847236D06F1FF3C03EB8C030C9DEE
:101090005946102223F0070704F154005A4B984791
:1010A00025F0004B594B0022BBF1040F34BF5D46C5
:1010B000042504F1240884F86320E564656640464D
:1010C00001939847C5F1050504F13800019B984745
:1010D0003346A563201D0F99226D4D4D2463646432
:1010E000A8470C9D3846EB0F49464A4D5246A84743
:1010F0000D9D206005B12C60474D484B98472B68EB
:1011000001332B606B68002B3ED0D5F8D8308BB301
:1011100005F10806E36CD5F8DC20D5F8E41093421D
:1011200088BF3D4A03EB830088BFC2F8DC30D5F8A6
:10113000E02006EB800001328B42C5F8E02088BF3A
:10114000354A414688BFC2F8E430354B9847354BA5
:101150009847D5F8D8309BB12F4B5B68DB6C9B452B
:101160000ED94EF60453CEF200034FF080521A60AF
:10117000012006E06B68DB6C9B4528BF6C60C7E70D
:10118000012003B0BDE8F08F6C602B6805F1080604
:10119000012BBFD1244F3046B84705F11C00B8479A
:1011A00005F13000B84705F14400B84705F16C0A75
:1011B00005F15800B84705F180095046B847484640
:1011C000B84705F19400B84705F1A800B84705F104
:1011D000BC00B847C5F8D0A0C5F8D4909AE7B200D3
:1011E00010460192B847019A0546206500287FF411
:1011F00045AF20460D4B98474FF0FF30C1E700BF89
:10120000611C0108096001082166010819A505088B
:10121000F90401082102010800000020559F05087B
:1012200021A50508899F050801A50508A51C010839
:101230002DE9F0411A4C1B4B0546984763689D42C7
:101240002BD02E464DB306F124073846DFF86480D4
:10125000C047B36C13B106F13800C0471248394695
:10126000124B9847D4F8E030D4F8E820013301322B
:10127000C4F8E0300E4BC4F8E8209847D4F8D830D2
:1012800003B10DB1BDE8F0814EF60453CEF2000378
:101290004FF080521A60BDE8F08166680025D2E701
:1012A00000000020559F0508A800002021A5050882
:1012B000899F050875A5050810B5064B0446984793
:1012C00024B1E46C044B9847204610BD034B5C6886
:1012D000F7E700BF559F0508899F0508000000201B
:1012E0002DE9F041274B0546042934BF0E4604265C
:1012F0009847254B5A68954240D02C46002D3DD04A
:10130000636EB3421ED021D3D5F1010538BF00254D
:10131000E26C1D4F934207F1080803EB8303626BF5
:1013200008EB830308BFE664C6F105019A426666CE
:10133000A1630FD035B14EF60453CEF200034FF047
:1013400080521A60114B9847BDE8F081003518BFF4
:101350000125DDE704F1240630460D4B9847E36C88
:10136000D7F8E42003EB8300934288BFC7F8E4304A
:1013700008EB80003146074B9847DBE75C680025A7
:10138000BEE700BF559F050800000020899F0508A3
:1013900075A5050821A505082DE9F041344D354B0B
:1013A000044698476B689C4254D02646002C51D086
:1013B00006F124073846DFF8CC80C047B36C13B180
:1013C00006F13800C0472A4E2B4B394606F1BC00C7
:1013D00098472A4B98470CB1BDE8F081D6F8D83031
:1013E0007BBBD6F8BC2033689A4239D0D6F8EC30B3
:1013F000002B38D1D6F8E43003EB830306EB8306E9
:10140000B3686BB9D5F8E430013BC5F8E430D5F8E2
:10141000E43003EB830305EB83039B68002BF1D0DF
:10142000D5F8E420164B02EB820203EB82025368EC
:1014300002F108015B688B4253600ED0DB686B6081
:10144000CAE74EF60453CEF200034FF080521A6002
:10145000BDE8F0816E680024AAE75B685360EDE7A1
:101460007460BDE8F0810123C6F8F030BDE8F0817A
:1014700000000020559F050821A50508899F050843
:101480000800002075A50508436B074A934201D068
:1014900000207047806C283B9842F9D0D0F10100C1
:1014A00038BF0020704700BFBC00002070B5044664
:1014B00060B11B4D6B68984208D01A4B9847636B1C
:1014C00005F1BC02934202D0174B984770BDA36C44
:1014D00005F194029342F7D0002BF5D104F12406D4
:1014E0003046124B9847D5F8E420E36C10489342FD
:1014F00088BFC5F8E43003EB830300EB830031467B
:101500000C4B98476B68E26CDB6C9A4221BF4EF63D
:101510000453CEF200034FF080521A60D4E700BFAC
:1015200000000020559F0508899F050875A505083E
:101530000800002021A50508F8B51B4C436B04F1F9
:10154000BC029342054602D000263046F8BD866CA8
:1015500004F194008642F7D0002EF5D1D4F8EC3097
:10156000E3B96268EB6CD66C05F12407B3423846E8
:101570000E4B34BF002601269847EB6CD4F8E420CC
:101580000B48934288BFC4F8E43003EB830300EBBD
:1015900083003946074B98473046F8BD05F13801BE
:1015A000044B98473046F8BD0000002075A505089B
:1015B0000800002021A5050810B54FF000430024C5
:1015C00084B08DE8180080222346029403940A48D0
:1015D0000A49FFF73FFD0128034601D004B010BDC2
:1015E0004FF0BF0080F31188054AC2F8D830054B90
:1015F000C2F8F4409847F1E781A40508DCC1060869
:1016000000000020B502010808B54FF0BF0080F3CC
:10161000118840F2000240F28143C2F20002002130
:10162000C0F60103C2F8D810984708BD40F2000385
:10163000C2F20003D3F8EC200132C3F8EC2070476B
:1016400049F6557310B5C0F60503984740F20002FD
:10165000C2F20002D2F8F44049F68973C0F60503DD
:101660009847204610BD00BF4FF0BF0080F311889F
:1016700040F20003C2F20003D3F8F4304FF0000050
:1016800080F311881846704740F20003C2F200034D
:10169000186870472DE9F84F404DD5F8EC30002B15
:1016A00069D1D5F8F4300133C5F8F430D5F8F43009
:1016B000002B4AD0D5F8F830D5F8F420374E9A42AE
:1016C0003CD3D6F8D0301B68002B33D0D6F8D030BE
:1016D000DB68DC68D6F8F420636A93425BD8304F4D
:1016E00006F10809DFF8C080BA4608E0D6F8D03025
:1016F000DB68DC68D6F8F420636A93424BD804F1C7
:10170000240B5846B847A36C04F1380003B1D04706
:10171000E36CD5F8E42003EB8300934209EB8000EF
:10172000594688BFC6F8E430C047D5F8D0301B68AA
:10173000002BDBD14FF0FF33C5F8F830D5F800317E
:101740000BB9184B9847BDE8F88FD5F8D030D5F8CD
:10175000D420C5F8D020C5F8D430D5F8FC300133FA
:10176000C5F8FC30D5F8D0301B6863B94FF0FF33B3
:10177000C5F8F830A0E7D5F800310133C5F80031DD
:10178000084B9847DAE7D5F8D030DB68DB685B6A4E
:10179000C5F8F83090E7C5F8F830CFE70000002032
:1017A00075A50508A1ED050821A505082DE9F84F47
:1017B000324C334B9847D4F8EC30013BC4F8EC3052
:1017C000D4F8EC30002B46D12268002A43D0DFF851
:1017D000B890DFF8B8B09846274604F1080A1DE033
:1017E000D7F8A030DD6805F1380005F12406C847B8
:1017F0003046C847EB6CD7F8E42003EB83009342F4
:101800000AEB8000314688BFC7F8E430D8476368E8
:10181000EA6CDB6C9A4228BF4FF00108D4F8943090
:10182000164A002BDCD1D2F800316BB1D2F800316E
:1018300053B1FFF72FFFD4F80031013BC4F800315A
:10184000D4F80031002BF4D1B8F1010F09D0D4F84D
:10185000F030012B05D000240A4B98472046BDE804
:10186000F88F00224EF60453C4F8F020CEF20003A5
:101870004FF0805201241A60EEE700BF0000002004
:10188000559F0508899F050875A5050821A5050828
:1018900038B538B94EF60453CEF200034FF08052FB
:1018A0001A6038BD154CD4F8EC300133C4F8EC3074
:1018B000D4F8F4506368451903F12400104B98479D
:1018C0006268D4F8F43055629D4210D3D4F8D00049
:1018D00061680C4B24319847D4F8F8309D4238BFEA
:1018E000C4F8F850FFF762FF0028D3D038BDD4F811
:1018F000D4006168034B24319847F3E700000020CF
:1019000075A505083DA5050838B5224C0368D4F82F
:10191000EC20CD180132C4F8EC20D4F8F420934226
:101920000DD9AB420DD80560FFF740FF50BB4EF616
:101930000453CEF200034FF080521A6038BDAB4220
:1019400003D8D4F8F4309D42EDD96368056003F103
:101950002400114B98476268D4F8F43055629D42D8
:101960000C4C10D3D4F8D00061680C4B243198474C
:10197000D4F8F8309D4238BFC4F8F850FFF716FF8E
:101980000028D4D038BDD4F8D4006168034B24318A
:101990009847C9E70000002075A505083DA5050882
:1019A000154BD3F8EC202AB11EE0D3F8E420013A1D
:1019B000C3F8E420D3F8E42002EB820203EB8202B6
:1019C0009268002AF1D0D3F8E4100C4A01EB8101AF
:1019D00002EB81014A6801F10800526882424A60C4
:1019E00006D0D2685A6070470122C3F8F0207047D1
:1019F00052684A60F5E700BF0000002008000020A0
:101A000070B5174C0D466168164E3831B0476068A6
:101A1000154B243098476B1C1AD0D4F8F410626828
:101A2000D4F8F4306D189D4255620BD3D4F8D00031
:101A300061682431B047D4F8F8309D4238BFC4F80B
:101A4000F85070BDD4F8D40061682431B04770BD3F
:101A5000616804F1BC002431044B984770BD00BF9D
:101A6000000000203DA5050875A5050821A505086D
:101A7000F8B5C368154CDD68154F05F138063046DA
:101A8000B847D4F8EC30D3B905F124063046B8474E
:101A9000EB6CD4F8E4200F48934288BFC4F8E430DC
:101AA00003EB830300EB830031460B4B98476368DD
:101AB000E86CDB6C984234BF00200120F8BD04F1D3
:101AC00094003146044B9847F1E700BF0000002026
:101AD00075A505080800002021A5050840F20003AF
:101AE000C2F20003D3F8FC20D3F8F43080E80C00F5
:101AF000704700BF70B5174B0D46044698472B68DA
:101B00005A1C24D0144A2168D2F8FC00814208BF34
:101B1000616804D0D2F8F4006168814215D9D2F826
:101B2000F4000D4A401A83420FD9D2F8F460D2F87B
:101B3000FC009B1BD2F8F4205918296084E80500AA
:101B40000025064B9847284670BD0125F9E700257A
:101B5000F7E700BF559F050800000020899F050892
:101B600040F20003C2F200030122C3F8F0207047E4
:101B7000064B10B55A68904206D028B100220430B6
:101B80001346034CA04710BD5868F7E7000000203B
:101B9000F904010840F20003C2F2000358687047DC
:101BA000F8B5174CC36C62680546D26C934210D2EC
:101BB000626804F10806D16C03EB8303426B06EB09
:101BC0008303C1F105019A42816303D06368DB6C32
:101BD000C364F8BD00F1240738460A4B9847636890
:101BE000D4F8E420DB6C3946934203EB8300EB64CA
:101BF00088BFC4F8E43006EB8000034B9847F8BD7B
:101C00000000002075A5050821A5050838B5044683
:101C1000E0B1C26C436E9A4218D000F12405284608
:101C20000B4B98470B4A636ED2F8E410C3F10500E2
:101C30008B42A0630848E36488BFC2F8E43003EB3A
:101C4000830300EB83002946044B984738BD00BF4F
:101C500075A50508000000200800002021A5050842
:101C6000430710B50B4B04461CBF20F00704083493
:101C70009847094A1368E418B4F5C04F08D2A34244
:101C800006D21460054CE418054B9847204610BD59
:101C90000024F9E72D160108401500204815002002
:101CA000AD170108704700BF41F24053C2F2000374
:101CB00000221A60704700BF41F24053C2F2000395
:081CC0001868C0F5C040704730
:105CC8002DE9F0478AB004460D4600F04DF8DFF89C
:105CD80094A09AF90030013306460F460FD02046AB
:105CE800294600F007F950B14FF000084FF00009BD
:105CF8002046294642464B4607F0A6FC20B93046C6
:105D080039460AB0BDE8F08701230093144B9AF88E
:105D18000060CDE9044501930023CDE902450893CD
:105D280056B9CDE90689684600F00CF970B1089BB0
:105D38008BB9DDE90667E2E74046494642464B46ED
:105D480007F03AFB022ECDE90601ECD100F008F984
:105D580021230360EBE700F003F9089B0360E8E701
:105D680044C30608080300202DE9F8430027B94674
:105D7800C7F6F077C7F6F0790F404F4504460D4651
:105D880002460B460E46804600F09980002976DDD3
:105D98005FEA215C00F0818026F07F43ACF2FF3C93
:105DA80023F470031CF0010F43F480131CBF4FEA67
:105DB800D8724FEA48084FEA6C0C18BF02EB43034D
:105DC80000274FEAD872162402EB430338464FEAFD
:105DD80048024FF400114518D60F9D424FEA42027F
:105DE800DEBFC5EB030368187F184908013C06EBC2
:105DF8004303F0D12026A0464FF000410EE0814633
:105E08001B1A954288BF013B521B64184846D50FA0
:105E180049085200013E05EB430315D0984201EBB7
:105E2800080503DB954298BF8342F0D105F000498D
:105E380005EB0108B9F1004FE1D1B8F1000FA8BF97
:105E480000F10109DCDADAE7134310D166087B10A8
:105E5800FA0703F17F5348BF46F0004603F50013E5
:105E6800344603EB0C5520462946BDE8F883611CEF
:105E78001CBF04F001031C19E8D10137E7E721F042
:105E880000460643EFD049BB8C464FEAD826ACF112
:105E9800150C4FEA4858002EF7D016F4801319D184
:105EA80076000133F002FBD5C3F10101C3F12002F2
:105EB80028FA02F28C44164308FA03F86CE707F054
:105EC80051F902460B462046294606F099FF04463A
:105ED8000D46C8E7202201210023E9E702460B46C8
:105EE80006F08CFF02460B4607F066FA04460D469C
:105EF800B9E700BF50EA010201D102207047D0F192
:105F0800010238BF0022B1F1004F08BF0028F4D0C9
:105F180021F000434FF6FF71A3F58010C7F6DF713B
:105F2800884201D804207047B3F5801F01D20320AE
:105F380070470020C7F6F070834214BF002002F0BB
:105F48000100704700207047002101F05BBD00BFD1
:105F580000210A2201F018BE00220A2301F074BDB4
:105F680040F21033C2F20003186870470F2AF0B4E9
:105F780040D941EA00039B073ED10C46034615462B
:105F88002668103D1E6066685E60A6689E60E668CA
:105F98001034DE6010330F2DF2D8A2F1100502F094
:105FA8000F0425F00F051035032C00EB05032944D9
:105FB80024D9A4F1040C1D460C464FEA9C0C01EBB5
:105FC8008C07043754F8046BBC4245F8046BF9D1CC
:105FD8000CF1010402F00302A40009191B193AB1DB
:105FE80001399A1811F8014F03F8014B9342F9D17E
:105FF800F0BC70470346F2E70346F1E72246EEE7B6
:1060080070B48407034644D0541E002A3FD0CEB251
:1060180002E0002C3BD0144603F8016B13F0030F89
:106028001D4604F1FF32F4D1032C29D9CAB20F2C32
:1060380084BF2B46264642EA022242EA024211D98E
:10604800103E1A605A609A60DA6010330F2EF7D843
:10605800A4F1100304F00F0423F00F031033032CF2
:106068001D440DD92E462346043B46F8042B032B2A
:10607800FAD8231F04F0030423F003030433ED18B4
:106088002CB1C9B22C1905F8011BA542FBD170BC73
:10609800704705461446C7E740F210330022C2F2A3
:1060A80000031B68C3F8A800C3F8AC20704700BF02
:1060B80040F210330122C2F20003F0B44FF22D4730
:1060C8001E6847F62D74C5F65107C4F6954400239B
:1060D800D6F8A850D6F8AC1007FB05F704FB0177F3
:1060E800A5FB044512193D4443EB0503C6E92A23E1
:1060F80023F00040F0BC70470CB4F0B59DB022AC62
:106108000E4602A96FF0004554F8042B4FF40277AD
:1061180004952346079502964FF6FF75ADF814705F
:106128000696ADF81650019401F03CFD029B002242
:106138001A701DB0BDE8F04002B070470EB440F2CE
:106148001033F0B59CB021ACC2F20003064602A998
:1061580054F8042B6FF0004518684FF40277234673
:10616800049507954FF6FF750296ADF814700696DC
:10617800ADF81650019401F015FD029B00221A702B
:106188001CB0BDE8F04003B0704700BF41EA00030F
:106198009B0710B414D10B68A3F1013222EA030261
:1061A80012F0803F0CD10A1D40F8043B114652F80A
:1061B800043BA3F1013424EA030414F0803FF3D034
:1061C8004A1E12F8013F00F8013B002BF9D10138B3
:1061D80010BC7047830770B5064614D10368A3F155
:1061E800013222EA030313F0803F0CD1031D1A4643
:1061F80053F8044BA4F1013525EA040414F0803F58
:10620800F5D0104600E0304603782BB1431C184601
:1062180001330478002CFAD100F070F9304670BDD3
:10622800C9B2F0B400294BD083070FD00378002BF4
:1062380073D0994242D0431C05E013F8012B002A81
:106248003BD091423AD09A071846F6D1036841EA02
:106258000127A3F1013247EA074722EA030212F0B5
:10626800803F1CD17B40A3F1013222EA030313F0E3
:10627800803F14D1021D02E014F0803F0FD1104678
:1062880052F8043BA3F1013687EA030426EA030324
:10629800A4F1013513F0803F25EA0404ECD003781B
:1062A800002B3AD0994209D0431C01E0914205D015
:1062B800184613F8012B002AF8D11046F0BC704795
:1062C80081070DD00378002BF8D0431C02E0027838
:1062D800002AF3D013F0030F184603F10103F6D197
:1062E8000368A3F1013222EA030313F0803F0AD1C5
:1062F800021D104652F8041BA1F1013424EA0101E1
:1063080011F0803FF5D00378002BD7D0431C1846F6
:1063180001330278002AFAD1D0E71846CEE700BF49
:1063280080EA010212F0030F40F03A8010F00302F5
:1063380020F0030021F0030150F804CB08BF51F806
:10634800043B0DD082F003024FEAC2026FF07F4394
:1063580023FA02F251F8043B4CEA020C43EA020326
:10636800ACF101329C4501BF22EA0C0212F0803FD9
:1063780050F804CB51F8043BF2D04FEA0C604FEAD6
:106388001C2C012828BFB0EB036F08BF1B0AF4D0F0
:1063980003F0FF034FEA1060A0EB0300704700BF53
:1063A80010F0030F0AD010F8012B11F8013B012A55
:1063B80028BF9A42F4D0A2EB030070474DF8045D61
:1063C8004DF8044D4FF0010242EA022242EA02422D
:1063D80001F0030C21F0030150F8044B51F8045B61
:1063E800BCF1020F26D04BD824F07F4CBCEB152F04
:1063F800A4EB020323EA04030DD113EAC21308BF76
:1064080051F8045B0AD18CEA040CBCEB056F0CD183
:1064180050F8044BE8E74FEA15255CE033F07F437A
:1064280052D10D784FEA146C55E04FEA146C05F020
:10643800FF0550E04FEA044CA4EB02034FEA1C4C62
:1064480023EA0403BCEB154F17D113EAC21308BFA4
:1064580051F8045B07D18CEA040CBCEB054F08D15A
:1064680050F8044BE6E71B042ED10D884FEA144C74
:1064780031E04FEA05454FEA144C4FEA15452AE04A
:1064880004F0FF0CBCEB156FA4EB020323EA040332
:106498000DD113EAC21308BF51F8045B0AD18CEA84
:1064A800040CBCEB052F0AD150F8044BE8E74FEA7F
:1064B800156510E014F0FF0F06D051F8045B4FEAA1
:1064C800142C25F07F4506E04FF000005DF8044BE2
:1064D8005DF8045B70470CF0FF0205F0FF0001282F
:1064E80028BF904204BF4FEA1C2C2D0AF3D0A2EB20
:1064F80000005DF8044B5DF8045B704780EA010218
:10650800844612F0030F4FD111F0030F32D14DF82A
:10651800044D11F0040F51F8043B0BD0A3F10132E4
:106528009A4312F0803F04BF4CF8043B51F8043BF7
:1065380016D100BF51F8044BA3F101329A4312F06F
:10654800803FA4F101320BD14CF8043BA24312F076
:10655800803F04BF51F8043B4CF8044BEAD0234673
:106568000CF8013B13F0FF0F4FEA3323F8D15DF825
:10657800044B704711F0010F06D011F8012B0CF8ED
:10658800012B002A08BF704711F0020FBFD031F865
:10659800022B12F0FF0F16BF2CF8022B8CF80020EC
:1065A80012F47F4FB3D1704711F8012B0CF8012B6F
:1065B800002AF9D1704700BF20F0030110F0030052
:1065C800C0F1000051F8043B00F1040C4FEACC0C78
:1065D8006FF000021CBF22FA0CF213434FF0010CBB
:1065E8004CEA0C2C4CEA0C4CA3EB0C0222EA0302FA
:1065F80012EACC1204BF51F8043B0430F4D013F073
:10660800FF0F1FBF013013F47F4F013013F47F0FCA
:1066180018BF0130704700BF41EA000313F0030FB1
:10662800034670B425D0AAB10C78013A03F8014B9F
:106638004CB11C4672B111F8015F013A04F8015BD4
:106648002346002DF6D12AB19A18002103F8011B20
:106658009342FBD170BC70470E4651F8044BA4F12D
:10666800013525EA040515F0803F05D1043A43F8C1
:10667800044B032AF0D8D6E73146D4E72DE9F007D2
:1066880001273C4600254FF0FF36631900EB060C46
:106698008B420DD21CF804C010F80380E0452ED2BE
:1066A80001241D469F1B63198B4200EB060CF1D396
:1066B8004FF0010A002554464FF0FF3C176063195C
:1066C80000EB0C0899420ED918F8048010F80390D2
:1066D800C1451AD901241D46CCEB030A6319994216
:1066E80000EB0C08F0D80CF101000136B0423CBFB9
:1066F800BA463046C2F800A0BDE8F00770470BD094
:1067080001272E463C46ED19BFE709D04FF0010A94
:10671800AC4654465544D2E7BC4205D00134B4E7F0
:10672800544505D00134CAE727461D460124ACE785
:10673800A2461D460124C2E72DE9F04FADF2244DD3
:10674800164680460D461046194607AA1C46FFF70E
:1067580095FF07AB0DF21C42039043F8044F934298
:10676800FBD1671E002308A834B1F25CF91A013383
:10677800A34240F82210F8D107993046039A7118BD
:1067880004F03CFB00287FD1DDF80CC02A46824685
:10679800671E0CF1FF3CCDF808C0B444CDF814C016
:1067A800DDF80CC005460194CCF1010CCDF810C001
:1067B80009E02DB1079A93423CBF0199C2EB01034E
:1067C8009A4400252246019B08EB020000210AEBAF
:1067D8000304A21A04F0C8FA00284FD1002C4DD0A7
:1067E80008EB040308A913F8013C51F82330002BE7
:1067F800DFD1039A954228BF2A46BA4211D208EB44
:106808000A0316F802C0B118985C844506D02FE038
:1068180011F8010F13F802C0844529D10132BA4298
:10682800F6D3039B02989D4228BF184618D2DDF87C
:1068380008C008EB0A0316F80C1013F80C20914254
:1068480040F08680059A06EB050B06E013F801C0B8
:1068580012F8019DE14503D10846411E5A45F5D17C
:106868000135854276D8079D019BAA445D1BA9E79F
:10687800DDF810C00025E2449244A3E7002009B0E7
:106888000DF5806DBDE8F08FDDF80CC02A46DDF807
:106898000CA04FF0000BCCEB04030DF1200963456D
:1068A80038BF6346671E0133254607930CF1FF3353
:1068B8000193B444039BCDF808C0C3F101030493CA
:1068C8000BEB050408EB02000021A21A04F04CFAB5
:1068D8000028D3D1002CD1D008EB040313F8013CD5
:1068E80059F8233063BBBA4508EB0B0015D2DDF825
:1068F80008C010F80A309CF800209A4218BF534686
:1069080021D1029A534605E012F8011F10F803C07E
:106918008C4518D10133BB42F6D3019B5A1CAED02B
:10692800DDF804C016F80C1010F80C20914206D1BE
:1069380013F1FF33A3D3F15CC25C9142F8D0079BFB
:106948009B442246BCE7DDF810C0E3449B44F8E7CB
:10695800039885E708EB0A0091E700BF2DE9F04F9F
:106968008046037887B00E46002B00F0F7800A783F
:106978009AB184460131012702E011F8012B5AB17E
:10698800934214BF002707F001071CF8013F0D468A
:10699800002BF2D12B7803BB1FB1404607B0BDE8EE
:1069A800F08F08F101003178FFF73AFCAD1B012D9B
:1069B80018BF0028074608BF8046EED0A8444045C7
:1069C80094BFC0EB080401241F2D09D92146324683
:1069D8002B46FFF7B1FE8046DFE74FF00008DCE703
:1069E800294605AA3046FFF749FE05997118019016
:1069F8003046019A04F002FA002852D1019B8346DE
:106A08008046013B0093F3180393019BC3F10103F4
:106A18000293224608EB0504B8180021A21A04F0D4
:106A2800A3F90028D9D1002CD7D0019B9B4528BFBA
:106A38005B469D4213D9F918F05CF21811F808105A
:106A4800884240F0858007EB080C05E012F8011F2A
:106A58001CF8030088427BD101339D42F6D89DE89B
:106A68000A005B457DD907EB0809725C19F801300B
:106A78009A4276D1039B06EB0B0A06E019F802004E
:106A880013F801CD844503D111464A1E5345F5D16B
:106A98000BF1010B8B4566D8059B9844C3EB050B9E
:106AA800B7E701984FF0000B22462B1A06EB0009B6
:106AB80000F1FF388246834238BF03463918013354
:106AC80000910593C0F1010302930BEB0504B8187C
:106AD8000021A21A04F048F900287FF47EAF002CA8
:106AE8003FF47BAF554598BF07EB0B0014D90098CE
:106AF80099F8002010F80B309A4224D14A465346A0
:106B080007EB0B0005E012F8011F10F803C08C45D5
:106B18001AD101339D42F6D8B8F1FF3F43463FF4FE
:106B28005AAF16F8081010F80820914207D113F14F
:106B3800FF33FFF450AFF15CC25C9142F7D0059B84
:106B48009B442246C1E75346029A93449B44F8E784
:106B580002994FF0000B884498445AE70D460127E4
:106B680018E7019994E7B84417E700BF0000000050
:106B78002DE9F04F9DB08946834610924A46002081
:106B88000021CDF85C90CDE90801114612F8013BCF
:106B98002D2B40D8DFE803F03A3F3F3F3F3F3F3FD0
:106BA8003F38383838383F3F3F3F3F3F3F3F3F3F10
:106BB8003F3F3F3F3F3F3F3F383F3F3F3F3F3F3FE4
:106BC8003F3F3F353F170126129601F10108CDF8E6
:106BD8005C804B78002B21D19A4604930026CDF88F
:106BE8005C901296109D0DB1179B2B60129E1EB1E2
:106BF800049F07F100470497504604991DB0BDE86B
:106C0800F08F00271297E0E71792BEE74FF0000ACF
:106C1800CDF810A0E2E7884600251295302B00F049
:106C2800D9800026049600262F2B1D4640F3E584C4
:106C3800392B00F3E28408F101023746344601E0BB
:106C4800392B17DC0F2C0DDC07EB870006EB8601D0
:106C5800082C03EB400003EB4103D4BFA0F130073D
:106C6800A3F130061792924612F8013B01342F2BFC
:106C78001D46E5DC584603F0ADFD01685846039112
:106C880003F0A8FD0068FFF797FC039902465046F9
:106C980004F070FD8246002800F0B48000210794BB
:106CA8000A46084625F02003452B0BD1079D45EAE7
:106CB8000103049D1D4340F0CD80099EDDF820A00E
:106CC80004968BE74FF0000C079B002B3FD00799E9
:106CD8003846C2EB0C09079D002C08BF0C4606F08D
:106CE800CBF9102DA8BF1025092D02460B46CDE97A
:106CF800082313DDA04B03EBC50353E9122306F069
:106D080031FACDE90401304606F0B6F902460B46E1
:106D1800DDE9040106F074F8CDE90801079E0F2E9D
:106D280000F3F380B9F1000F4FD040F38485B9F137
:106D3800160F00F338859049DDE9082301EBC909EE
:106D4800D9E9000106F00EFA824604914AE7049E4A
:106D58000E433AD1002840F09882493D252D00F293
:106D6800F782DFE815F0FA02F502F502F502F502FE
:106D78008102F502F502F502F502F502F502F502C7
:106D8800F502F502F502F502F502F502F502F50243
:106D9800F502F502F502F502F502F502F502F50233
:106DA800F502F502F502FA02F502F502F502F5021E
:106DB8008102531C17935378282B00F0F685002284
:106DC80008921346CFF6F8730993099FDDF820A0BF
:106DD800049707E798F80130582B00F0B883782B10
:106DE80018BF08F1010200F0B2831146179212F899
:106DF800013B302BF9D08846002B00F02B8201256F
:106E0800049510E75846179D03F0E4FC0068FFF767
:106E1800D3FB2B1817932D5C002C40F0D881302D14
:106E2800214605D10133179301311D78302DF9D052
:106E3800A5F13103082B00F22D82303DDDF85C808E
:106E480040F0A1840A46404601210795431C179348
:106E58004578BFE1DDF85C9009F10103179399F8D3
:106E680001502B2D00F0CE832D2D00F069820023D8
:106E78000A93A5F13003092B84BFCDF85C904FF03D
:106E8800000C3FF621AF302D06D1179B0133179325
:106E980013F8015B302DFAD0A5F13103082B3FF62A
:106EA80011AF179BA5F1300C03F1010ACDF85CA0D6
:106EB8005D780B932F2D13DD392D11DC03F1020AB8
:106EC800534601E0392D0BDC0CEB8C0C17939A46DA
:106ED80005EB4C0C1D780133ACF1300C2F2DF1DC97
:106EE8000B9BC3EB0A0ABAF1080FC8BF44F61F6C24
:106EF80004DC44F61F639C45A8BF9C460A9B002BF4
:106F08003FF4E2AECCF1000CDEE6079E751B4D4463
:106F1800002D40F30E8415F00F010AD01648DDE964
:106F2800082300EBC101D1E9000106F01BF9CDE906
:106F3800080135F00F0540F0B1810998DDF820A06F
:106F48000B9504900097584641462246079B04F04B
:106F580009F8B9F1000F1190C0F2688400270D9765
:106F6800119E29EAE977DDE908450C360E97139654
:106F7800CDF828A076E000BFD8BA06080F9B002BF2
:106F880000F0018200270026C3F6F077AC46002007
:106F9800CDF830A0C3F6F07008904FF0000A5346C1
:106FA800C7F6F07AC7F6E0730CEA0A0A9A4500F0C9
:106FB8001C820B9DBAF1D46F8CBF00230123002DD6
:106FC80008BF0023FBB10C98A5A3D3E900230899B7
:106FD80006F044FB98B10C98089906F085FB002848
:106FE80000F0A88206F048F80C9008910F9F002F37
:106FF80040F08A82089D05F100430C9E1F4607F168
:10700800D663CAEB03070A98049904F02BFA0246E0
:107018000B463046394606F0A5F802460B460A9854
:10702800049905F0EDFE04460D468C460A9004913D
:107038000B9E3EB90023C7F6F0730CEA03039A458A
:1070480000F00A825846189903F036FF5846414620
:1070580003F032FF5846494603F02EFF5846079979
:1070680003F02AFF119E584616AF716803F0FCFE24
:10707800336913999A1C9200804600F10C00FEF7C0
:1070880075FF049B009719A80A9A0190584604F0C6
:1070980063FA01211890584603F0FEFF1699199BD0
:1070A8000029AABF0D9F0E9E7E180B9FB4BFC1EB8F
:1070B800060EDDF838E0C7EB0101B8BF0D9ECF180A
:1070C80081466FF47F7087420B98B4BF01F2334357
:1070D800C3F1360306EB030A73441F18B245B4BF65
:1070E80053463346BB42A8BF3B460D99002BC2BF4F
:1070F800C3EB0A0AC3EB0707C3EB060691B10A46BE
:107108005846494604F070F8189A81465846494648
:1071180003F0CCFF189903465846039303F0CCFEBE
:10712800039B1893BAF1000F05DD5846189952468B
:1071380004F0A4F818900E9A22B14146584604F07B
:1071480053F88046002F05DD414658463A4604F07C
:1071580095F88046002E05DD49465846324604F02B
:107168008DF881461899424658464FF0000A04F0B7
:1071780003F94946C668C0F80CA007900F9604F0BA
:10718800DDF85045C0F2418200F0918207984946E7
:1071980004F03CFA00224FF0804306460F4606F002
:1071A8005DFA00287FF4EAAE00233946C3F6E0739F
:1071B8003046002205F0D6FF0F9F0C9001F10043E6
:1071C800089107B1089B0C9EAC461F46E5E6514660
:1071D80052460794A5F130030120092B3FF662AD12
:1071E80001F1010C1D4617986146002B3FF42EAEA5
:1071F800012900F0D883079B0A9203F1010AC918F4
:107208001A4653460B94102A08DC07EB870A06EB4C
:107218008604092BD4BF4FEA4A07660001338B4224
:10722800F1D10A9A63460B9C0799102900F314833D
:107238008C44D218BCF1090FD5BF07EB870706EBC2
:10724800860605EB470705EB4606079D0021ED1866
:107258000795FBE59A460493C4E400BFAFF30080AA
:107268000000C0FFFFFFDF41AF48179A10F8011F69
:10727800134600293FF49DAD5B780132402B02DDB7
:107288005A2BD8BF20338B42F0D00998DDF820A0C4
:107298000490A3E400220120079203E5B5F59A7F44
:1072A80000F33A822D11012D40F378839F4E4FF061
:1072B800000ADDE90823049615F0010F1046194667
:1072C8004FEA65050AF1010A05D0D6E9002305F061
:1072D80049FF02460B460836012DEDDC10461946DB
:1072E800CDE90801049E099806EBCA01A0F1547083
:1072F8000990DDE90823D1E9000105F033FF0023F7
:107308000022C7F6F073C7F6A042CDE90801099933
:107318000B40934200F200820022C7F6904293424B
:1073280040F29F824FF6FF714FF0FF300E46002566
:10733800C7F6EF760B95099682460890049601E603
:1073480001250A9509F10203179399F8025090E56F
:10735800099ADDF820A0049240E47548179A10F8BD
:10736800011F1346002900F0EB825B780132402BA5
:1073780002DD5A2BD8BF20338B42F0D0099BDDF8B1
:1073880020A004932AE4AC46002C40F09D80C5F36D
:107398001303FBB90023304639460022C3F6F073C5
:1073A800039506F051F9DDF80CC0002840F0DC81A7
:1073B80000230022C3F6E0733046394605F0D2FEBA
:1073C800DDF80CC0024601F100430C900891164606
:1073D8001F46E2E50020002701460026C3F6F071AB
:1073E800CBF6F0770C900891D7E5ACF15475049B77
:1073F8000A9A20462946CDE9046716461F46CDE974
:10740800146704F02FF802460B46DDE9040105F085
:10741800A9FE02460B462046294605F0F1FC00234A
:10742800C7F6F0734FF6FF72C7F69F420B4004464B
:10743800934240F285804FF6FF73159FC7F6EF73AE
:107448009F4200F058814FF6FF754FF0FF34C7F6A2
:10745800EF750A940495F5E508990C98CDF80CC0D9
:1074680006F01AF905F018FE02460B460C98089922
:1074780005F0C4FC0F9ADDF80CC006460F467ABB2F
:1074880074BBCCF313035BBB21A3D3E9002306F041
:10749800DBF800283FF4D6ADDDF828A05846189947
:1074A80003F00AFD5846414603F006FD5846494692
:1074B80003F002FD5846119903F0FEFC584607995F
:1074C80003F0FAFCFFF78EBB012C83D1002D81D18C
:1074D8004FF0000ACDF810A02223CBF80030DDE7EA
:1074E800304639460CA3D3E9002306F0ADF800284E
:1074F800D2D1304639460AA3D3E9002306F0C2F8B0
:1075080000283FF49FADC7E7089B76E5AFF30080FE
:107518009535A094FFFFCF3F9535A094FFFFDF3F3F
:1075280035E5AF350000E03F5BC30608C8BB060879
:107538004FC3060800260C90C3F6F076089655E56A
:1075480001F1547C0A906546CDF810C070E5129E92
:1075580018ABA34D5846009317A901962A4619ABB4
:1075680002F07EFD10F00706044604BFB246CDF8CF
:1075780010A03FF437AB062E00F00C81189A3AB1F0
:1075880029681AA804F090F85846189903F094FC52
:10759800013E199B042E0AD8DFE806F0241F1903C0
:1075A80024006FF000464FF0FF370996089723072D
:1075B80055BF09980999DDF820A041F0004B52BF4A
:1075C8000490DDF820A0CDF810B0FFF70BBB002326
:1075D8001D46C7F6F0750995E9E71A981B990890B2
:1075E8000991E4E71A9A03F2334308921B9A22F4AA
:1075F800801242EA03520992D9E7C2463746344616
:10760800FFF738BB00230A939CE6CDE908457EBB0B
:10761800089F6FBBC5F3130353BB5346C7F6F073FC
:107628002B40B3F1D66F23D9079D6B6913B92B692A
:10763800012B1DDD01220799584603F01FFE49461C
:10764800079003F07BFE002812DD0B9D002D40F013
:107658009481099E26F000431B0D1B05A3F580139A
:107668004FF0FF3008906FEA13536FEA0353099302
:107678000B9D002D00F08280002714973A46DDE923
:107688000801C3F650121592DDE9142305F06AFDCE
:107698000F460646CDE908678246099F0491002FE8
:1076A8007FF4FCAE089800287FF4F8AE14E70F9E2C
:1076B800CDE90845DDF828A0002E00F095804FF6AA
:1076C800FF7225F07F4121F47001C0F20F02914250
:1076D8002B46089900F0CF80CB07C9D550460499AE
:1076E80003F0C0FE02460B465046049905F088FB9D
:1076F800CDE90801BCE7149801307FF4A4AE00225C
:10770800089213469246C7F6F0730993099E2223FE
:10771800CBF800300496C1E6002622233746CBF882
:107728000030C7F6F07708960997B2460497FFF736
:1077380059BA3FF402AC6D4215F00F030AD0294A3A
:10774800DDE9080102EBC303D3E9002305F034FEA9
:10775800CDE908012D1140F0AC800999DDF820A091
:107768000B950491FFF7EEBB0F9A00231E46CBF64C
:10777800E073C3F6E07608960C9228E6099EDDF8D9
:1077880020A004968AE601230A46404600219C462A
:10779800079149E54FF0000A08F10103CDF810A060
:1077A8001793FFF71FBA079EC6F1250399453FF7C0
:1077B800ACABC6F10F0A0B4CCAEB0909DDE908238B
:1077C80004EBCA0104EBC904D1E9000105F0CAFCC5
:1077D800D4E9002305F0C6FC82460491FFF702BAFB
:1077E80040070020D8BA06080999C1F31303002BF3
:1077F80035D1089B002B3FF428AFDA077FF538AF67
:107808005046049903F02EFE02460B465046049952
:1078180005F0F4FA02460B46CDE9082300220023BE
:1078280005F008FF00287FF453AE21E7C9F10005F1
:107838000D95FFF795BB19F1160FFFF666AB6C4B6C
:10784800DDE90801A3EBC909D9E9002305F0B4FD76
:1078580082460491FFF7C6B90021FFF7F7BA089BE3
:10786800CBE701F15471002509910B950491DDF8DE
:1078780020A0FFF767BB0B9F002F7BD00022C7F625
:10788800F0722A40B2F1D46F74D8120D4FF0FF3065
:10789800C2F16B0200FA02F291427FF41DAF00229E
:1078A8000020C7F6F07208901A4002F5801209927B
:1078B800DEE61F2D3BDC15F0100F14BF6A260026EC
:1078C800002D0B9614DD4B4EDDE9082315F0010F52
:1078D8001046194605D0D6E9002305F043FC0246B8
:1078E8000B4608366D10F1D110461946CDE908014E
:1078F8000B9D7DB1099AC2F30A53C3F16B03002BA8
:1079080008DD1F2B63DD0021342B089167DD4FF064
:107918005C720992089E0022099D00233046B246F7
:107928002946049505F086FE00283FF40BAB4FF07E
:10793800000A2223CDF810A0CBF80030FFF752B987
:107948002D4C1146179214F8010F0B4618B35B78AB
:107958000131402B02DD5A2BD8BF20338342F2D0AD
:1079680001321792002508952E46C7F6F07609963B
:10797800FFF72BBA4FF0FF328EE7099F27F000433D
:107988001B0D1B05B3F1D66F3FF668AEB3F15C7FF4
:107998003FF672AE9CE501311791E3E7174D4FF0C2
:1079A800000A04959EE40B463EE417A814491AAA57
:1079B80002F000FE05287FF402AA1B9B1A9943F0E7
:1079C800FF4343F4E00309930891FFF7FEB94FF032
:1079D800FF32089D02FA03F31D4008959AE74FF01D
:1079E800FF31203B01FA03F31340099392E700BFEC
:1079F800D8BA060880BA060853C30608C8BB0608E2
:107A08005407002040F210330A46C2F20003014630
:107A18001868FFF7ADB800BF38B50A46094B0146EC
:107A28001868FFF7A5F804460D46FEF763FA20B17B
:107A38002046294605F078FE38BDBDE8384003F0F9
:107A480095BE00BF100300202DE9F04F85B0994680
:107A58000B4602914B490390D1F800801C4614F85C
:107A6800015B08EB05012346497801F00801C9B21A
:107A78000029F3D12D2D7BD02B2D05BF24460B4695
:107A88000B4614F8015B39F0100112D1D9F101004D
:107A980038BF0020302D04D058B14FF00A09CB462A
:107AA80008E0217801F0DF01582965D008B14FF0CE
:107AB8000809CB46002B59460CBF6FF000464FF023
:107AC80000468DE80C003046002705F083F9304663
:107AD8008A46594605F050F8BC469DE80C0016E069
:107AE800303DA94525DD844594BF0021012151EA97
:107AF800D77729D15545D4BF00210121844518BF26
:107B0800002109BB0BFB0C5C012714F8015B08EB97
:107B18000501497801F00406F6B2002EE0D111F013
:107B2800030106D0012914BF572137216D1AA94531
:107B3800D9DC791C0BD0C3B9604612B197B9029B46
:107B4800136005B0BDE8F08F4FF0FF37DDE703990C
:107B5800002B0CBF6FF000404FF0004022230B6059
:107B6800002AEED0013C0294E9E7CCF1000CE3E7EF
:107B780014F8015B012386E74FF010096578CB46BE
:107B8800023497E70C03002030B440F21034C2F2FC
:107B980000040D46134601462A46206830BCFFF70C
:107BA80053BF00BF2DE9F04FC5B0894614460F9367
:107BB800099002F00FFE00230022CDE91823006887
:107BC8001790FEF7F9FCB9F80C3003F080031BB2EC
:107BD8001A9023B1D9F81030002B00F0C0870DF1AE
:107BE800D00ACB46D046D1460DF1CF050023C5EBD0
:107BF8000A06109307950A941C931B930C931D96E1
:107C0800CDF89CA0299328930A9D2B78252B18BF83
:107C1800002B00F0BC806A1C164601323378252BF5
:107C280018BF002BF8D10A9D771B11D0289C0A9801
:107C38000134299D072C89E881003D442894D8BF48
:107C480009F10809299500F382800C9DED190C951E
:107C58003378002B00F0F08601364FF0FF342020F7
:107C68002B21354600230A960D938DF87B30089317
:107C780015F8013BA3F12002582A00F25381DFE8EE
:107C880012F06401510151010C02510151015101DD
:107C980051015101510111028800510161006C012B
:107CA800510187018C018C018C018C018C018C01A4
:107CB8008C018C018C01510151015101510151017B
:107CC800510151015101510151019D0153025101CD
:107CD80053025101510151015101880251015101D1
:107CE800D20151015101510151015101310251019A
:107CF800510121025101510151015101510151011B
:107D080051015101510151014202F801530253023C
:107D180053020702F8015101510159005101C601EE
:107D2800E5018D02590051018B00510108015101F3
:107D38005101B201089E46F01006089698E776426F
:107D48000F930D96089E46F00406089690E709984A
:107D5800594627AA03F064FD48B9D14675E7099842
:107D6800594627AA03F05CFD002800F0F882D9469E
:107D7800B9F80C300C9D03F040031BB2002B18BF60
:107D88004FF0FF350C950C9845B0BDE8F08F0A9E72
:107D98005EE78DF87B106BE70F9E0A9500258DF83E
:107DA8007B5036680F9815931196061D1199002976
:107DB80000F06687002C1198C0F22B8729462246CE
:107DC80002F0D2FF002800F0CA8711991295401AD4
:107DD8000E90A04240F33C860F9624EAE475129E6A
:107DE8009DF87B300B950E94169613B10B9E0136B9
:107DF8000B96089B13F00203139302D00B9D0235D8
:107E08000B95089E16F08406149640F0DE810D9DB1
:107E18000B982E1A002E40F3D881102E299D40F37E
:107E280006874FF01008289CA44F02E0103E102E41
:107E380016DD01341035072C89E88001289409F1F2
:107E480008092995F2DD0998594627AAD14603F071
:107E5800E7FC00288BD1103E299D102E289CE8DCD9
:107E68000134C9F80070072CC9F804603544289417
:107E78002995D8BF09F1080940F3A88109985946FE
:107E880027AA03F0CDFC00287FF471AF299DD146C5
:107E98009CE1089E0A95F006159340F12D810F9DEF
:107EA8002B6804350122191C0F9518BF01210020E9
:107EB8008DF87B00002CA2BF089D25F08005089551
:107EC800002C18BF41F00101C9B2002900F0B782A7
:107ED800012A00F0F783022A0DF1CF0200F0E483B3
:107EE80003F0070110463031013ADB080170F7D181
:107EF800089E1190F50740F10684302900F0A68607
:107F0800C2EB0A0611920E96302200F8012C0E9D43
:107F180000269DF87B30A542B8BF254612940B95E4
:107F2800169662E70A951593002B00F085850125C2
:107F38008DF8A8302AAE00230B950E958DF87B306E
:107F4800119600261296169653E79DF87B30002B63
:107F58007FF48EAE8DF87B008AE615F8013B2A2B5C
:107F680000F07287A3F130020024092A3FF682AE9E
:107F78002E46002416F8013B04EB840402EB44046B
:107F8800A3F13002092A3546F4D944EAE47471E6CB
:107F9800089E46F0800608966AE62E460022A3F15F
:107FA800300C16F8013B02EB8202A3F1300735468C
:107FB800092F0CEB4202F2D90D925BE6089E0A9556
:107FC80046F010060896089D1593EE0656D50F9EA6
:107FD800336804360F96002BC0F27A840CBF002158
:107FE8000121012266E70A95354D15931C95089DD8
:107FF800EA066ED50F9E336804360F96089EF6077C
:1080080000F1BD83191C18BF012102224FE70A9510
:10801800089DED0640F1A2840F9E0C9D336804363E
:108028000F961D60F0E50A95089D159345F010051B
:108038000895089E16F010020ED00F9D00222B689E
:1080480004350F95991A18BF012130E7089E0A9543
:1080580016F010021593F0D1089E16F0400100F0BA
:1080680073840F9D2B8804350F95191C18BF0121A7
:108078001DE70A95089D1593EE06A8D4089D6D0680
:1080880040F179840F9EB6F9003004360F96A2E7C6
:10809800089E46F040060896EAE5089E46F0010666
:1080A8000896E5E50F9E36680D960F9E331D0D9ECA
:1080B800002EFFF644AE0F93DAE500BFA8BA060813
:1080C80070C306080A95089DA74EEA0615931C96E4
:1080D80090D4089D6B0640F131840F9E3388043696
:1080E8000F968BE70A95089D159345F0100508959E
:1080F800089EF0063FF5D3AE089E710640F10D8448
:108108000F9D2B88CDE6159300220F9B0A9501251C
:108118001E1D0B951B680E952AAD0F968DF87B20BA
:1081280011958DF8A8300CE70A950F9D1593E91D58
:1081380021F0070101F108060F9691E8C0003046CA
:108148003946CDE9180130463946FDF7D3FE0128F6
:10815800304640F0C78300220023394605F074FA00
:10816800002840F0BE859DF87B3003250B95089DBF
:1081780000267E4A25F080057D490895159D1296B2
:108188000326472DD8BF11460E9611910026169644
:108198002BE6089E46F00806089669E50F9B7820AE
:1081A8000A9530221D1D0F951B68724D089E8DF88B
:1081B8007C200222191C46F002068DF87D0018BFAB
:1081C800012108961C95159071E6299D9DF87B3034
:1081D8008BB1289C0DF17B03C9F8003001230134D1
:1081E800C9F80430072C1D442894D8BF09F10809A0
:1081F800299500F3F581139B83B1289C1FABC9F81F
:10820800003002230134C9F80430072C1D44289497
:10821800D8BF09F10809299500F3ED81149E802E35
:1082280000F0218112980E9BC61A002E3ADD102EFE
:10823800289CD8BF504F1EDD4FF010084E4F02E06B
:10824800103E102E17DD01341035072C89E8800107
:10825800289409F108092995F2DD0998594627AAB1
:10826800D14603F0DDFA00287FF481AD103E299D48
:10827800102E289CE7DC0134C9F80070072CC9F8D7
:108288000460354428942995D8BF09F1080909DD07
:108298000998594627AA03F0C3FA00287FF467AD66
:1082A800299DD146089EF3056AD4289C0E9B01346B
:1082B800119E072C1D44C9F80430C9F8006029959F
:1082C800289400F37E8109F10809089E73073BD5BD
:1082D8000D980B99461A002E36DD102E289CD8BF13
:1082E800264F1EDD4FF01008244F02E0103E102EDE
:1082F80017DD01341035072C89E88001289409F12D
:1083080008092995F2DD0998594627AAD14603F0AC
:1083180087FA00287FF42BAD103E299D102E289C4B
:10832800E7DC0134C9F80070072CC9F8046035444B
:108338002894299508DD0998594627AA03F070FA68
:1083480000287FF414AD299D0C9E0B990D9881424D
:10835800ACBF761836180C96002D7FF400AD0023BC
:10836800D146289350E400BF8CC1060860C30608B4
:1083780064C3060870C30608B8BA0608A8BA06088F
:10838800159E652E40F3B280DDE918010022002316
:1083980005F050F9002800F03D81289C0123C9F818
:1083A800043001350134994B072CC9F80030D8BF87
:1083B80009F108092995289400F3E382209B109E6F
:1083C800B34203DB089EF6077FF57FAF1A9E289C11
:1083D800AD19179E0134072CC9F800601A9EC9F818
:1083E8000460D8BF09F108092995289400F3A983E6
:1083F8001098461E002E7FF768AF102E289CC4BF29
:108408004FF01008824F04DCCFE0103E102E40F3EE
:10841800CD8001341035072C89E88001289409F1B2
:1084280008092995F1DD0998594627AAD14603F08C
:10843800F7F900287FF49BAC299D289CE5E7002AE2
:1084480040F0CA80089EF1075CBF0E92CDF844A0A8
:108458007FF55DAD1D9D30230DF1CF068DF8CF3032
:1084680011960E9553E50D980B99461A002E7FF735
:10847800D9AE102E289CD8BF654F1EDD4FF01008CE
:10848800634F02E0103E102E17DD01341035072C23
:1084980089E88001289409F108092995F2DD0998ED
:1084A800594627AAD14603F0BBF900287FF45FACF0
:1084B800103E299D102E289CE7DC0134C9F8007075
:1084C800072CC9F80460354428942995D8BF09F1C8
:1084D80008097FF7A7AE0998594627AA03F0A0F91B
:1084E80000287FF444AC299DD1469BE6109E289C29
:1084F800012E3EDD119E013401350123072CC9F8F8
:108508000430C9F80060D8BF09F1080629952894F5
:1085180000F3C68101341A991798072C0D4471602D
:1085280030602894299500F3C7810836DDE91801E1
:108538000022002305F07EF8002840F0E980109A18
:1085480001341198531E7360421C072C32601D447D
:10855800289429951DDC083601341B98072C23AB79
:10856800054433607060299528942ADC06F10809CF
:10857800ABE6089EF207BDD40134119E01350123F4
:10858800072CC9F80430C9F800602995289440F3ED
:10859800E3820998594627AA03F042F900287FF494
:1085A800E6AB5646299D289CD6E7194F0134C9F8F1
:1085B8000070072CC9F804603544289429957FF782
:1085C80082AE0998594627AA03F02AF900287FF4B1
:1085D800CEABD146299D78E60E91CDF844A096E41D
:1085E8000998594627AA03F01BF900287FF4BFAB66
:1085F800299DD146FFE50998594627AA03F010F9A5
:1086080000287FF4B4AB299DD14607E6A4C106082B
:10861800B8BA0608209E002E40F3BE81109E169818
:1086280011998642A8BF0646109A002E11440E9151
:108638000FDD289CAD19119A0134C9F80460072C84
:10864800C9F80020D8BF09F108092995289400F332
:10865800F282169B26EAE6769E1B002E40F3B9802E
:10866800102E289CD8BFB24F40F39C804FF01008C2
:10867800AF4F03E0103E102E40F3948001341035C4
:10868800072C89E88001289409F108092995F1DD6A
:108698000998594627AAD14603F0C2F800287FF462
:1086A80066AB299D289CE5E71C9D03F00F00114649
:1086B800013A1B09285C0870F7D1C1EB0A05119132
:1086C8000E9524E4092B08D81D9D30330DF1CF06F3
:1086D8008DF8CF3011960E9519E44CF6CD450DF175
:1086E800CF01CCF6CC45A5FB030208460139D208D8
:1086F80002EB8206A3EB4606134606F1300202702F
:10870800002BF0D11190C0EB0A030E93FFF7FFBBCB
:10871800109901F1FF38B8F1000F7FF71DAFB8F1DC
:10872800100F834FC8BF4FF0100905DC1DE0A8F1FA
:108738001008B8F1100F18DD013486E880021035F2
:108748000836072C28942995F1DD0998594627AA57
:10875800564603F065F800287FF409ABA8F1100825
:10876800299DB8F1100F289CE6DC013486E88001C9
:10877800072C4544289429957FF7EDAE09E719465B
:108788000222002B3FF493AB159D3022089E012155
:108798008DF87C20022246F002068DF87D5008965E
:1087A800FFF785BB0134C9F80070072CC9F80460CD
:1087B800354428942995D8BF09F1080909DD099895
:1087C800594627AA03F02CF800287FF4D0AA299D3F
:1087D800D146209B109A11981699934200EB0106F6
:1087E80042DB0898C1073FD40E981099871BCB1A13
:1087F800BB42B8BF1F46002F0EDD289CED19C9F8F3
:1088080000600134C9F80470072C29952894D8BF52
:1088180009F1080900F3268227EAE7769E1B002E55
:108828007FF753AD102E289CC4BF4FF01008404F5F
:1088380004DCBAE6103E102E7FF7B8AE01341035CE
:10884800072C89E88001289409F108092995F1DDA8
:108858000998594627AAD14602F0E2FF00287FF47A
:1088680086AA299D289CE5E7289C1A990134179A1D
:10887800072C0D44C9F80410C9F80020D8BF09F125
:10888800080929952894AFDD0998594627AA02F0C6
:10889800C7FF00287FF46BAA209BD146299DA3E738
:1088A8000998594627AA02F0BBFF00287FF45FAA5F
:1088B800299D5646289C2DE60998594627AA02F074
:1088C800AFFF00287FF453AA299D5646289C2DE621
:1088D8005B42191C18BF01212D228DF87B20012233
:1088E800FFF7E8BA3946FDF705FB002840F0BA80E3
:1088F8000325089E0B950F4A26F080060E49159D04
:1089080008960326472DD8BF114612909DF87B3054
:1089180011910E961690FFF768BA0F9E01223368E0
:1089280004360F96191C18BF0121FFF7C0BA00BF03
:10893800B8BA060868C306086CC306080F9D2B68FA
:1089480004350F95FFF75ABB0F9E0A463368043665
:108958000F96191C18BF0121FFF7A9BA0F9D089E91
:108968002B68043516F0400F0C9E0F9514BF1E801F
:108978001E60FFF749B90F9D2B6804350F95FFF767
:108988002ABB0998594627AA02F04AFF00287FF413
:10899800EEA9299DD14611E5289C0123C9F8043088
:1089A80001350134AC4B072CC9F80030D8BF09F1A8
:1089B80008092995289400F3E2802EB9109919B96D
:1089C800089AD0077FF581AC289C1A9B0134179828
:1089D800072C1D44C9F80430D8BF09F1080CC9F8A0
:1089E80000002995289400F302817642002E40F376
:1089F800ED80102E994FC4BF4FF01008DDF8249079
:108A080004DCCBE0103E102E40F3C8800134103552
:108A1800072C8CE8800128940CF1080C2995F1DDCD
:108A28004846594627AA02F0FBFED44600287FF4A0
:108A38009EA9299D289CE5E7299BD946002B3FF450
:108A480097A90998594627AA02F0EAFEFFF790B9B4
:108A58000E9B0F9623EAE37316950B939DF87B30D4
:108A6800FFF7C3B9601C00F0CF80159921F02005ED
:108A7800472D02D1002C08BF0124089A002F42F488
:108A880080721392C0F2788100201290B5F14602EC
:108A980051425141002940F0FF80452D40F06A8144
:108AA80004F101080221CDF80480324600913B46CA
:108AB80020A90998029121A9039122A9049100F003
:108AC800BFFA80441190304600220023394604F052
:108AD800B1FD50B9229B984598BF984605D93022D8
:108AE80003F8012B43452293FAD1119E472DC6EB7B
:108AF8000806109600F0FD80159E652E40F3D08183
:108B0800159D209A662D00F04A81109DAA42C0F258
:108B18003881089EF60700F1828122EAE27567260D
:108B28000B950E9215961692129D002D00F011814C
:108B3800139E2D238DF87B30002312930896FFF7A0
:108B480055B90998594627AA02F06AFE00287FF409
:108B58000EA9299DD1464BE409F10806FCE40998C1
:108B6800402101F049FEC9F80000C9F810000028AA
:108B780000F098814023C9F81430FFF730B80998FD
:108B8800594627AA02F04CFE00287FF4F0A8209E40
:108B9800D146299D002E7FF417AF0FE70134CCF89A
:108BA8000070072CCCF80460354428942995D8BF68
:108BB8000CF1080C0ADD0998594627AA02F030FE84
:108BC80000287FF4D4A8299DD446289C119E0134FE
:108BD800072CD8BF0CF10809CCF80060109E35446A
:108BE800CCF80460289429957FF76FABE9E40998DD
:108BF800594627AA02F014FE00287FF4B8A8209E40
:108C0800D446299D289CF0E61598062420F02005D6
:108C180033E71295FDF7D0FC0F96129E9DF87B3036
:108C2800169620EAE0750E900B95FFF7DEB8289CA3
:108C38000B4FFFF715B90998594627AA02F0F0FD1E
:108C480000287FF494A8299DD14602E5119DC5EB23
:108C58000A050E95FFF75BB9A4C10608B8BA06085D
:108C6800A8BA06080998594627AA02F0D9FD00288B
:108C78007FF47DA8209BD146109E299DF31ACBE551
:108C88000F96062C28BF06248A4E24EAE4750E9413
:108C98000B951196FFF755B9032000900DF1880E3A
:108CA80020A8324602903B4621A801940390CDF8B3
:108CB80010E00998069100F0C3F9472D0699119024
:108CC80002D1089AD30711D5119B03EB0408002998
:108CD8003FF4F9AE1B78302B00F0A980209B984414
:108CE800F1E62D238DF87B30FFF73FBA229B1B1A44
:108CF8001093209BD81C1A4602DB9C42BFF605AF96
:108D0800159D023D1595013B159D002B20938DF86F
:108D18008C50C0F2BD802B228DF88D20092B49DCA8
:108D280030228DF88E2024AA30338DF88F30109D94
:108D380023ABD31A1B93012D2B440E9340F397803A
:108D48000E9E0025169501360E9626EAE6760B96B7
:108D5800EAE6139D9DF87B300895FFF746B824EAAC
:108D6800E47512900B959DF87B300F960E94169033
:108D7800FFF73BB8022090E72D2307F10047129335
:108D880084E6002A109DD4BFC2F1020301235B19B7
:108D9800672623EAE3750E9315960B95C3E6002A1A
:108DA8005DDDACBB089EF10732D422EAE2750E9273
:108DB8000B95B8E646F267610DF19A05C6F2666151
:108DC80081FB0360DA172C46013DC2EBA00202EBDF
:108DD8008200A3EB40001346092B00F130022270F9
:108DE800EEDC0DF19B003033A842DAB204F8012C16
:108DF80053D90DF18D01234601E013F8012B83426D
:108E080001F8012FF9D144A8C4EB4002F63A8EE7E5
:108E1800013414190E9424EAE4760B9683E6531C65
:108E2800672523EAE3760E9315950B967BE6304685
:108E380000220023394604F0FDFB00287FF44EAFE2
:108E4800C4F1010320934AE70F9E331D3468002CB8
:108E5800BFF631A90F934FF0FF34FEF709BF8CB965
:108E6800089DEB070ED401260B960E965BE6089E2E
:108E780016F001037FF464AF0E9D169325EAE5759D
:108E88000B9551E602340E9424EAE4760B964AE6F2
:108E98002D225B428DF88D2040E70DF18E0246E7CA
:108EA800209B30E7099E4FF0FF350C230C9533606B
:108EB800FEF769BF84C3060870B59AB00D466946C7
:108EC8006FF00044009502944FF4027605944FF633
:108ED800FF74ADF80C600495ADF80E40FEF762FE25
:108EE800009B00221A701AB070BD00BF30B440F267
:108EF8001034C2F200040D46134601462A46206883
:108F080030BCFFF7D9BF00BF2DE9F04F8146036998
:108F180083B00D69002001919D4200F38E80EA1C08
:108F280001F11404013D09F1140892008B184A4418
:108F38001F1D59685068013103F01EFE06460028BF
:108F480041D04FF0000E424623467046A24653F8E1
:108F5800041B14681FFA81FC4FEA114BA1B206FBEF
:108F68000CEC091806FB0BFE0EEB1C4E1FFA8CFCD2
:108F7800CCEB01011FFA8EF04FEA1E4EC0EB1440F5
:108F88001FFA81FC00EB21404CEA004100149F428B
:108F980042F8041BDBD22B1D544609EB83035A68A5
:108FA8008AB91A1D98450CD252F8042C4AB9043BC8
:108FB80001E012682AB9013D98451A46A3F1040355
:108FC800F7D3C9F810504846019902F0B7F90028BC
:108FD80032DB013643464FF0000C54F8040B196895
:108FE8001FFA80FA000C8AB2C0EB1141CAEB0202E8
:108FF800A742944401EB2C421FFA8CFC4CEA024134
:109008004FEA224C43F8041BE7D22B1D09EB8303DC
:109018005A688AB91A1D98450CD252F8042C4AB9D4
:10902800043B01E012682AB9013D98451A46A3F1AC
:109038000403F7D3C9F81050304603B0BDE8F08FE9
:109048002DE9F04F9B469BB0036C07469246279C40
:1090580053B1426C0125194605FA02F59D605A6024
:1090680001F02AFF00233B64BBF1000539DB002334
:10907800236000231A46C7F6F073C7F6F0722B4038
:10908800934217D00022002350465946D04604F098
:10909800D1FA00282BD026980123289903600029AB
:1090A80000F0D680A24B03F1FF390B6048461BB095
:1090B800BDE8F08F269842F20F730360BAF1000FF3
:1090C80000F0AD80DFF8709228990029EED099F869
:1090D8000330002B00F0538209F10803289A13602B
:1090E800E4E725F000450123AB462360C1E719AB4F
:1090F80038460093524618AB01935B46C5F30A56AF
:1091080002F02AFA0B90002E40F09280DDF8608081
:109118006FF48263199E46449E42C0F24D824FF618
:109128000E4306F21242CFF6FF732AFA02F29B1B95
:1091380005FA03F0104303F09FFF013E0123139348
:10914800A1F1F87100230022C3F6F87303F056FE6C
:1091580071A3D3E9002304F005F871A3D3E9002330
:1091680003F04EFE044630460D4603F095FF6EA30D
:10917800D3E9002303F0F6FF02460B4620462946B2
:1091880003F03EFE04460D4604F086FA2946002206
:1091980000230490204604F057FA002840F0F58197
:1091A8000499162900F2EE810498524661495B46FB
:1091B80001EBC001D1E9000104F064FA002800F0D5
:1091C800038204990022129201390491C6EB080621
:1091D800B6F1010942BFC9F10009CDF81C904FF062
:1091E800000901D40020079004990029C0F2DB810E
:1091F800894400220F910C92249B092B2BD801251E
:10920800052B02DD0025043B24932498831E032BA1
:1092180023D8DFE813F04703440335031702464B0E
:10922800C5F31305454A002D0CBF914699464BE7F7
:109238002BF07F43002223F47003504643F07F5302
:10924800A6F2FF36DDF8608043F44011139279E707
:10925800DFF8EC902AE700232493002438467C6446
:1092680021464FF0FF320E9201F0FEFD0E9B259431
:109278000A930690386401200D90199B002BC0F2C8
:10928800C18004980E2800F3BD8025990A9ACB0F57
:10929800002ACCBF002303F00103264A02EBC002D8
:1092A800D2E90089002B40F04F8442464B46504695
:1092B800594604F081F8544604F0EEF9069E8246B9
:1092C80003F0EAFE42464B4603F04CFF0B460246CB
:1092D8005946204603F092FD0AF1300306F8013B97
:1092E8000A9B012B04460D465ED000230022C4F2DF
:1092F800240303F037FF0022002304460D4604F040
:1093080099F9002840F0E88406990A9A8E1C039778
:1093180001EB020B21E000BF61436F63A787D23FD7
:10932800B3C8608B288AC63FFB799F501344D33F4C
:10933800A5C10608D8BA060898C306088CC306084B
:10934800A4C1060803F00EFF0022002304460D46C0
:1093580004F070F9002840F0BD8442464B46204690
:10936800294604F029F8B24604F096F9074603F0B6
:1093780093FE42464B4603F0F5FE02460B46204656
:10938800294603F03BFD002300225E4507F1300E1D
:10939800C4F2240306F801EC06F1010604460D4662
:1093A800D0D15646BA46039F22462B462046294628
:1093B80003F026FD04460D464046494622462B4604
:1093C80004F042F9002800F03585049B3246DDF8A8
:1093D800189016F8014C0696159302E013F8014C04
:1093E8001A46531E392C40F00A859945F6D1302388
:1093F800159989F800304B460692013131220491C3
:109408001A70ABE00D99002940F0E0800C9D079C94
:10941800DDF83480B9F1000FC8BF002C09DDA14583
:10942800B4BF4B4623460798E41AC3EB0909C01A90
:1094380007900C9900291ADD0D9A002A00F0428441
:10944800002D10DD41462A46384601F0CDFE0B9A24
:1094580080463846414601F029FE0B9906463846B3
:1094680001F02AFD0B960C9B5A1B40F086840121C3
:10947800384601F011FE06460F98002805DD3146F2
:1094880038460F9A01F0B0FE06462499012940F3A8
:10949800C08000250F9B0120002B40F04C8300EB7F
:1094A800090313F01F0300F03482C3F12002042AD9
:1094B80040F34F85C3F11C030798E4189944C0187A
:1094C8000790079A002A04DD38460B9901F0D6FE6A
:1094D8000B90B9F1000F05DD314638464A4601F0D8
:1094E800CDFE0646129B002B40F0088324990A9A69
:1094F8000229D4BF00230123002AC8BF0023002B60
:1095080000F00E820A99002940F0FC8131460522BC
:109518000A9B384601F0DAFC06460B98314601F002
:109528000DFF002840F3EE81069B002504983122A8
:109538009946013003F8012B0490069338463146CA
:1095480001F0BAFCB8F1000F08D0454518BF002D4E
:1095580040F03E823846414601F0AEFC38460B9951
:1095680001F0AAFC0699002204980A70431C269A66
:109578001360289B002B3FF499AD196096E509F11B
:109588000303ABE50123129320E6049803F084FD5E
:1095980022462B4604F04EF800287FF401AE0498CA
:1095A80001380490FCE5079B002204980F921B1ACF
:1095B800414207930C911FE64FF6EE30CFF6FF704D
:1095C800801B0AFA00F0B6E51290FFE5249A012AFA
:1095D80040F3DA830A990C9A4B1E9A42A8BFC3EB50
:1095E800020506DA0C9800250F991A1A0C938918A7
:1095F8000F910A9A002AC0F2D883079C0A9B079AFF
:10960800384601219944D218079201F045FD804659
:1096180000E7BAF1000F7FF43CAFCBF313025546D5
:10962800002A7FF437AF0025C7F6F0750BEA050569
:10963800002D3FF42FAF079A09F1010901250132E6
:10964800079227E701230D932598049BC3180E93CF
:109658005A1C002A40F328830E2A8CBF002505F0E7
:1096680001050A920021172A796409D901240423E3
:109678005B00214603F1140001349042F8D9796463
:10968800384601F0F1FB06903864002D3FF4F5AD43
:109698000499CDE910AB002940F3A58101F00F0230
:1096A800A54B4FEA211803EBC20318F0100FD3E9BA
:1096B800004500F08681A14B5946504608F00F0836
:1096C8004FF0030BD3E9082303F076FECDE9080138
:1096D800B8F1000F11D0994E18F0010F2046294615
:1096E80007D0D6E900230BF1010B03F03BFD04463C
:1096F8000D4608365FEA6808EED1DDE90801224622
:109708002B4603F059FECDE90801129951B1002307
:10971800DDE908010022C3F6F07303F095FF002885
:1097280040F0DE82584603F0B7FCDDE9082303F079
:1097380019FD00230022C4F21C0303F061FB0A9AFE
:109748008246A1F1507B002A00F0BF80049B0A9E4C
:1097580015930D98002800F07581774B00210020A3
:10976800C3F6E07103EBC603069D53E9022303F039
:1097780023FE52465B4603F041FB82468B46DDE9F9
:10978800080103F089FF044603F086FC3034E4B294
:1097980002460B46DDE9080103F030FB05F8014BF2
:1097A800CDE9080150465946DDE9082303F06AFF70
:1097B800002840F0BF830021DDE908230020C3F61C
:1097C800F07103F01BFB02460B465046594603F066
:1097D80059FF002840F0E382012E40F301810699E9
:1097E800CDF858908E19DDE90889149708962E4609
:1097F80010E000210020C3F6F07103F0FFFA524692
:109808005B4603F021FF002840F0C782089A964281
:1098180000F0E38000230022C4F224035046594696
:1098280003F0A0FC00230022C4F2240382468B46E6
:109838004046494603F096FC04460D4603F02CFFCB
:10984800074603F029FC02460B462046294603F04A
:10985800D5FA07F1300452465B46E4B206F8014BEC
:109868008046894603F0F0FE42464B460028C0D0A9
:10987800159B3546DDF81890149F049306966DE6FF
:1098880001220D922599002940F317820A460E29D4
:109898008CBF002505F001050E910A91E2E6002231
:1098A8000D92D1E600200D90ECE7584603F0F4FB4A
:1098B800DDE9082303F056FC00230022C4F21C0350
:1098C80003F09EFA8246A1F1507B00230022C4F2E5
:1098D8001403DDE9080103F091FA52465B465C4641
:1098E800CDE9080103F0CEFE0646002840F0A78027
:1098F8005246DDE908010BF1004303F0A5FE0028FC
:109908006ED0B046259A0025DDF81890D24304920F
:1099180014E61C230799E4189944C9180791D0E55F
:109928000D99002940F03A8100240B9DDDF828901C
:10993800DDF818A007E000BFD8BA0608C8BB0608BB
:1099480001F0C4FA054631462846FFF7DDFA0A2237
:109958000023294600F1300B0AF804B001343846D8
:109968004C45EDDBDDF818A00A980B950025012879
:10997800ACBF82440AF1010A01220B99384601F072
:109988007DFC31460B9001F0D9FC002840F33F8262
:109998001AF8012C069902E013F8012C9A46392A84
:1099A8000AF1FF3340F074829942F5D1DDF818903E
:1099B80031230499CDF818A0013189F800300491B9
:1099C800BCE5DDE910234FF0020BCDE908237FE663
:1099D8003846294601F070FABCE5DDF85890149F26
:1099E800DDE910AB49E4049B5C42002C00F0A28145
:1099F80004F00F02A54BDDE9100103EBC203D3E924
:109A0800002303F0AFFB2411CDE9080100F08E829A
:109A18009F4D4FF0020B02460B46E60710461946CB
:109A280007D5D5E900230BF1010B03F09BFB024698
:109A38000B4608356410F0D1CDE9082365E6002609
:109A4800B04671E5731E1493149852468F495B46CD
:109A5800069D01EBC001D1E9000103F083FBCDE9CC
:109A68001601DDE9080103F017FE044603F014FBB4
:109A7800303402460B46DDE9080103F0BFF9012E38
:109A880005F8014B82468B4622D0069ABA46541EE8
:109A98009046A41900230022C4F2240303F062FBB9
:109AA8000F46064603F0F8FD834603F0F5FA0BF17E
:109AB800300B02460B463046394603F09FF908F84A
:109AC80001BFA045E6D1149B57468B468246ED1848
:109AD80000230022C3F6E073DDE9160103F090F9D4
:109AE80052465B4603F0B0FD002800F02A81DDF8FD
:109AF80018902A4615F8014C069572E40B983146E1
:109B080001F01CFC0028BFF6F1AC0B9938460A227C
:109B1800002301F0DBF90D990B90049801380490AB
:109B280041BB0E98002803DC2499022900F30D821A
:109B38000E9A0A92F8E6336906EB8303186901F076
:109B48005FFAC0F12000AAE40A98002840F070816A
:109B5800002340460022C4F21403494603F002FBE6
:109B680052465B4603F084FD0A9EB04600287FF407
:109B7800C9AED9E400230A224146384601F0A6F9C5
:109B8800249A80460E980028CCBF00230123022A7D
:109B9800D8BF0023002B40F0D4810A90002C05DDAB
:109BA80041463846224601F069FB8046002D40F0C8
:109BB8005881CDF83480069AB346DDF8349045468E
:109BC8000B9E541C0A9B0AF001000790D3180C93B3
:109BD80059463046FFF798F929468046304601F045
:109BE800ADFB59464A468246384601F0C5FB08F1A6
:109BF80030020592611E0A91C2680346002A3DD0D0
:109C0800012219463846029201F056F9029A249B1D
:109C1800134303D10798002800F07281BAF1000FAE
:109C2800C0F2C78024995AEA010103D1079B002B8F
:109C380000F0BF80002A00F33A810C9BA246059AE7
:109C48009C4204F8012C00F0498131460A22002385
:109C5800384601F03BF94D4506461BD029460A22F5
:109C68000023384601F032F949460A22002301341C
:109C78000546384601F02AF98146A9E719463046D3
:109C8800029301F05BFB029B0246BAE7D8BA0608CA
:109C9800C8BB0608294638460A22002301F016F9EF
:109CA80001340546814693E70E2A0A928CBF0023A9
:109CB800012300211D407964E2E401230E930A93F5
:109CC8002593F6E738460B990C9A01F08DFA0B901C
:109CD800FFF7CDBB039F5646DDF8189006963DE486
:109CE8000A9A002A3FF4E1AD0E9B002B7FF778AE6D
:109CF80000230022C4F22403DDE9080103F032FA4C
:109D0800CDE908010BF1010004990139159103F01F
:109D1800C3F902460B46DDE9080103F023FA0023E4
:109D28000022C4F21C0303F06BF80E9E8246A1F1D8
:109D3800507B0EE5DDE910014FF0020BCDE908017B
:109D4800E3E40021DDE916230020C3F6E07103F007
:109D580055F852465B4603F095FC00283FF440AEA8
:109D68002B46013D13F8012C302AF9D01599DDF85E
:109D7800189006930491FFF7F1BB38460B9901F050
:109D880033FA0B90FFF773BB1398002800F0888014
:109D980003F233430C9D079C31E4149F3546DDF8EC
:109DA80018902A460695FFF71CBB079B9C1A0023B0
:109DB80025E40B96002A5E46DDF814B0CDF8349001
:109DC8005C4610DD01220B99384601F057FA3146FE
:109DD8000B9001F0B3FA002840F3A180392C08F168
:109DE800310B00F08380DDF828A0DDF81890DDF84D
:109DF80034800AF801BBCDF818A0FFF79FBB15986F
:109E08000692621C0490D2B21A70FFF7A7BB03D166
:109E18001BF0010F7FF4BCAD53460AF1FF3A13F86B
:109E2800012C302AF8D0DDF818900693FFF786BB8E
:109E3800002666E54046494622462B4603F0FAFBD3
:109E480000283FF449AF1AF0010FDDF818903FF4ED
:109E580045AF0498324616F8014C06961590FFF760
:109E6800C0BAD8F80410384600F0FEFFD8F8103011
:109E780008F10C019A1C9200044600F10C00FCF752
:109E880075F838462146012201F0F8F90D9092E65E
:109E98000132DDF818901A70CDF818A0FFF74EBB04
:109EA800189B0C9D079CC3F13603FFF7A8BB0B96C4
:109EB8005E46DDF814B0CDF83490BBF1390F15D0FB
:109EC800DDF828A00BF1010CDDF81890DDF83480DE
:109ED8000AF801CBCDF818A0FFF730BB0B96C8469F
:109EE8005E46CDF83490DDF814B045E5DDF828A0DD
:109EF8003923DDF834801A4606990AF8013B4EE505
:109F08000B965E46DDF814B0CDF83490BBF1390FEE
:109F1800ECD0BAF1000FC8BF08F1310B63E77FF44A
:109F280062AF1BF0010F3FF45EAF57E74FF0020B33
:109F3800FFF7EBBB159ADDF8189006950492FFF72A
:109F48000DBB0E9B0A93FFF7DDBA0E980A90FFF738
:109F5800D9BA3FF4B6AAC3F13C03DBE4AFF30080FF
:109F680002694B112DE9F001934200F114072DDA33
:109F7800043300EB8202143211F01F0100EB83035B
:109F880003F1040C29D05C680CF104039A42C1F176
:109F9800200824FA01F438D93D461E6806FA08F666
:109FA800344345F8044B53F8044B9A4224FA01F41D
:109FB800F3D8CCEB0203053B23F00303C318183393
:109FC8001C60E4B10433DF1BBF101AE000230361F7
:109FD80000234361BDE8F0017047624584BF6346D2
:109FE8003946F3D953F8044B9A4241F8044BF9D84F
:109FF8006FEA0C039B1823F00303C3181833DF1B05
:10A00800BF100761002FE5D1E2E73B46D8E700BF64
:10A018000F4810210F4B3022D154013110F8012F75
:10A02800C9B2002AF8D10C481A216122D154013151
:10A0380010F8012FC9B2002AF8D108481A21412284
:10A04800D154013110F8012FC9B2002AF8D1704754
:10A05800ACC30608B0720120A4C306089CC3060856
:10A068002DE9F04F8BB08846A14E069209930790D0
:10A0780000F0B0FB00680290FCF79EFA029B1A18E9
:10A0880096F83030039012F801AC002B00F00981EB
:10A09800D8F800309D1C9A78302A40F0FE810333AE
:10A0A80000271D4613F8012B0137302AF9D016F87E
:10A0B80002B0DFF83C92BBF1000F00F0F5802B787E
:10A0C8004FF0000B19F80340002C00F000826A1CC6
:10A0D800144601322378F35C002BF9D199462046C7
:10A0E8000299039A01F046FBE8B12378BBF1000F0F
:10A0F80000F0C181C4EB0B0B4FEA8B020592502B89
:10A1080000F09B80702B00F098802246C8F8002051
:10A11800B9F1000F0DD0002F0CBF062700273846D5
:10A128000BB0BDE8F08FBBF1000F00F0BE812378C3
:10A13800E0E7631B4946013B072B03DD5B10013158
:10A14800072BFBDC079800F08FFEA54200F11403F3
:10A158000490089380F0DB819B46039B4FF0000836
:10A168004746C3F1010C0FE0202F5FD03A46043771
:10A1780014F8013C4C46A542F35C03F00F0303FAC4
:10A1880002F348EA030819D214F8013C04F1FF3934
:10A198005345E9D109EB0C039D42E5D818460299CD
:10A1A800039A0193CDF800C001F0E4FA019BDDF8B1
:10A1B80000C00028D8D11C46A542E5D3089B4046DC
:10A1C8004BF8048B0499C3EB0B0B4FEAAB030B6101
:10A1D8005D0100F015FF069A1468281AA04200F3E2
:10A1E8002581C0F24B81002506980599836899421C
:10A1F80000F3F680069805994368994280F2008139
:10A208005E1AB44276DCC268022A00F06F81032A23
:10A2180000F09881012A00F0868107985027049958
:10A2280000F04AFE14980023036078E74BF8048B8B
:10A238004FF00008042742469AE763782B2B00F07A
:10A24800F2802D2B00F0EA80601C4FF0000BF15CCF
:10A2580000293FF45AAF19293FF757AF437810390F
:10A26800DFF88CC0421C1CF8033093B1192B10DCAA
:10A27800023001E0192B0CDC024601EB81010130B0
:10A2880092F800C003EB4101103916F80C30002B8E
:10A29800F0D1BBF1000F00D04942059B5B18059334
:10A2A80034E7FFF7B5FEF3E628460299039A01F072
:10A2B80061FA002840F09D8003982C182B5C19F84F
:10A2C8000320002A00F0EB80302B40F00B81631C48
:10A2D8001D4613F8012B302AFAD0B35C002B40F04E
:10A2E80002814FF00109A3464F462C46F7E600BF0E
:10A2F800B0720120771E002D40F0E780002F04DDAA
:10A308000498394601F0F4F9054608997B110122B1
:10A3180007F01F070498A41B51F8233002FA07F22C
:10A3280031461A4218BF45F00205FFF719FE069B91
:10A3380002275B680593002D69D00698C368022B35
:10A3480000F0EA80032B5DD0012B5ED1AA075CD513
:10A3580008990B682B43DB0757D5049B0026049903
:10A368001D69089B01EB85001430194653F8042B2E
:10A37800B2F1FF3F40F0EB80984243F8046CF4D808
:10A38800049A93689D42B8BF2B4680F2F9800499DD
:10A3980001EB830201330B6101235361022F00F0AB
:10A3A800D98004990B699D420EDB14F01F0400F05C
:10A3B800AC80049B03EB8505286900F021FEC4F1FD
:10A3C8002003984280F2A18004980121FFF7C8FD7C
:10A3D800069A0598936801300590984240F3958055
:10A3E8000798A327049900F067FD149A00231360C7
:10A3F80095E62B782C46CDF814B04FF001097EE68F
:10A40800012798E7159B002BA7D147F01007049B5D
:10A4180014980360059B0998036080E64FF0010BD0
:10A42800A378A01C13E74FF0000BF9E7061B04986C
:10A43800314601F05DF90546A8B1731E049801255F
:10A4480003F01F015A1105FA01F100EB820252696B
:10A45800114208D0AB4205DD0498B11E01F048F95D
:10A46800032500B9022504983146FFF779FD059BBD
:10A478009B190593B8E6CDF814B040E6251A04995F
:10A488002A46079800F0FAFE059B5B1B00250593FA
:10A49800049000F114030893A6E6002707E6059246
:10A4A8004FF001092BE62C468146039904EB010B7A
:10A4B800635CF25C002A7AD00BF10102144612F8B0
:10A4C800013BF15C0029F9D114E601251DE7284676
:10A4D8000299039A01F04EF90028E4D0A1462C46CF
:10A4E800CB4602E62546A3460127F0E51598002845
:10A4F8007FF493AE099A62270498089913600123A0
:10A50800149A03610B60106009E621277FE7DDF8E4
:10A5180020B04FF0000851E6159AC2F10103002B54
:10A528003FF473AF19E7A6427FF477AE012CE1DD63
:10A538000498611E01F0DCF800283FF46EAE069A1C
:10A548005368D7E7159900293FF467AED2E701327F
:10A558000A6023E7069A22271368013BA3427FF487
:10A5680056AF63110498012204F01F0400EB830323
:10A5780002FA04F25B691A4214BF2127222746E730
:10A5880051680798013100F06FFC0646049800F105
:10A598000C01036906F10C009A1C9200FBF7E6FC1B
:10A5A80004990798049600F087FC3369EFE65C4647
:10A5B800A0E500BF2DE9F04F85B0DFF8B0810C466B
:10A5C8000290924698F83030002B00F0AF80236854
:10A5D8005A1113F01F0303930AEB8202009201D071
:10A5E80004320092009A002399460099CB464E46C1
:10A5F80042F8043C0439029B0191DDF804C0196853
:10A6080064464B78002B34D018F80320002A70D108
:10A61800202B00F285805E4527DDB9F1070FCCBFFE
:10A6280000230123644528BF002393B1C9F1080919
:10A63800226823464FEA8909C9F12007586800FAB9
:10A6480007F5154320FA09F21D6043F8042F9C45CD
:10A65800F4D8544598BF4FF0080906D9002244F8A9
:10A66800042C043CB346A446914601314B78002B98
:10A67800CAD1002E56D0B9F1070FCCBF0023012351
:10A68800644528BF002393B1C9F10809226823460D
:10A698004FEA8909C9F12005596801FA05F0104304
:10A6A80021FA09F2186043F8042F6345F4D3A24550
:10A6B8003FD20198524654F8041B1346A04243F86F
:10A6C800041B1A46F7D20199002243F8042B994239
:10A6D800FBD2009951F8043C4BB9019B9A4502D131
:10A6E80039E09A4538D053F8042D002AF9D00520CE
:10A6F80019E009F101090136B9F1080F07DC2368EF
:10A708001B0102F00F0201311A432260AEE75445E3
:10A71800ABD900234FF0010944F8043C043CF0E7AE
:10A72800292B1DD0042005B0BDE8F08FFFF770FC81
:10A738004DE7039A002ACCD0009A039952F8043CBA
:10A74800C1F120024FF0FF3121FA02F21340009AC2
:10A7580042F8043CC0E75346012205201A60E2E7AC
:10A76800029B02311960002E85D1DBE7B07201200F
:10A7780010B5144622B110460A49FBF7D1FD08B9B5
:10A78800094810BD20460849FBF7CAFD0028F7D044
:10A7980020460649FBF7C4FD034B00280CBF1846AA
:10A7A800002010BDB8C306084CC30608D8BE06086A
:10A7B80040F26870C2F20000704700BF40F2687350
:10A7C800C2F20003186A7047004870478C070020DF
:10A7D8000020704700487047AC07002040F2103353
:10A7E8000A46C2F2000301461868FFF7C1BF00BF5E
:10A7F80000487047AC0700202DE9F04F01F10B0429
:10A80800162C83B006462DD924F00704E30F8C429A
:10A818002CBF194643F0010100292CD1304600F025
:10A828001FFBB4F5FC7F2BD24FEAD40CB94F07EBD2
:10A83800CC02D368934200F00082596803F10808FB
:10A84800DA68304621F0030499681B195C68CA600D
:10A8580044F0010491605C6000F004FB404603B0E2
:10A86800BDE8F08F002310248C422CBF194643F01A
:10A8780001010029D2D00C234FF000083360EDE726
:10A888005FEA542C04BF4FEAD40C4FEA4C0540F061
:10A898008980A04F07EB8505EB689D4206D10DE046
:10A8A800002A80F24981DB689D4207D0596821F06F
:10A8B80003010A1B0F2AF3DD0CF1FF3C0CF1010C1C
:10A8C800944A3B6902F1080E734508BFD2F8049018
:10A8D80022D0586820F00300011B0F2900F379816A
:10A8E8000029C2F814E0C2F810E066DAB0F5007F7B
:10A8F80080F04581C1084FF0010802EBC1008910C2
:10A9080008FA01F851688568D86048EA0109C2F870
:10A9180004909D60EB60836001224FEAAC0302FA69
:10A9280003F34B4554D819EA030F0DD193402CF08B
:10A93800030C19EA030F0CF1040C05D15B000CF1B0
:10A94800040C19EA030FF9D007EBCC09E046484696
:10A95800C268904207D150E1002980F27881D2681C
:10A96800904200F04A81556825F00305291B0F29FC
:10A97800F2DD90461319D56844F0010058F8084FE5
:10A9880041F0010C50603046C3F804C0E560AC608B
:10A998007B613B61C3F80CE0C3F808E0595000F054
:10A9A80061FA5BE7BCF1040F00F2D5804FEA941C12
:10A9B8000CF1380C4FEA4C056BE71A1803F108083C
:10A9C8003046536843F00103536000F04BFA45E703
:10A9D800BD686B6823F003094C4504D8C4EB090330
:10A9E8000F2B00F39B80DFF830A105EB0902D7F8A5
:10A9F8000814DAF800300131234408BF03F1100BC2
:10AA080006D003F580530F3323F47F6323F00F0B35
:10AA180030465946019200F097FE019AB0F1FF3F87
:10AA2800804600F05B81824200F22781DAF8043028
:10AA380042455B44CAF8043000F05981D7F808143D
:10AA48003046013117BFC2EB0802324B9B18CAF8D7
:10AA5800043008BFC3F8088418F007031FBFC3F108
:10AA68000802C3F58053904403F1080208EB0B0376
:10AA780008BF4FF480521B051B0DC3EB020B594650
:10AA880000F062FE431C00F03E81C8EB00025A440D
:10AA980042F00102DAF80430BD42C7F808805B448E
:10AAA800C8F80420CAF8043017D0B9F10F0F40F2E3
:10AAB8000481A9F10C02696822F007024FF0050E23
:10AAC800A8180F2A01F0010142EA01016960C0F8E3
:10AAD80004E0C0F808E000F21A81DAF82C20BD681A
:10AAE800934284BF0C4AD362DAF83020934284BF81
:10AAF800094A13636A6822F003029442C4EB020312
:10AB080001D80F2B0ADC30464FF0000800F0AAF9F4
:10AB1800A4E600BFE4070020740E00202A1943F0C1
:10AB2800010344F0010430466C6005F108085360E5
:10AB3800BA6000F097F991E65918DA689C683046CF
:10AB48004D6803F1080845F00105E26094604D6026
:10AB580000F088F982E6BCF1140F9CBF0CF15B0C85
:10AB68004FEA4C057FF695AEBCF1540F00F28E808B
:10AB78004FEA143C0CF16E0C4FEA4C0589E6420A88
:10AB8800042A73D9142A9CBF02F15B094FEA4905CC
:10AB980008D9542A00F2C3804FEA103909F16E0926
:10ABA8004FEA490507EB8505DFF8B481AA68AA4290
:10ABB80076D0516821F00301884202D2926895420A
:10ABC800F7D1D068D7F80490D8609A60D3608360D2
:10ABD800A2E61D1941F00107556144F00104156111
:10ABE80030465C6003F10808C5F80CE0C5F808E0D9
:10ABF8006F60695000F036F930E608F10108083056
:10AC080018F0030F7FF4A4AE4A461CF0030FA2F11C
:10AC180008010CF1FF3C00F09A8012688A42F4D0D7
:10AC28007A685B0093423FF6D3AE002B3FF4D0AE78
:10AC38001A4200F09180C44686E603F108025B6977
:10AC48009A4208BF0CF1020C3FF43AAEF5E5904683
:10AC58005519D368304658F8082F6968D36041F011
:10AC680001019A60696000F0FDF8F7E54FEA901974
:10AC780009F138094FEA490594E7BD423FF4D6AED9
:10AC8800374B9D686A6822F0030236E7BCF5AA7F55
:10AC980019D84FEAD43C0CF1770C4FEA4C05F8E58B
:10ACA8000125D8F804104FEAA909104605FA09F554
:10ACB80045EA0109C8F8049086E701234546C8F823
:10ACC8000430002219E740F254539C450BD84FEA50
:10ACD800944C0CF17C0C4FEA4C05DAE5BD686A68C7
:10ACE80022F0030209E7FC254FF07E0CD1E511059F
:10ACF800090D00297FF4A2AEBA680BEB090141F0F7
:10AD080001015160E9E601224FF0000BC2E630462E
:10AD180005F1080101F098FB124B5B68DDE6B2F51E
:10AD2800AA7F06D84FEAD03909F177094FEA4905D1
:10AD380038E740F25451FC258A424FF07E099EBF05
:10AD48004FEA904909F17C094FEA49052AE77A68F0
:10AD580022EA03027A6064E75B0008F1040867E707
:10AD6800E4070020740E00208307C9B270B440D0F5
:10AD7800541E002A3FD003788B4221D0431C04E0A4
:10AD880004B30278013C8A421AD013F0030F184624
:10AD980003F10103F4D1032C16D8651E94B103788E
:10ADA8008B420DD0421C002302E004788C4207D06D
:10ADB8009D42104603F1010302F10102F5D1002082
:10ADC80070BC70472046FBE741EA012646EA064682
:10ADD8000246043013687340A3F1013525EA0303E2
:10ADE80013F0803F03D1043C032CF1D8D5E710467B
:10ADF800D3E71446CFE71046E2E700BF032A70B452
:10AE080022D941EA00039B0713D00578013A0C7850
:10AE18000023A54206D01BE010F8015F11F8014F8E
:10AE2800A54215D1934203F10103F5D1002070BC6E
:10AE380070470C460346043104301E682568AE424C
:10AE480008D1043A032AF4D8002ADED11046EEE7E6
:10AE5800281BECE721461846002AD6D1F6E700BFA2
:10AE6800704700BF704700BF38B50546C36C0C4635
:10AE78004BB153F8240080B1026843F82420002322
:10AE88000361C36038BD0421212201F061FA034641
:10AE9800E8640028EDD1002038BD01232846194672
:10AEA80003FA04F56A1D920001F052FA0028F2D064
:10AEB80044608560E3E700BF31B1C36C4A6853F86A
:10AEC8002200086043F82210704700BF2DE9F047C0
:10AED8008846D1F810A082B0814601F114050024FB
:10AEE8002F680134BEB23F0C02FB063602FB07F3A3
:10AEF80003EB1643B6B206EB03461B0CA24545F816
:10AF0800046BEDDC53B1D8F8082092450ADA08EB57
:10AF18008A020AF10101C8F810105361404602B0D4
:10AF2800BDE8F087D8F80410484601930131FFF7CF
:10AF38009BFFD8F8102008F10C0102329200044659
:10AF480000F10C00FBF712F8D8F80410D9F84C20DF
:10AF5800019B52F82100C8F8000042F82180A04661
:10AF6800D5E700BF2DE9F84348F639651F46C3F613
:10AF7800E30503F1080306460C46904685FB0310DB
:10AF8800DB17C3EB6000012837DD012500216D00C8
:10AF98000131A842FBDC3046FFF766FF089B43619E
:10AFA8000123B8F1090F0146036122DD04F1090903
:10AFB80044444D4615F8013B0A223046303BFFF722
:10AFC80085FFA5420146F5D109EB0804083C474531
:10AFD8000CDDC8EB0707E71914F8013B0A223046D5
:10AFE800303BFFF773FFBC420146F5D10846BDE888
:10AFF800F8830A344FF00908E9E70021CBE700BFDE
:10B00800034600201A0C01D11B04102013F07F4FB7
:10B0180001D108301B0213F0704F01D104301B011D
:10B0280013F0404F01D102309B00002B02DB5B0084
:10B0380001D4202070470130704700BF03680246E2
:10B0480013F0070007D0D9071FD498071FD49B080F
:10B0580002201360704799B209B91B0C102013F035
:10B06800FF0F01D108301B0A190701D104301B0951
:10B07800990701D102309B08D90704D45B0801D194
:10B0880020207047013013607047002070475B082C
:10B0980001201360704700BF10B50C460121FFF76F
:10B0A800E3FE01224461026110BD00BF2DE9F04FAB
:10B0B8000C460E6985B015691746AE4204DA324669
:10B0C8003C462E460F461546A36806EB0508616800
:10B0D8009845C8BF0131FFF7C7FE00EB880900F1AA
:10B0E800140309F11409019000204B4503D243F8D9
:10B0F800040B9945FBD807EB850504EB8606143746
:10B10800143514341436AF4257D2019ACDF808904A
:10B11800A946CDF80C8002F1180CA04657F8044B4C
:10B12800A0B2F0B14246ACF10403002452F8041B6B
:10B138001D681FFA81FA090C1FFA85FB2D0C00FB0C
:10B148000ABA00FB0151544401EB1441A4B244EA89
:10B1580001450C0C964243F8045BE7D81C6057F88D
:10B16800044C240C21D05CF8041C4246634600259C
:10B178000846B2F800A0000C89B29B4604FB0A00FE
:10B18800451941EA054143F8041C53F8040B52F8E9
:10B19800041B1FFA80FA090C04FB01A101EB1541FD
:10B1A8000D0C9642E5D8CBF80010B9450CF1040C0B
:10B1B800B4D8DDF80890DDF80C80B8F1000F0BDD8D
:10B1C80059F8043CA9F104091BB105E059F8043DFC
:10B1D80013B9B8F10108F9D1019B1846C3F81080DA
:10B1E80005B0BDE8F08F00BF12F003032DE9F04170
:10B1F800144680460F462BD1A4101BD0D8F84860BF
:10B208002EB92EE0641015D03568B5B12E46E0078A
:10B21800F8D5394632464046FFF748FFB7B17A6855
:10B228006410D8F84C3053F82210396043F8227073
:10B238000746E9D13846BDE8F081314632464046F6
:10B24800FFF734FF306006460560E0E70746D9E7B8
:10B25800094A5D1E002352F82520FFF737FE0746EE
:10B26800CAE7404640F27121FFF716FF0023C8F8ED
:10B27800480006460360CAE7C8BA06082DE9F84F31
:10B2880093460A6988464FEA6B158B6805EB020AF4
:10B2980081460AF1010649689E4203DD5B000131DF
:10B2A8009E42FBDC4846FFF7DFFD002D024600F119
:10B2B80014040ADD00231F46013344F8047BAB4223
:10B2C800FAD102EB830303F11404D8F8107008F1E3
:10B2D800140508EB870714371BF01F0B21D0CBF19F
:10B2E80020030021286800FA0BF0014344F8041BEE
:10B2F80055F8041BAF4221FA03F1F3D8216009B1D4
:10B308000AF10206D9F84C30013ED8F8041010466C
:10B31800166153F82120C8F8002043F82180BDE8C1
:10B32800F88F55F8043BAF4244F8043BEAD955F886
:10B33800043BAF4244F8043BF3D8E3E703460A6909
:10B34800006930B4801A0FD1043203F11405920059
:10B358009B1889180433043153F8042D51F8044D0F
:10B36800A24203D19D42F7D330BC7047944294BFA8
:10B3780001204FF0FF30F7E72DE9F84F8B460446E0
:10B38800114658469146FFF7D9FF051E61D0BCBF4C
:10B398005B46CB462046B8BF9946DBF80410ACBFE5
:10B3A8004FF000084FF00108FFF75EFDDBF8107062
:10B3B80009F11405D9F810300BF1140600240BEB31
:10B3C800870C09EB83090CF1140C09F1140900F13D
:10B3D800140AC0F80C8056F8048B534655F804AB91
:10B3E80032461FFA88F109191FFA8AFBCBEB0101D3
:10B3F8004FEA1A44C4EB184404EB214489B241EAE9
:10B4080004412414A94543F8041B9A46E3D8B445DB
:10B41800984614D952F8045BA9B22D0C0C1905EB07
:10B428002445A4B244EA05412C14944543F8041B6E
:10B43800F0D8F343634423F0030304334344043B49
:10B4480021B953F8042D013F002AFAD00761BDE85D
:10B45800F88F20462946FFF707FD01234561036160
:10B46800BDE8F88F0023C7F6F0730B40A3F15073C3
:10B47800002B02DD1946002070475B4200211B1596
:10B48800132B0BDD322B02DD0123184670470122F6
:10B49800C3F1330302FA03F3184670474FF400224E
:10B4A800002042FA03F170472DE9F84300F114082F
:10B4B80006698946043600EB86063446374654F852
:10B4C800045B2846FFF79CFD0A28C0F12003C9F851
:10B4D800003018DCB045C0F10B0125FA01F738BF80
:10B4E80054F8084C47F07F5747F4401334BF24FA08
:10B4F80001F10021153005FA00F541EA0502104670
:10B508001946BDE8F8830021B04502D254F8081C5A
:10B51800371FB0F10B0418D005FA04F5C0F12B0061
:10B52800474545F07F5521FA00F645F4401545EAB0
:10B53800060388BF57F8045C01FA04F18CBF25FAAA
:10B5480000F0002040EA0102D9E745F07F550A469D
:10B5580045F44013D3E700BF2DE9F041012182B043
:10B568001D461446FFF780FCC5F30A5725F07F43B4
:10B57800A84623F4700306460FB143F480130193E1
:10B58800002C22D002A840F8084D6846FFF756FD67
:10B59800019B00282ED1009A7261002B0CBF012458
:10B5A8000224B3613461DFB9089A06EB8403A0F280
:10B5B800324010601869FFF723FD099BC0EB441067
:10B5C8001860304602B0BDE8F08101A8FFF736FDEB
:10B5D80001231C463361019B73612030002FE3D0A7
:10B5E800089AA7F23348C0F1350340441060099A1D
:10B5F8001360E6E7C0F12001009A03FA01F123FA8B
:10B6080000F30A4301937261C7E700BF2DE9F043D5
:10B6180083B0884669460646FFF746FF0D4604464E
:10B6280001A94046FFF740FFD6F810C0D8F810E04F
:10B638002F462646CEEB0C0E0B4689460246804620
:10B648009DE80300C1EB000C0CEB4E1EBEF1000F91
:10B65800C3BF05EB0E5724463D46A3EB0E59DCBF8E
:10B6680012464B462046294601F0A6FE03B0BDE827
:10B67800F08300BF172810B504460CDD0021002018
:10B68800C3F6F07100230022C4F2240301F06AFD1E
:10B69800013CF7D110BD034B03EBC004D4E904010E
:10B6A80010BD00BFC8BA060870B40139156902F1A7
:10B6B80014034E11013602EB8505143500EB86069E
:10B6C800AB420CD2014653F8044B9D4241F8044B5F
:10B6D800F9D8AB1A153B23F003030433C01886428C
:10B6E80004D9002340F8043B8642FBD870BC70475D
:10B6F80030B44B11046900F114029C42B8BF2346D0
:10B7080000DB11DC043300EB8300031D9A4218D2DE
:10B7180053F8043C2BB9824213D250F8043D002B55
:10B72800F9D0012030BC704711F01F01EAD000EBBE
:10B738008304646924FA01F505FA01F1A142F0D104
:10B74800E0E70020EEE700BF38B50546064C08469E
:10B75800002323604EF0CAFB431C00D038BD236889
:10B76800002BFBD02B6038BDB07301200020C7F63A
:10B77800C070704770B4002A45D041EA000313F046
:10B78800030329D1032A27D905680C68A54223D1C8
:10B79800141F3AD0A5F1013222EA050515F0803FC1
:10B7A8000DD03AE05B686A68A3F10135934225EA57
:10B7B80003052ED1043C28D015F0803F27D10D4633
:10B7C800034604310430032CECD8661E2CB91C79CE
:10B7D8002A79A01A70BC7047561E04780A789442D9
:10B7E800F7D1C6B18CB101368B1C891904E08B42A4
:10B7F80003F101030BD044B110F8014F13F8012CE9
:10B808009442F4D0E5E71046E4E72046E2E700205A
:10B81800E0E7661EE1E73046DCE71846DAE700BFF6
:10B828002DE9F04F83B09468924601900D46176851
:10B83800002C74D04FF0000B08688B685C46002C15
:10B848004CD09C421E4698464DD3B5F80CE01EF4E9
:10B85800906F33D06B69621C29690EF4806E03EB1C
:10B868004303461A901903EBD3734FEA63098145E2
:10B878004A4638BF81460FFA8EF038BF4A4600283C
:10B8880034D001981146FEF7B7FF8046002837D01C
:10B8980032462969FAF76AFBAA8922F4906242F0D3
:10B8A8008002AA8108EB0600C6EB0902C5F81080E1
:10B8B8002646A0462860C5F81490AA604246594614
:10B8C80000F088FEDAF80820AB682868141B9B1B78
:10B8D800AB6040442860CAF8084004B3D7F800B009
:10B8E8007C680837ABE72646A046E7E7019800F0F2
:10B8F800CFFE80460028D5D10198296900F0A4FD23
:10B90800019A0C234FF0FF3013600023AA8942F0FC
:10B918004002AA81CAF80830CAF8043002E020467A
:10B92800CAF8044003B0BDE8F08F00BF2DE9F04F1E
:10B93800B3B009938B89059103F080030B901BB278
:10B948001BB10B69002B00F0C384974F904622ACC3
:10B958000DF1870C002326460394CCEB04040E93C8
:10B96800CDF808C00693119415961793169398F876
:10B978000030002B18BF252B00F0468308F1010288
:10B98800154601322B78252B18BF002BF8D1B5EBC3
:10B9980008040FD0169A17990132C6F80080072AB2
:10B9A800214474601692179100F3B3830836069BFE
:10B9B8001B1906932B78002B00F03983002205F120
:10B9C800010813464FF0FF358DF84F200A92049274
:10B9D80018F8012BA2F12001582900F23282DFE881
:10B9E80011F0670130023002620130023002300289
:10B9F800300230023002D10081013002DE008301C2
:10BA080030027C016B016B016B016B016B016B01F7
:10BA18006B016B016B0130023002300230023002E0
:10BA28003002300230023002300259003002300257
:10BA3800300230023002300230023002300230026E
:10BA4800BA0030023002300230023002A500300263
:10BA580030024B0130023002300230023002300234
:10BA68003002300230023002E5005F00300230025E
:10BA78003002E9015F0030023002E4013002F001D7
:10BA8800C000A5019E013002BC013002A9003002AD
:10BA980030020502DDF810C04CF0100CCDF810C0D3
:10BAA8008DF84F30049BD80640F18383099C2368A6
:10BAB80004340994002BC0F289839DF84F200CBFF1
:10BAC800002001200121002DA2BF049C24F0800445
:10BAD8000494002D18BF40F00100C0B2002800F007
:10BAE8009582012900F04D8302290DF1870100F0AC
:10BAF8003C8303F007000C4630300139DB08207026
:10BB0800F7D1DDF810C023461CF0010F40F09B83ED
:10BB1800039B1B1B07930895079DDDF820C065450F
:10BB2800B8BF6546002A51D001354FE0049B43F069
:10BB380010030493049CE20600F19181049B5B06C8
:10BB480040F18D81099C0121238804340994181C33
:10BB580018BF012012E0DDF810C04CF0100CCDF831
:10BB680010C0049B13F0100200F03983099C0021D7
:10BB7800236804340994581A18BF012000228DF84C
:10BB88004F20A0E7099CDDF824C024680CF10402CA
:10BB9800002C0A9480F24283644209920A94049C1D
:10BBA80044F00404049413E7F0BB0608099B01253C
:10BBB800002207951C1D09941B6818AC8DF84F20AE
:10BBC8008DF860304FF0000CCDF820C0049BDDF8F4
:10BBD80010C013F002030C9318BF02351CF084093F
:10BBE80040F050810A9BC5EB030BBBF1000F40F3FB
:10BBF8004981BBF1100F179940F37A839E4B4FF0A0
:10BC0800100ACDF83C80D8461094CB46169AA9461F
:10BC18000D930B9C059D04E0A8F11008B8F1100FD6
:10BC280018DD0132103186E880040836072A16929A
:10BC38001791F1DD2046294615AA22AEFFF7F0FD3F
:10BC4800002840F0FB81A8F110081799B8F1100FEF
:10BC5800169AE6DC4D46109CD946C346DDF83C8072
:10BC680001320D9B072A5944169286E80808179155
:10BC780000F3C882083607E1DDF810C08DF84F30B0
:10BC88007E4B1CF0100F0E9300F0BA80099C2368BD
:10BC980004340994049CE40700F1C080181C18BF00
:10BCA800012002216AE7049C44F0010404948FE611
:10BCB800002B08BF20238BE640460021A2F1300C60
:10BCC80010F8012B01EB8101A2F130048046092C08
:10BCD8000CEB4101F2D90A917CE6049C44F0800403
:10BCE800049475E62B2373E618F8012B2A2A00F032
:10BCF8001583A2F13001002509293FF66BAE4046B5
:10BD0800002510F8012B05EB850501EB4505A2F18F
:10BD1800300109298046F4D945EAE5755AE6DDF887
:10BD280010C04CF0100CCDF810C051E6099B302221
:10BD3800DDF810C002211C1D09941B684CF0020C90
:10BD48004F4C8DF850207822181CCDF810C08DF873
:10BD5800512018BF01200E9410E7DDF824C04FF0E1
:10BD680000098DF84F900CF1040ADCF80040002C13
:10BD780000F0C282002D2046C0F2968249462A462B
:10BD8800FEF7F2FF002800F0C182001B9DF84F204B
:10BD9800A8420790CDF824A0C4BF0795CDF82090FD
:10BDA8003FF7BAAECDF82090B6E6049C44F01004F4
:10BDB80004940DE6DDF810C04CF0400CCDF810C02E
:10BDC80006E68DF84F30049BD90600F14782DDF86E
:10BDD80010C01CF0400F00F04182099CDDF818C02B
:10BDE800236804340994A3F800C0C0E5DDF810C046
:10BDF800234C1CF0100F8DF84F300E947FF446AF93
:10BE0800DDF810C01CF0400F00F04582099C238823
:10BE180004340994049CE4077FF540AF18460221D6
:10BE2800002B3FF4ABAEDDF810C001208DF8512097
:10BE3800022130224CF0020C8DF85020CDF810C0B1
:10BE48009CE68DF84F30002A00F0F1800125002390
:10BE58008DF8602018AC07958DF84F30B2E6DDF804
:10BE680024C00121DCF800300CF1040CCDF824C00A
:10BE7800181C18BF012081E6F0BB06088CC1060813
:10BE880070C306081799169A9DF84F3063B10132AE
:10BE98000DF14F0333600123072A1944736016928A
:10BEA800179100F34A8108360C9B5BB1013214AB41
:10BEB80033600223072A194473601692179100F31E
:10BEC80048810836B9F1800F00F0C980DDF820C03C
:10BED800079BC3EB0C0ABAF1000F3CDDBAF1100F57
:10BEE800DFF81C932DDDCDF820804FF0100BD046E5
:10BEF800AA464D46A1460B9C04E0A8F11008B8F1EB
:10BF0800100F18DD0132103186E820080836072A9C
:10BF180016921791F1DD2046059915AA22AEFFF772
:10BF28007FFC002840F08A80A8F110081799B8F122
:10BF3800100F169AE6DC4C46A9465546C246DDF86F
:10BF4800208001325144072A86E80006169217918C
:10BF580000F3E8800836079B0132072A3460194449
:10BF680016927360D8BF06F10803179100F3BB80DF
:10BF7800049C620734D50A98441B002C30DD102C31
:10BF8800169ADCBF9D480D9020DD9C481026DDF8F0
:10BF98002C90DDF814A00D9002E0103C102C15DD5B
:10BFA800013210311F605E600833072A169217911C
:10BFB800F3DD4846514615AAFFF732FC22AB0028AC
:10BFC8003CD1103C1799102C169AE9DC01320D98D7
:10BFD800072A2144169283E81100179100F3218162
:10BFE800069B0A9CA542ACBF5B191B190693002946
:10BFF80040F083800023169398F8003022AE002B7F
:10C0080018BF252B7FF4BAAC4546D3E400297DD16F
:10C01800049CE0075CBF079122AC7FF57CAD119BC7
:10C028000DF18704079330238DF8873073E5179B4C
:10C0380023B10B9815AA0599FFF7F2FBDDF814C098
:10C04800069CBCF80C3003F040031BB2002B18BF51
:10C058004FF0FF340694069833B0BDE8F08F0A9B82
:10C06800C5EB030ABAF1000F7FF730AFBAF1100F32
:10C07800DFF88C912CDDCDF830804FF0100BD046D6
:10C08800AA464D46A1460B9C04E0A8F11008B8F159
:10C09800100F17DD0132103186E820080836072A0C
:10C0A80016921791F1DD2046059915AA22AEFFF7E1
:10C0B800B7FB0028C2D1A8F110081799B8F1100FE2
:10C0C800169AE7DC4C46A9465546C246DDF830804C
:10C0D80001325144072A86E800061692179100F3A8
:10C0E800EB800836F2E60B9815AA0599FFF798FB3E
:10C0F8000028A3D1179922AB3AE70B9815AA0599FE
:10C10800FFF78EFB00283FF475AF97E7079022AC46
:10C1180001E50B9815AA0599FFF782FB00288DD138
:10C1280022AE44E40B9815AA0599FFF779FB00287D
:10C1380084D1179922AE169A0DE70B9815AA05997E
:10C14800FFF76EFB00287FF479AF179922AE169A95
:10C15800AAE60B9815AA0599FFF762FB00287FF459
:10C168006DAF179922AE169AACE6DDF838C003F029
:10C178000F000C4601391B091CF800002070F6D18D
:10C18800C6E4092B57D94CF6CD490DF18700CCF6FA
:10C19800CC49A9FB03C104460138C90801EB810C4D
:10C1A800A3EB4C0C0B460CF130012170002BF0D1A5
:10C1B800AEE4DDF810C01CF0400F63D0099CB4F960
:10C1C800003004340994002BBFF677AC5B422D2273
:10C1D800181C8DF84F2018BF0120012173E4DDF8E9
:10C1E80010C01CF0400141D0099C1146238804343A
:10C1F8000994181C18BF0120C0E400BFF0BB060852
:10C2080000BC06080B9815AA0599FFF709FB00283A
:10C218007FF414AF179922AE169A35E60992FFF704
:10C22800D7BB0B9815AA0599FFF7FAFA00287FF4EF
:10C2380005AF1799D4E6119C30338DF887300794F1
:10C248000DF1870467E430283FF462AC03980C468C
:10C25800401A3021079003F8011C5CE4099C23680C
:10C2680004340994069C1C60FFF781BBDDF824C0E8
:10C27800DCF800300CF1040CCDF824C0181C18BFF1
:10C2880001207BE4DDF824C0DCF800300CF1040C5C
:10C29800CDF824C00EE4DDF824C0DCF800300CF141
:10C2A800040CCDF824C0F5E4CDF824A0FAF784F9FD
:10C2B8009DF84F20079075E50B9815AA0599FFF78B
:10C2C800AFFA00287FF4BAAE179922AE169AFDE5A8
:10C2D80040210192FEF790FA059C019A20602061A6
:10C2E80050B3DDF814C04023CCF81430FFF72DBB51
:10C2F800154B169A0D93B3E4062D28BF0625CDF8E5
:10C3080024A0079525EAE575104C5BE49DF84F20BD
:10C31800CDF824A007950890FFF7FEBBDDF824C0F0
:10C328000CF10402DCF80050002DBFF677AF09923B
:10C338004FF0FF35FFF74CBB0B9C4FF0FF330693D4
:10C348000C23236087E600BFF0BB060884C30608F9
:10C3580010B501FB02F1FEF74FFA044670B150F830
:10C36800042C22F00302043A242A1CD8132A98BF6A
:10C37800034605D800221A605A609A60204610BD0C
:10C3880000211B2A016098BF00F108034160F1D920
:10C39800242A8160C16011BF00F11003016100F11E
:10C3A80018034161E6E70021F9F72AFE204610BD8F
:10C3B800F8B50F46214D0446FEF752FDAB685E689E
:10C3C80026F0030606F6EF73DF1B3F0B013F3F0322
:10C3D800B7F5805F07DB00212046FFF7B5F9AB68AA
:10C3E8009B19984204D02046FEF73CFD0020F8BD7A
:10C3F80079422046FFF7A8F901300DD0104BF61B03
:10C40800A968204646F001061A684E60D71B1F60CF
:10C41800FEF728FD0120F8BD00212046FFF794F91A
:10C42800AB68C21A0F2ADEDD42F001025A60054BE2
:10C438001B68C01A024B1860D5E700BFE40700204C
:10C44800780E0020EC0B0020F8B50D4606460029B2
:10C4580055D0FEF705FD55F8041CDFF868C1A5F1B5
:10C46800080421F00103E218DCF80800576890423C
:10C4780027F0030764D011F00101576032D0002182
:10C48800D0194068C00706D4DB199068002949D044
:10C49800D268C260906043F00102E3506260E1B983
:10C4A800B3F5007F2CD35A0A042A65D89809383086
:10C4B80041000CEB810C4349DCF80820624566D04A
:10C4C800516821F003018B4202D292689445F7D15A
:10C4D800D368E360A260D4609C603046BDE8F84051
:10C4E800FEF7C0BC55F8080C0CF10805241A1B18F7
:10C4F800A068A8423ED0E568C560A860C0E7F8BD5E
:10C50800DB080121DCF804000CEBC3029B1001FAE4
:10C5180003F3E26091681843CCF80400A160CC6092
:10C528009460DAE7284DA842B2D1CCF8144043F021
:10C538000102CCF81040E060A0606260E350CCE7F4
:10C54800FF18CB0707D455F8083CE41AFF18A2686F
:10C55800E368D3609A6047F0010363601B4BCCF833
:10C5680008401B689F42B8D3194B30461968FFF73B
:10C578001FFFB2E7012183E702F15B004100142AA3
:10C5880097D9542A0CD8180B6E30410091E701272F
:10C598004D688010134607FA00F005434D6098E790
:10C5A800B2F5AA7F03D8D80B7730410081E740F273
:10C5B80054518A4203D8980C7C30410079E7FC2119
:10C5C8007E2076E7E4070020EC070020F00B00202F
:10C5D800740E00208842F0B411D98C18A0420ED2F3
:10C5E8008518531E4AB121462A4611F8014D013BD0
:10C5F800B3F1FF3F02F8014DF7D1F0BC70470F2AA5
:10C6080040D941EA00039B073ED10C460346154634
:10C618002668103D1E6066685E60A6689E60E668D3
:10C628001034DE6010330F2DF2D8A2F1100502F09D
:10C638000F0425F00F051035032C00EB05032944E2
:10C6480024D9A4F1040C1D460C464FEA9C0C01EBBE
:10C658008C07043754F8046BBC4245F8046BF9D1D5
:10C668000CF1010402F00302A40009191B19002AA5
:10C67800C3D001399A1811F8014F03F8014B9342BE
:10C68800F9D1BAE70346F2E70346F2E72246EEE7B6
:10C698002DE9F04F0C4683B081461746002900F07B
:10C6A8002A8107F10B05FEF7DBFB54F8043C162D35
:10C6B800A4F1080A23F003067DD810214FF00008E2
:10C6C8000D46BD4238BF48F00108B8F1000F40F0F0
:10C6D80018818E4275DADFF8B4C30AEB0602DCF87B
:10C6E8000800904200F01281D2F804E02EF0010B0D
:10C6F8009344DBF804B01BF0010F1CBFC64672461A
:10C7080078D0DB0700F1D18054F8083CC3EB0A0B62
:10C71800DBF8043023F003039B19002A75D082420A
:10C7280000F045810EEB030888456EDBD1685B4657
:10C738009068321F242AC1608860DBF80C1053F817
:10C74800080FC160886000F28E81132A9CBF1946C9
:10C75800204625D921681B2A98BF04F10800CBF888
:10C7680008106168CBF80C1098BF0BF1100117D9AD
:10C77800A168242A14BF04F1100004F11800CBF8B2
:10C788001010E168CBF8141011BF0BF118012269E1
:10C798000BF12001CBF8182004BF6269CBF81C20EC
:10C7A80002681C460A60DA4643684B6083688B60FF
:10C7B800DBF8043006E025F0070529464FEAD5786E
:10C7C8007FE7B046C5EB08020F2A5AD80AEB0802E1
:10C7D80003F0010343EA0803CAF80430536843F03E
:10C7E8000103536048462746FEF73CFB384603B032
:10C7F800BDE8F08F2EF0030E0EEB0608884580DBAF
:10C80800D1689268D1608A60DCE78B424DDB5F4675
:10C81800DBF80C10321F57F8080F242AC160886013
:10C8280000F2B580132A9CBF3946204625D92168D5
:10C838001B2A98BF04F10800CBF808106168CBF8F0
:10C848000C1098BF0BF1100117D9A168242A14BF46
:10C8580004F1100004F11800CBF81010E168CBF8CF
:10C86800141011BF0BF1180122690BF12001CBF84C
:10C87800182004BF6269CBF81C2002683C46984621
:10C8880090E70AEB050103F001038E181D4342F0FF
:10C898000102CAF804504A6048467368083143F0F8
:10C8A80001037360FFF7D0FD9CE739464846FDF762
:10C8B800A3FF0746D8B154F8043CA0F1080123F0BF
:10C8C80001025244914200F0C880321F242A6AD8DB
:10C8D800132A9CBF0346224638D81168196051684C
:10C8E800596092689A6048462146FFF7ADFD484670
:10C8F800FEF7B8FA7AE7114603B0BDE8F04FFDF746
:10C908007BBF0C230027C9F800306FE7426805F1A8
:10C91800100822F0030E0EEB06024245B8BF02468D
:10C92800FFF6EFAE0AEB0503521B42F00102484640
:10C938005A60274654F8042CCCF8083002F001025B
:10C94800154344F8045CFEF78DFA4FE723681B2A69
:10C9580098BF04F1080203606368436098BF00F160
:10C968000803BAD9A368242A14BF04F1100204F1F9
:10C9780018028360E368C36011BF00F110032169E6
:10C9880000F11803016104BF61694161A5E721460F
:10C9980038460193FFF71EFE019B3C46DA4698464F
:10C9A800DBF804300EE72146FFF714FE9BE705F19C
:10C9B80010020EEB03089045FFF627AF5F46DBF841
:10C9C8000C30321F57F8081F242ACB60996053D8BF
:10C9D800132A9CBF3B46224625D923681B2A98BFA9
:10C9E80004F10802CBF808306368CBF80C3098BF24
:10C9F8000BF1100317D9A368242A14BF04F11002FD
:10CA080004F11802CBF81030E368CBF8143011BFEA
:10CA18000BF1180321690BF12003CBF8181004BFA0
:10CA28006169CBF81C1011681960516859609268E7
:10CA38009A600BEB0503C5EB080242F00102484679
:10CA48005A60DBF80420CCF8083002F001021543E4
:10CA5800CBF80450FEF706FAC8E650F8042C22F08A
:10CA68000308B044AEE6214618461C46DA46FFF7EE
:10CA7800B1FDDBF80430A5E638462146CDF804C000
:10CA8800FFF7A8FDDDF804C0D3E700BFE4070020E6
:10CA980038B50C460968054609B1FFF7F9FF28467D
:10CAA8002146BDE83840FFF7CFBC00BF214B70B529
:10CAB80005461B68984230D0C26CA2B100231E46BE
:10CAC80052F8231039B10C682846FFF7BDFC2146FF
:10CAD800002CF8D1EA6C0136202E3346F0D12846D6
:10CAE8001146FFF7B1FC296C11B12846FFF7ACFCE1
:10CAF800D5F8481151B105F5A676B14206D00C68B3
:10CB08002846FFF7A1FCA6422146F8D1696D11B16C
:10CB18002846FFF799FCAB6B03B970BDEB6B284651
:10CB28009847D5F8E0120029F7D02846BDE87040AC
:10CB3800FFF7AEBF10030020F8B50746B8B1D7F825
:10CB4800486176B175686C1E08D4023506EB850518
:10CB580055F8043D013C9847631CF9D13668002E0E
:10CB6800F0D1FB6B13B138469847F8BDF8BD014BBF
:10CB78001F68E4E7100300204A1E08BF7047C0F092
:10CB88002481884240F21681114200F01781B0FAE0
:10CB980080F3B1FA81F2A2EB0303C3F11F0304A2ED
:10CBA80002EB03134FF000029F4600BFAFF3008073
:10CBB800B0EBC17F00BF42EB020228BFA0EBC170FF
:10CBC800B0EB817F00BF42EB020228BFA0EB81706F
:10CBD800B0EB417F00BF42EB020228BFA0EB4170DF
:10CBE800B0EB017F00BF42EB020228BFA0EB01704F
:10CBF800B0EBC16F00BF42EB020228BFA0EBC160DF
:10CC0800B0EB816F00BF42EB020228BFA0EB81604E
:10CC1800B0EB416F00BF42EB020228BFA0EB4160BE
:10CC2800B0EB016F00BF42EB020228BFA0EB01602E
:10CC3800B0EBC15F00BF42EB020228BFA0EBC150BE
:10CC4800B0EB815F00BF42EB020228BFA0EB81502E
:10CC5800B0EB415F00BF42EB020228BFA0EB41509E
:10CC6800B0EB015F00BF42EB020228BFA0EB01500E
:10CC7800B0EBC14F00BF42EB020228BFA0EBC1409E
:10CC8800B0EB814F00BF42EB020228BFA0EB81400E
:10CC9800B0EB414F00BF42EB020228BFA0EB41407E
:10CCA800B0EB014F00BF42EB020228BFA0EB0140EE
:10CCB800B0EBC13F00BF42EB020228BFA0EBC1307E
:10CCC800B0EB813F00BF42EB020228BFA0EB8130EE
:10CCD800B0EB413F00BF42EB020228BFA0EB41305E
:10CCE800B0EB013F00BF42EB020228BFA0EB0130CE
:10CCF800B0EBC12F00BF42EB020228BFA0EBC1205E
:10CD0800B0EB812F00BF42EB020228BFA0EB8120CD
:10CD1800B0EB412F00BF42EB020228BFA0EB41203D
:10CD2800B0EB012F00BF42EB020228BFA0EB0120AD
:10CD3800B0EBC11F00BF42EB020228BFA0EBC1103D
:10CD4800B0EB811F00BF42EB020228BFA0EB8110AD
:10CD5800B0EB411F00BF42EB020228BFA0EB41101D
:10CD6800B0EB011F00BF42EB020228BFA0EB01108D
:10CD7800B0EBC10F00BF42EB020228BFA0EBC1001D
:10CD8800B0EB810F00BF42EB020228BFA0EB81008D
:10CD9800B0EB410F00BF42EB020228BFA0EB4100FD
:10CDA800B0EB010F00BF42EB020228BFA0EB01006D
:10CDB800104670470CBF012000207047B1FA81F27D
:10CDC800C2F11F0220FA02F0704708B14FF0FF309D
:10CDD80000F00EB80029F8D02DE90340FFF7CCFE8B
:10CDE800BDE8064002FB00F3A1EB0301704700BF5A
:10CDF800704700BF81F0004102E000BF83F00043AC
:10CE080030B54FEA41044FEA430594EA050F08BFDD
:10CE180090EA020F1FBF54EA000C55EA020C7FEAA1
:10CE2800645C7FEA655C00F0E2804FEA5454D4EB1E
:10CE38005555B8BF6D420CDD2C4480EA020281EAE8
:10CE4800030382EA000083EA010180EA020281EA20
:10CE58000303362D88BF30BD11F0004F4FEA013172
:10CE68004FF4801C4CEA113102D0404261EB410181
:10CE780013F0004F4FEA03334CEA133302D0524207
:10CE880063EB430394EA050F00F0A780A4F10104C3
:10CE9800D5F1200E0DDB02FA0EFC22FA05F28018FD
:10CEA80041F1000103FA0EF2801843FA05F35941E3
:10CEB8000EE0A5F120050EF1200E012A03FA0EFC62
:10CEC80028BF4CF0020C43FA05F3C01851EBE3718C
:10CED80001F0004507D54FF0000EDCF1000C7EEBA9
:10CEE80000006EEB0101B1F5801F1BD3B1F5001FE7
:10CEF8000CD349085FEA30004FEA3C0C04F1010406
:10CF08004FEA445212F5800F80F09A80BCF1004F2E
:10CF180008BF5FEA500C50F1000041EB045141EAB0
:10CF2800050130BD5FEA4C0C404141EB010111F4B1
:10CF3800801FA4F10104E9D191F0000F04BF01465C
:10CF48000020B1FA81F308BF2033A3F10B03B3F13A
:10CF580020020CDA0C3208DD02F1140CC2F10C02CA
:10CF680001FA0CF021FA02F10CE002F11402D8BF28
:10CF7800C2F1200C01FA02F120FA0CFCDCBF41EAF4
:10CF88000C019040E41AA2BF01EB0451294330BDC3
:10CF98006FEA04041F3C1CDA0C340EDC04F11404A0
:10CFA800C4F1200220FA04F001FA02F340EA030077
:10CFB80021FA04F345EA030130BDC4F10C04C4F1BD
:10CFC800200220FA02F001FA04F340EA030029469D
:10CFD80030BD21FA04F0294630BD94F0000F83F4E7
:10CFE800801306BF81F480110134013D4EE77FEACA
:10CFF800645C18BF7FEA655C29D094EA050F08BF16
:10D0080090EA020F05D054EA000C04BF19461046F6
:10D0180030BD91EA030F1EBF0021002030BD5FEA3A
:10D02800545C05D14000494128BF41F0004130BD62
:10D0380014F580043CBF01F5801130BD01F00045B6
:10D0480045F0FE4141F470014FF0000030BD7FEA29
:10D05800645C1ABF194610467FEA655C1CBF0B4624
:10D06800024650EA013406BF52EA033591EA030F3B
:10D0780041F4002130BD00BF90F0000F04BF002133
:10D08800704730B54FF4806404F132044FF0000566
:10D098004FF0000150E700BF90F0000F04BF0021DF
:10D0A800704730B54FF4806404F1320410F0004545
:10D0B80048BF40424FF000013EE700BF42004FEA40
:10D0C800E2014FEA31014FEA02701FBF12F07F43BD
:10D0D80093F07F4F81F06051704792F0000F14BFBA
:10D0E80093F07F4F704730B54FF4607401F00045FE
:10D0F80021F0004120E700BF50EA010208BF704755
:10D1080030B54FF000050AE050EA010208BF704749
:10D1180030B511F0004502D5404261EB41014FF4B2
:10D12800806404F132045FEA915C3FF4DCAE4FF0B6
:10D1380003025FEADC0C18BF03325FEADC0C18BF9D
:10D14800033202EBDC02C2F1200300FA03FC20FAEE
:10D1580002F001FA03FE40EA0E0021FA02F114443B
:10D16800C1E600BF70B54FF0FF0C4CF4E06C1CEA50
:10D1780011541DBF1CEA135594EA0C0F95EA0C0FC5
:10D1880000F0DEF82C4481EA030621EA4C5123EA38
:10D198004C5350EA013518BF52EA033541F4801167
:10D1A80043F4801338D0A0FB02CE4FF00005E1FB1A
:10D1B80002E506F00042E0FB03E54FF00006E1FB64
:10D1C80003569CF0000F18BF4EF0010EA4F1FF04A7
:10D1D800B6F5007F64F5407404D25FEA4E0E6D41E7
:10D1E80046EB060642EAC62141EA55514FEAC520F8
:10D1F80040EA5E504FEACE2EB4F1FD0C88BFBCF574
:10D20800E06F1ED8BEF1004F08BF5FEA500E50F124
:10D21800000041EB045170BD06F0004646EA0101EA
:10D2280040EA020081EA0301B4EB5C04C2BFD4EB1C
:10D238000C0541EA045170BD41F480114FF0000E15
:10D24800013C00F3AB8014F1360FDEBF002001F083
:10D25800004170BDC4F10004203C35DA0C341BDCFD
:10D2680004F11404C4F1200500FA05F320FA04F0CF
:10D2780001FA05F240EA020001F0004221F0004103
:10D2880010EBD37021FA04F642EB06015EEA430E76
:10D2980008BF20EAD37070BDC4F10C04C4F12005A6
:10D2A80000FA04F320FA05F001FA04F240EA020059
:10D2B80001F0004110EBD37041F100015EEA430E2A
:10D2C80008BF20EAD37070BDC4F1200500FA05F24A
:10D2D8004EEA020E20FA04F301FA05F243EA0203C9
:10D2E80021FA04F001F0004121FA04F220EA0200D8
:10D2F80000EBD3705EEA430E08BF20EAD37070BD1E
:10D3080094F0000F0FD101F00046400041EB0101FD
:10D3180011F4801F08BF013CF7D041EA060195F0DF
:10D32800000F18BF704703F00046520043EB030399
:10D3380013F4801F08BF013DF7D043EA0603704786
:10D3480094EA0C0F0CEA135518BF95EA0C0F0CD091
:10D3580050EA410618BF52EA4306D1D181EA0301D7
:10D3680001F000414FF0000070BD50EA410606BFD1
:10D378001046194652EA430619D094EA0C0F02D116
:10D3880050EA013613D195EA0C0F05D152EA03365B
:10D398001CBF104619460AD181EA030101F0004179
:10D3A80041F0FE4141F470014FF0000070BD41F0C2
:10D3B800FE4141F4780170BD70B54FF0FF0C4CF49C
:10D3C800E06C1CEA11541DBF1CEA135594EA0C0FBB
:10D3D80095EA0C0F00F0A7F8A4EB050481EA030E08
:10D3E80052EA03354FEA013100F088804FEA0333EF
:10D3F8004FF0805545EA131343EA12634FEA0222BD
:10D4080045EA111545EA10654FEA00260EF000417D
:10D418009D4208BF964244F1FD0404F5407402D2CF
:10D428005B084FEA3202B61A65EB03055B084FEA60
:10D4380032024FF480104FF4002CB6EB020E75EB5D
:10D44800030E22BFB61A754640EA0C005B084FEA85
:10D458003202B6EB020E75EB030E22BFB61A754602
:10D4680040EA5C005B084FEA3202B6EB020E75EB4D
:10D47800030E22BFB61A754640EA9C005B084FEAC5
:10D488003202B6EB020E75EB030E22BFB61A7546D2
:10D4980040EADC0055EA060E18D04FEA051545EAC1
:10D4A80016754FEA06164FEAC30343EA52734FEA6A
:10D4B800C2025FEA1C1CC0D111F4801F0BD141EAE3
:10D4C80000014FF000004FF0004CB6E711F4801F48
:10D4D80004BF01430020B4F1FD0C88BFBCF5E06F28
:10D4E8003FF6AFAEB5EB030C04BFB6EB020C5FEA38
:10D4F800500C50F1000041EB045170BD0EF0004E8D
:10D508004EEA113114EB5C04C2BFD4EB0C0541EABE
:10D51800045170BD41F480114FF0000E013C90E6BB
:10D5280045EA060E8DE60CEA135594EA0C0F08BF7F
:10D5380095EA0C0F3FF43BAF94EA0C0F0AD150EA7E
:10D5480001347FF434AF95EA0C0F7FF425AF104611
:10D5580019462CE795EA0C0F06D152EA03353FF439
:10D56800FDAE1046194622E750EA410618BF52EAB6
:10D5780043067FF4C5AE50EA41047FF40DAF52EA8A
:10D5880043057FF4EBAE12E74FF0FF3C06E000BF27
:10D598004FF0010C02E000BF4FF0010C4DF804CD34
:10D5A8004FEA410C7FEA6C5C4FEA430C18BF7FEAF4
:10D5B8006C5C1BD001B050EA410C0CBF52EA430C22
:10D5C80091EA030F02BF90EA020F0020704710F1A2
:10D5D800000F91EA030F58BF994208BF90422CBF31
:10D5E800D8176FEAE37040F0010070474FEA410C2A
:10D5F8007FEA6C5C02D150EA013C07D14FEA430C48
:10D608007FEA6C5CD6D152EA033CD3D05DF8040BB8
:10D61800704700BF8446104662468C4619466346EA
:10D6280000E000BF01B5FFF7B7FF002848BF10F1C1
:10D63800000F01BD4DF808EDFFF7F4FF0CBF012006
:10D6480000205DF808FB00BF4DF808EDFFF7EAFF82
:10D6580034BF012000205DF808FB00BF4DF808ED3D
:10D66800FFF7E0FF94BF012000205DF808FB00BF32
:10D678004DF808EDFFF7CEFF94BF012000205DF8BC
:10D6880008FB00BF4DF808EDFFF7C4FF34BF0120C9
:10D6980000205DF808FB00BF4FEA410212F50012B6
:10D6A80015D211D56FF47873B3EB625212D94FEAE1
:10D6B800C12343F0004343EA505311F0004F23FACB
:10D6C80002F018BF404270474FF00000704750EA20
:10D6D800013005D111F0004008BF6FF000407047DD
:10D6E8004FF00000704700BF4A0011D212F5001237
:10D6F80011D20DD56FF47873B3EB62520ED44FEAA2
:10D70800C12343F0004343EA505323FA02F0704721
:10D718004FF00000704750EA013002D14FF0FF305F
:10D7280070474FF0000070474FEA4102B2F1E04302
:10D7380024BFB3F5001CDCF1FE5C0DD901F0004CF0
:10D748004FEAC0024CEA5070B2F1004F40EB830040
:10D7580008BF20F00100704711F0804F21D113F16C
:10D768003872BCBF01F00040704741F480114FEAA5
:10D778005252C2F11802C2F1200C10FA0CF320FA2E
:10D7880002F018BF40F001004FEAC1234FEAD3234B
:10D7980003FA0CFC40EA0C0023FA02F34FEA4303B5
:10D7A800CCE77FEA625307D150EA01331EBF4FF03E
:10D7B800FE4040F44000704701F0004040F0FE4059
:10D7C80040F40000704700BF80F0004002E000BF56
:10D7D80081F0004142001FBF5FEA410392EA030F54
:10D7E8007FEA226C7FEA236C6AD04FEA1262D2EB9E
:10D7F8001363C1BFD218414048404140B8BF5B42A3
:10D80800192B88BF704710F0004F40F4000020F03B
:10D818007F4018BF404211F0004F41F4000121F051
:10D828007F4118BF494292EA030F3FD0A2F101029B
:10D8380041FA03FC10EB0C00C3F1200301FA03F1D9
:10D8480000F0004302D5494260EB4000B0F5000FFC
:10D8580013D3B0F1807F06D340084FEA310102F1BB
:10D868000102FE2A51D2B1F1004F40EBC25008BF6D
:10D8780020F0010040EA03007047490040EB000037
:10D8880010F4000FA2F10102EDD1B0FA80FCACF166
:10D89800080CB2EB0C0200FA0CF0AABF00EBC25065
:10D8A80052421843BCBFD0401843704792F0000F53
:10D8B80081F4000106BF80F400000132013BB5E7A6
:10D8C8004FEA41037FEA226C18BF7FEA236C21D01C
:10D8D80092EA030F04D092F0000F08BF0846704781
:10D8E80090EA010F1CBF0020704712F07F4F04D14F
:10D8F800400028BF40F00040704712F100723CBF62
:10D9080000F50000704700F0004343F0FE4040F48B
:10D91800000070477FEA226216BF08467FEA236349
:10D928000146420206BF5FEA412390EA010F40F434
:10D93800800070474FF0000304E000BF10F0004380
:10D9480048BF40425FEA000C08BF704743F0964367
:10D9580001464FF000001CE050EA010208BF704782
:10D968004FF000030AE000BF50EA010208BF704709
:10D9780011F0004302D5404261EB41015FEA010C1E
:10D9880002BF84460146002043F0B64308BFA3F116
:10D998008053A3F50003BCFA8CF2083AA3EBC253F8
:10D9A80010DB01FA02FC634400FA02FCC2F1200217
:10D9B800BCF1004F20FA02F243EB020008BF20F04E
:10D9C8000100704702F1200201FA02FCC2F12002B4
:10D9D80050EA4C0021FA02F243EB020008BF20EAA9
:10D9E800DC7070474FF0FF0C1CEAD0521EBF1CEAD7
:10D9F800D15392EA0C0F93EA0C0F6FD01A4480EAC5
:10DA0800010C400218BF5FEA41211ED04FF00063AD
:10DA180043EA501043EA5111A0FB01310CF00040D9
:10DA2800B1F5000F3EBF490041EAD3715B0040EAFF
:10DA3800010062F17F02FD2A1DD8B3F1004F40EBCF
:10DA4800C25008BF20F00100704790F0000F0CF0A2
:10DA5800004C08BF49024CEA502040EA51207F3A66
:10DA6800C2BFD2F1FF0340EAC250704740F4000041
:10DA78004FF00003013A5DDC12F1190FDCBF00F032
:10DA880000407047C2F10002410021FA02F1C2F1E0
:10DA9800200200FA02FC5FEA310040F1000053EA7C
:10DAA8004C0308BF20EADC70704792F0000F00F0CA
:10DAB800004C02BF400010F4000F013AF9D040EAD0
:10DAC8000C0093F0000F01F0004C02BF490011F464
:10DAD800000F013BF9D041EA0C018FE70CEAD15362
:10DAE80092EA0C0F18BF93EA0C0F0AD030F0004CE2
:10DAF80018BF31F0004CD8D180EA010000F0004096
:10DB0800704790F0000F17BF90F0004F084691F053
:10DB1800000F91F0004F14D092EA0C0F01D142028D
:10DB28000FD193EA0C0F03D14B0218BF084608D156
:10DB380080EA010000F0004040F0FE4040F40000A0
:10DB4800704740F0FE4040F4400070474FF0FF0C33
:10DB58001CEAD0521EBF1CEAD15392EA0C0F93EA7A
:10DB68000C0F69D0A2EB030280EA010C49024FEACC
:10DB7800402037D04FF0805343EA111143EA101385
:10DB88000CF000408B4238BF5B0042F17D024FF43D
:10DB9800000C8B4224BF5B1A40EA0C00B3EB510F18
:10DBA80024BFA3EB510340EA5C00B3EB910F24BF01
:10DBB800A3EB910340EA9C00B3EBD10F24BFA3EB86
:10DBC800D10340EADC001B0118BF5FEA1C1CE0D14E
:10DBD800FD2A3FF650AF8B4240EBC25008BF20F001
:10DBE800010070470CF0004C4CEA50207F32C2BF55
:10DBF800D2F1FF0340EAC250704740F400004FF0F2
:10DC08000003013A37E792F0000F00F0004C02BF22
:10DC1800400010F4000F013AF9D040EA0C0093F0EC
:10DC2800000F01F0004C02BF490011F4000F013B46
:10DC3800F9D041EA0C0195E70CEAD15392EA0C0FAE
:10DC480008D142027FF47DAF93EA0C0F7FF470AFE6
:10DC5800084676E793EA0C0F04D14B023FF44CAF29
:10DC680008466EE730F0004C18BF31F0004CCAD1BE
:10DC780030F000427FF45CAF31F000437FF43CAFFA
:10DC88005FE700BF4FF0FF3C06E000BF4FF0010C1C
:10DC980002E000BF4FF0010C4DF804CD4FEA4002FE
:10DCA8004FEA41037FEA226C18BF7FEA236C11D048
:10DCB80001B052EA530C18BF90EA010F58BFB2EBFB
:10DCC800030088BFC81738BF6FEAE17018BF40F07B
:10DCD800010070477FEA226C02D15FEA402C05D12F
:10DCE8007FEA236CE4D15FEA412CE1D05DF8040BB4
:10DCF800704700BF844608466146FFE70FB5FFF747
:10DD0800C9FF002848BF10F1000F0FBD4DF808EDFE
:10DD1800FFF7F4FF0CBF012000205DF808FB00BFEF
:10DD28004DF808EDFFF7EAFF34BF012000205DF849
:10DD380008FB00BF4DF808EDFFF7E0FF94BF012096
:10DD480000205DF808FB00BF4DF808EDFFF7D2FF93
:10DD580094BF012000205DF808FB00BF4DF808EDD6
:10DD6800FFF7C8FF34BF012000205DF808FB00BFA3
:10DD78004FEA4002B2F1FE4F0FD34FF09E03B3EBD0
:10DD880012620DD94FEA002343F0004310F0004F10
:10DD980023FA02F018BF404270474FF00000704766
:10DDA80012F1610F01D1420205D110F0004008BF05
:10DDB8006FF0004070474FF00000704742000ED2ED
:10DDC800B2F1FE4F0BD34FF09E03B3EB126209D4AE
:10DDD8004FEA002343F0004323FA02F070474FF064
:10DDE8000000704712F1610F01D1420202D14FF0D9
:10DDF800FF3070474FF00000704700BF80B5A2B0F9
:10DE080000AF4FF0C80049F67163C0F606039847A3
:10DE18004FF00003C7F8843040F6A943C0F6020368
:10DE28009847C7F88400D7F88430002B11D140F602
:10DE3800AD73C0F602039847C7F8840007F10403DE
:10DE4800D7F88400194640F60503C0F60203984740
:10DE580000E000BF4FF0000041F2AD13C0F602032E
:10DE680098474FF00103184607F18807BD4680BD63
:10DE780080B400AF47F2B053C2F200031846BD4663
:10DE880080BC704780B582B000AF786078684FF08A
:10DE980000014FF0320246F20903C0F60103984729
:10DEA8007B684FF0010283F820207B684FF0010265
:10DEB80083F829207B684FF0000242F00F0283F8B4
:10DEC80021204FF0000283F822204FF0000283F84F
:10DED80023204FF0000283F824207B684FF00002D3
:10DEE80042F00F0283F827204FF0000283F8282021
:10DEF8007B684FF0FF3283F82A204FF0FF3283F817
:10DF08002B204FF0FF3283F82C204FF0FF3283F89C
:10DF18002D207B684FF0000242F00A0283F82E2081
:10DF28004FF0000283F82F204FF0000283F83020D2
:10DF38004FF0000283F831204FF00003184607F134
:10DF48000807BD4680BD00BF80B586B000AF7860C9
:10DF58004FF00003FB6007F10C034FF480101946E3
:10DF68004DF2C163C0F60303984738613B69002B43
:10DF780010D078684DF68D63C0F6010398474FF0CE
:10DF88002C00396941F20573C0F60203984740F244
:10DF9800426334E04FF032037B61FB68012B02D10E
:10DFA8004FF02E037B617B6978684FF480111A4625
:10DFB8004DF29173C0F60303984738613B69002B13
:10DFC80010D078684DF68D63C0F6010398474FF07E
:10DFD8002C00396941F20573C0F60203984740F2F4
:10DFE80042630CE0FB68032B07DCFB687868194682
:10DFF8004EF21103C0F6010398474FF0000318468C
:10E0080007F11807BD4680BD80B483B000AF7860C3
:10E0180039603B68012B12D17B684FF0000242F057
:10E02800140283F82E204FF0000283F82F204FF0BF
:10E03800000283F830204FF0000283F831204FF0BF
:10E048000003184607F10C07BD4680BC704700BFA7
:10E0580090B585B000AF786078684FF480114FF0C4
:10E0680032024FF004034DF23954C0F60304A047BE
:10E07800F860FB68002B01D0FB6800E0FB681846DD
:10E0880007F11407BD4690BD80B400AF4FF0000300
:10E098001846BD4680BC704780B500AF40F2693372
:10E0A800C0F6020398470346D3F83A35184680BDB0
:10E0B80080B582B000AF786078684FF000014FF00B
:10E0C800680246F20903C0F6010398474FF00003BF
:10E0D800184607F10807BD4680BD00BF80B584B06B
:10E0E80000AF78607B68002B02D140F2853373E083
:10E0F80040F26933C0F6020398470346D3F83A352D
:10E10800C72B02D940F25C6366E07B68B3F9003044
:10E118009BB21BB218464EF29953C0F601039847BA
:10E12800F860FB68002B2EDA40F26933C0F6020370
:10E1380098470346D3F83A35FB6040F26933C0F696
:10E14800020398470346D3F83A2502F10102C3F8BF
:10E158003A257B6803F1490318464FF000014FF058
:10E16800070246F20903C0F6010398477B6803F1EA
:10E178005C0318464FF000014FF0070246F209030E
:10E18800C0F6010398477868F9684FF24573C0F6FE
:10E1980003039847B860BB68002B08D04FF00F0006
:10E1A800B96841F2DD33C0F60203984713E04FF433
:10E1B800803040F25553C0F602039847B860BB68F8
:10E1C800002B08D04FF00F00B96841F2DD33C0F6DC
:10E1D8000203984700BFBB68184607F11007BD4601
:10E1E80080BD00BF80B596B000AF786039603B68ED
:10E1F800012B6ADC07F10803184679684FF004021E
:10E2080045F67573C0F60103984778684FF000012A
:10E218004FF0680246F20903C0F6010398473A89AD
:10E228007B681A807B6803F1020207F1080303F197
:10E2380002031046194646F20553C0F601039847F3
:10E24800BA7E7B6883F82220FA7E7B6883F82320D5
:10E25800BA8B7B689A84FA8B7B68DA8497F82020DB
:10E268007B6883F82820B7F921309AB27B68A3F835
:10E27800292097F823207B6883F82B207A6A7B680B
:10E28800DA62BA6A7B681A637B6803F1340307F1C0
:10E298002C02106818609188927999809A717B682D
:10E2A80003F13B0307F133021168196091889279F1
:10E2B80099809A717B6803F1420307F13A02116869
:10E2C80019609188927999809A713B68022B15DCC4
:10E2D8007B684FF0000283F864204FF0000283F857
:10E2E80065204FF0000283F866204FF0000283F8A3
:10E2F80067207B684FF0000283F863204FF000032B
:10E30800184607F15807BD4680BD00BF90B583B0D9
:10E3180000AF786039603B68002B02D140F285334A
:10E3280018E07B68002B0ADB7C6840F26933C0F692
:10E33800020398470346D3F83A359C4202D340F289
:10E34800853307E0386879684FF24573C0F60303F0
:10E3580098470346184607F10C07BD4690BD00BF15
:10E3680080B582B000AF40F26933C0F60203984727
:10E3780003464FF0000283F83A254FF0000283F875
:10E388003B254FF0000283F83C254FF0000283F84C
:10E398003D254FF4803040F25553C0F602039847AC
:10E3A80078607B68002B08D04FF00F00796841F245
:10E3B800DD33C0F60203984700BF7B68184607F1B3
:10E3C8000807BD4680BD00BF90B5A1B000AF0346A9
:10E3D800FB804FF00003FB674FF00003BB6718E0BA
:10E3E80007F10C031846B96F4FF068024FF6F103B6
:10E3F800C0F603039847F867FB6F002B61D1BB8910
:10E40800B7F906201BB29A420FD0BB6F03F1010384
:10E41800BB67BC6F40F26933C0F6020398470346F6
:10E42800D3F83A359C42DBD300E000BF40F26933B1
:10E43800C0F6020398470346D3F83A3503F1FF3391
:10E448007B67BA6F7B6F9A421BDA07F10C03184699
:10E45800796F4FF068024FF6F103C0F6030398474F
:10E46800F867FB6F002B2ED107F10C031846B96F24
:10E478004FF24573C0F603039847F867FB6F002B0C
:10E4880023D140F26933C0F6020398470346D3F814
:10E498003A2502F1FF32C3F83A254FF4803040F2B2
:10E4A8005553C0F602039847F867FB6F002B0DD051
:10E4B8004FF00F00F96F41F2DD33C0F602039847C1
:10E4C80004E000BF02E000BF00E000BFFB6F184699
:10E4D80007F18407BD4690BD90B585B000AF786060
:10E4E80039604FF00003FB601DE03868F9684FF0B1
:10E4F80068024FF6F103C0F603039847B860BB689B
:10E50800002B01D0BB681BE03B68B3F900309BB21D
:10E518001AB27B689A4202D14FF0000310E0FB6800
:10E5280003F10103FB60FC6840F26933C0F60203A3
:10E5380098470346D3F83A359C42D6D340F28E33F7
:10E54800184607F11407BD4690BD00BF80B582B0DC
:10E5580000AF786039607B68002B06DB7B68B3F519
:10E56800937F02D83B68002B02D140F2853309E043
:10E57800386879684FF068024FF6F103C0F6030374
:10E5880098470346184607F10807BD4680BD00BFF7
:10E5980090B59FB000AF78604FF000037B671BE039
:10E5A80007F108031846796F4FF068024FF6F10338
:10E5B800C0F60303984738673B6F002B01D03B6FC9
:10E5C80017E03B891AB27B689A4201D17B6F10E051
:10E5D8007B6F03F101037B677C6F40F26933C0F600
:10E5E800020398470346D3F83A359C42D8D34FF0F4
:10E5F800FF33184607F17C07BD4690BDF0B58BB0D8
:10E6080004AF78607B6893F838301A467B6893F8D3
:10E618003930796891F83A10084607F108010090F6
:10E62800084649F6CC71C0F6060143F64924C0F6FF
:10E638000504A0477B6893F83F301A467B6893F837
:10E648004030796891F84110084607F108010090B8
:10E65800084649F6CC71C0F6060143F64924C0F6CF
:10E668000504A0477B6893F846301A467B6893F800
:10E678004730796891F84810084607F1080100907A
:10E68800084649F6CC71C0F6060143F64924C0F69F
:10E698000504A0477B68B3F849309BB21A467B68EB
:10E6A80093F84B30796891F84C100E46796891F8D8
:10E6B8004D100D46796891F84E100C46796891F81E
:10E6C8004F10084607F1080100960195029403903F
:10E6D800084649F6DC71C0F6060143F64924C0F63F
:10E6E8000504A0477B68B3F85C309BB21A467B6888
:10E6F80093F85E30796891F85F100E46796891F862
:10E7080060100D46796891F861100C46796891F8A7
:10E718006210084607F108010096019502940390DB
:10E72800084649F6DC71C0F6060143F64924C0F6EE
:10E738000504A04707F11C07BD46F0BD80B582B0AF
:10E7480000AF786078684FF000014FF4C17246F26C
:10E758000903C0F6010398477B6818464EF279739F
:10E76800C0F60103984707F10807BD4680BD00BF02
:10E7780080B582B000AF786078684FF000014FF440
:10E78800AA7246F20903C0F6010398477B684FF066
:10E79800300283F846217B684FF0FF3283F8492125
:10E7A8004FF0FF3283F84A217B684FF0010283F86B
:10E7B8004B2107F10807BD4680BD00BF90B583B067
:10E7C80000AF4FF000037B6040F26933C0F60203EC
:10E7D80098470346D3F82235002B2FD04FF000037B
:10E7E8003B6020E03B684FF4C17202FB03F247F242
:10E7F800F453C2F20003D318184639684DF6C5031E
:10E80800C0F6030398477860786841F25523C0F64C
:10E818000203984747F60963C0F6020398473B6826
:10E8280003F101033B603C6840F26933C0F6020320
:10E8380098470346D3F822359C42D3D37B681846C1
:10E8480007F10C07BD4690BD80B584B000AF786075
:10E858007B684FF4C17202FB03F247F2F453C2F231
:10E868000003D318184679684DF6C503C0F60303AC
:10E878009847F860F86841F25523C0F602039847B4
:10E88800FB68184607F11007BD4680BD90B589B0F2
:10E8980000AF4FF00003FB6140F26933C0F602039A
:10E8A80098470346D3F822353B613B69002B40F378
:10E8B800F8814FF0FF333B603B4618464FF4A851B0
:10E8C800C0F210014DF67123C0F603039847F860B3
:10E8D800F86841F25523C0F602039847FB68002BFD
:10E8E80002D04FF00D033B604FF4AA737B613B6885
:10E8F800012B03D14FF0DB037B614BE03B68022B1C
:10E9080003D14FF0DD037B6144E03B68032B03D167
:10E918004FF0DE037B613DE03B68042B03D14FF4ED
:10E928009F737B6136E03B68052B03D14FF4A073DE
:10E938007B612FE03B68062B03D140F243137B61D8
:10E9480028E03B68072B03D140F245137B6121E0A7
:10E958003B68082B03D140F249137B611AE03B68FE
:10E96800092B03D140F24B137B6113E03B680A2B60
:10E9780003D14FF4A6737B610CE03B680B2B03D1EA
:10E988004FF4A6737B6105E03B680C2B02D14FF472
:10E99800A6737B617B69B3F5AA7F02D04FF00103B0
:10E9A800FB6140F26933C0F60203984703464FF013
:10E9B800000283F822254FF0000283F823254FF048
:10E9C800000283F824254FF0000283F825254FF034
:10E9D8000003BB6160E147F60963C0F6020398478C
:10E9E800BB694FF4C17202FB03F247F2F453C2F25F
:10E9F8000003D31818464EF24573C0F60103984732
:10EA0800BB694FF4C17202FB03F247F2F453C2F23E
:10EA18000003D3181846B9697A694DF61D33C0F654
:10EA280003039847F860F86841F25523C0F60203DB
:10EA38009847FB68002B08D04FF01F00F96841F297
:10EA48000573C0F60203984722E13B680C2B11DCE2
:10EA5800BB694FF4C17202FB03F247F2F453C2F2EE
:10EA68000003D2183B68104619464EF6E943C0F633
:10EA780001039847BB694FF4C17202FB03F303F526
:10EA8800A87247F2F453C2F20003D31803F1040347
:10EA980018464FF000014FF0070246F20903C0F68E
:10EAA8000103984740F26933C0F6020398470346CA
:10EAB800D3F8F630002B62D040F26933C0F6020377
:10EAC80098470346D3F8FA30BB6047F2F453C2F2D2
:10EAD8000003BA694FF4C17101FB02F29B181B884D
:10EAE8001AB2BB689A424AD147F2F453C2F2000301
:10EAF800BA694FF4C17101FB02F29B1803F150038C
:10EB0800D3F8014040F26933C0F602039847034640
:10EB1800D3F8FE2013464FEAC3739B1A4FEA430308
:10EB2800E3187B607B68C3F100037B60BB694FF42B
:10EB3800C17202FB03F303F5A87247F2F453C2F261
:10EB48000003D31803F10403184642F2E913C0F690
:10EB580005039847BB694FF4C17202FB03F303F541
:10EB6800A87247F2F453C2F20003D31803F1040366
:10EB78001846796842F6DD33C0F605039847BB6945
:10EB88004FF4C17202FB03F247F2F453C2F20003DE
:10EB9800D31818464EF62573C0F60103984747F276
:10EBA800F453C2F20003BA694FF4C17101FB02F2D7
:10EBB8009B189B78002B3BD147F2F453C2F2000319
:10EBC800BA694FF4C17101FB02F29B1803F5A073F7
:10EBD8001B79022B0ED147F2F453C2F20003BA6933
:10EBE8004FF4C17101FB02F29B1803F5BC733A4A5A
:10EBF800C3F8052047F2F453C2F20003BA694FF490
:10EC0800C17101FB02F29B1803F5A0731B79032B5A
:10EC18000ED147F2F453C2F20003BA694FF4C1713E
:10EC280001FB02F29B1803F5BC732C4AC3F80520BC
:10EC380040F26933C0F6020398470346D3F8222509
:10EC480002F10102C3F8222547F2F453C2F200038D
:10EC5800BA694FF4C17101FB02F29B181B881BB201
:10EC68004FF01300194641F64113C0F602039847C6
:10EC7800BB694FF4C17202FB03F247F2F453C2F2CC
:10EC88000003D318184640F20573C0F602039847EC
:10EC9800BB6903F10103BB61BA693B699A42FFF69C
:10ECA8009AAE40F26933C0F6020398470346D3F898
:10ECB80022253B699A4202D040F2436307E0FB6990
:10ECC800002B02D14FF0000301E040F25A631846CE
:10ECD80007F12407BD4690BD00FF7F4700000000F4
:10ECE800B0B5BCB000AF786039607B6807F1080147
:10ECF8001A464FF0DE03084611461A4645F6757364
:10ED0800C0F6010398473B68012B07D14FF0000379
:10ED180087F8E3304FF0000387F8E4303B68022BB4
:10ED280003DC4FF0010387F8E5303B68032B00F361
:10ED3800B98097F8E3207B6883F8642097F8E4208B
:10ED48007B6883F8652097F8E5207B6883F8662060
:10ED58007B6803F167031D4607F16C040FCC28603C
:10ED68006960AA60EB6023782B74D7F87E207B68F3
:10ED7800C3F87920D7F882307A68C2F87D30D7F89E
:10ED880086307A68C2F88130D7F88A307A68C2F853
:10ED98008530D7F88E307A68C2F88930D7F8923043
:10EDA8007A68C2F88D3097F896207B6883F89120AE
:10EDB80097F897207B6883F8922097F898207B68CB
:10EDC80083F8932097F899207B6883F8942097F824
:10EDD8009A207B6883F895204FF00003C7F8EC3041
:10EDE8004BE0D7F8EC3003F164034FEA430307F133
:10EDF800F002D31833F8E13C99B27B68D7F8EC20DD
:10EE080002F1980223F812104FF00003C7F8E83017
:10EE180029E0D7F8EC2013464FEA83039B18D7F86C
:10EE2800E8209B1803F144034FEA430307F1F0027B
:10EE3800D31833F8DD3C99B27868D7F8EC2013463C
:10EE48004FEA83039B18D7F8E8209B1803F1740353
:10EE58004FEA4303C3180A465A80D7F8E83003F14B
:10EE68000103C7F8E830D7F8E830042BD1DDD7F82C
:10EE7800EC3003F10103C7F8EC30D7F8EC30052B80
:10EE8800AFDD7B684FF0000283F896204FF0000258
:10EE980083F897204FF0000283F898204FF0000283
:10EEA80083F899203B68042B10DC7B684FF0000244
:10EEB80083F83F214FF0000283F840214FF0000211
:10EEC80083F841214FF0000283F842213B68072B69
:10EED80008DC7B684FF0FF3283F849214FF0FF329E
:10EEE80083F84A213B68092B04DC7B684FF0010258
:10EEF80083F84B213B680C2B07DC7B68064AC3F878
:10EF08004C217B68044AC3F850214FF0000318468F
:10EF180007F1F007BD46B0BD0000000080B584B021
:10EF280000AF78604FF00003FB607B689B78082B8C
:10EF38001BD17B68D3F84D30184647F20D03C0F655
:10EF480003039847B860B86849F24943C0F602031A
:10EF58009847F860FB68002B07D04FF02700F96846
:10EF680041F20573C0F602039847FB68184607F19B
:10EF78001007BD4680BD00BF80B584B000AF786083
:10EF88004FF00003FB607B689B78082B1BD17B68E4
:10EF9800D3F84D30184647F20D03C0F603039847DF
:10EFA800B860B86849F27D43C0F602039847F86034
:10EFB800FB68002B07D04FF02800F96841F2057371
:10EFC800C0F602039847FB68184607F11007BD46CC
:10EFD80080BD00BF80B500AF40F26933C0F60203C0
:10EFE80098470346D3F82235184680BD80B584B0CB
:10EFF80000AF4EF6DD73C0F60103984778604FF016
:10F008000003BB604FF00003FB6018E0F8684FF2A4
:10F018007143C0F60103984738603B68002B09D05C
:10F028003B6893F86630002B05D0BB6803F10103F9
:10F03800BB6000E000BFFB6803F10103FB60FA68F6
:10F048007B689A42E2DBBB68184607F11007BD46A9
:10F0580080BD00BF80B586B000AF78607B68002BAC
:10F0680002D140F28533D9E07B68B3F900309BB216
:10F078001BB218464FF2A933C0F6010398477861CE
:10F088007B68B3F900309BB21BB218464FF20D43B0
:10F09800C0F60103984738613B69002B48D07B696B
:10F0A800002B45DB7B68B3F900309BB21BB24FF0F5
:10F0B8001200194641F64113C0F6020398477B68CF
:10F0C8009A783B699B789A4206D038694EF2457324
:10F0D800C0F60103984764E07B689B78062B0ED046
:10F0E8007B68D3F84D203B69D3F84D309A4206D05F
:10F0F80038694EF24573C0F60103984751E07B68C2
:10F108009B78062B4DD17B6893F85E203B6993F87A
:10F118005E309A4205D17B681A6E3B691B6E9A4233
:10F128003FD038694EF24573C0F60103984738E07E
:10F138004EF6DD73C0F601039847B860BB683D2BF7
:10F1480002DD40F2416369E0BB687B61BB684FF454
:10F15800C17202FB03F247F2F453C2F20003D31860
:10F168003B6140F26933C0F6020398470346D3F87F
:10F17800222502F10102C3F822257B68B3F9003089
:10F188009BB21BB24FF01100194641F64113C0F66D
:10F198000203984738694EF24573C0F60103984751
:10F1A80000E000BF3B69184679684FF4AA7245F63B
:10F1B8007573C0F6010398473B6903F5AA731846AF
:10F1C80042F2E913C0F6050398473B6918464EF624
:10F1D8002573C0F6010398473B69184679694DF6CF
:10F1E800C503C0F603039847F860FB68002B13D1EA
:10F1F8004FF4803040F25553C0F602039847F86048
:10F20800FB68002B09D04FF00F00F96841F2DD339D
:10F21800C0F60203984700E000BFFB68184607F1F4
:10F228001807BD4680BD00BF80B584B000AF4FF061
:10F238000003BB604EF6DD73C0F6010398477860A3
:10F248004FF00003FB6015E0FB684FF4C17202FB4E
:10F2580003F247F2F453C2F20003D318BB60BB6851
:10F2680018464EF68173C0F601039847FB6803F110
:10F278000103FB60FA687B689A42E5DB40F2693378
:10F28800C0F60203984703464FF0000283F8222590
:10F298004FF0000283F823254FF0000283F824255D
:10F2A8004FF0000283F825254FF00003184607F1B8
:10F2B8001007BD4680BD00BF90B587B000AF78602D
:10F2C8004FF000037B614FF00003FB604EF6DD73E7
:10F2D800C0F601039847B8604FF000033B6152E065
:10F2E8003B694FF4C17202FB03F247F2F453C2F2D6
:10F2F8000003D318FB60FB68B3F900309BB21AB265
:10F308007B689A4204D03B6903F101033B613AE010
:10F31800FB6818464EF68173C0F60103984740F221
:10F328006933C0F6020398470346D3F8222502F151
:10F33800FF32C3F822253C6940F26933C0F6020364
:10F3480098470346D3F822359C4221D2BB6803F183
:10F35800FF334FF4C17202FB03F247F2F453C2F2D7
:10F368000003D318F86819464FF4AA7245F6757366
:10F37800C0F60103984738694EF65103C0F60103F9
:10F388009847786104E03A69BB689A42A8DB00E0D4
:10F3980000BF7B69184607F11C07BD4690BD00BF3A
:10F3A80080B586B000AF78604FF000033B614EF641
:10F3B800DD73C0F601039847F8604FF000037B61E6
:10F3C80014E078694FF27143C0F601039847386139
:10F3D8003B69B3F900309BB21AB27B689A4201D1FB
:10F3E8007B6909E07B6903F101037B617A69FB684A
:10F3F8009A42E6DB4FF0FF33184607F11807BD467F
:10F4080080BD00BF80B586B000AF78604FF00003C4
:10F418003B614EF6DD73C0F601039847F8604FF084
:10F4280000037B6114E078694FF27143C0F6010371
:10F43800984738613B69B3F900309BB21AB27B68D0
:10F448009A4201D13B6909E07B6903F101037B61C1
:10F458007A69FB689A42E6DB4FF00003184607F129
:10F468001807BD4680BD00BF80B582B000AF786088
:10F478007B68002B08DB4EF6DD73C0F60103984766
:10F4880002467B689A4202DC4FF0000309E07B6881
:10F498004FF4C17202FB03F247F2F453C2F20003C5
:10F4A800D318184607F10807BD4680BD80B586B059
:10F4B80000AF0346FB804FF000033B614EF6DD735F
:10F4C800C0F601039847F8604FF000037B6115E030
:10F4D80078694FF27143C0F60103984738613B6978
:10F4E800B3F949319BB2B7F906201BB29A4201D150
:10F4F8003B6909E07B6903F101037B617A69FB6879
:10F508009A42E5DB4FF00003184607F11807BD469D
:10F5180080BD00BF80B582B000AF786078684FF0DA
:10F5280000014FF0800246F20903C0F60103984734
:10F538004FF00003184607F10807BD4680BD00BF1D
:10F5480080B586B000AF78604FF00003FB6007F12C
:10F558000C034FF48060C0F2100019464DF2C163ED
:10F56800C0F60303984778617B69002B10D0786850
:10F578004FF21D53C0F6010398474FF02D007969EB
:10F5880041F20573C0F60203984740F2426325E052
:10F598004FF080033B613B6978684FF48061C0F2AB
:10F5A80010011A464DF29173C0F60303984778612B
:10F5B8007B69002B10D078684FF21D53C0F6010309
:10F5C80098474FF02D00796941F20573C0F60203A0
:10F5D800984740F2426301E04FF00003184607F1F4
:10F5E8001807BD4680BD00BF90B585B000AF7860F4
:10F5F80078684FF48061C0F210014FF080024FF03C
:10F6080001034DF23954C0F60304A047F860FB68C3
:10F61800002B01D0FB6800E0FB68184607F11407CF
:10F62800BD4690BD80B584B000AF786078684FF073
:10F6380000014FF0540246F20903C0F6010398474F
:10F648007B684FF000021A734FF0000262F03D022F
:10F658005A734FF0000242F001029A734FF0000211
:10F66800DA737B684FF000021A744FF000025A7484
:10F678004FF000029A744FF00002DA747B684FF082
:10F68800000242F001021A754FF000025A754FF05D
:10F6980000029A754FF00002DA757B684FF000029D
:10F6A80042F008021A764FF000025A764FF0000234
:10F6B8009A764FF00002DA767B684FF0000262F02B
:10F6C8007F021A774FF0000242F025025A774FF076
:10F6D80000029A774FF00002DA777B684FF0000259
:10F6E80083F820204FF0000283F821204FF0000219
:10F6F80083F822204FF0000283F823207B684FF024
:10F70800000242F0010283F824204FF0000283F83F
:10F7180025204FF0000283F826204FF0000283F8DE
:10F7280027207B684FF0000242F0080283F8282067
:10F738004FF0000283F829204FF0000283F82A20B6
:10F748004FF0000283F82B207B684FF0000242F054
:10F7580002021A724FF000025A724FF000029A72B7
:10F768004FF00002DA724FF00003FB6013E07A6892
:10F77800FB68D31803F12C034FF000021A707A6863
:10F78800FB68D31803F134034FF000021A70FB68CA
:10F7980003F10103FB60FB68072BE8DD7B684FF092
:10F7A800000262F00B0283F83C204FF0000242F0A6
:10F7B800010283F83D204FF0000283F83E204FF00D
:10F7C800000283F83F207B684FF0000262F00B02D2
:10F7D80083F840204FF0000242F0010283F84120F4
:10F7E8004FF0000283F842204FF0000283F84320D4
:10F7F8007B684FF0000283F844204FF0000283F842
:10F8080045204FF0000283F846204FF0000283F8AD
:10F8180047207B684FF0FF3283F848204FF0FF32D3
:10F8280083F849204FF0FF3283F84A204FF0FF3227
:10F8380083F84B207B684FF0000242F0050283F802
:10F848004C204FF0000283F84D204FF0000283F85F
:10F858004E204FF0000283F84F207B684FF00002E3
:10F8680042F0050283F850204FF0000283F851203F
:10F878004FF0000283F852204FF0000283F8532023
:10F888004FF00003184607F11007BD4680BD00BFC2
:10F8980080B586B000AF78604FF00003BB6007F119
:10F8A80008034FF40060C0F2100019464DF2C1631E
:10F8B800C0F603039847F860FB68002B10D07868FF
:10F8C8004FF22D63C0F6010398474FF02E00F968F8
:10F8D80041F20573C0F60203984740F242634DE0D7
:10F8E8004FF054037B61BB68012B02D14FF04403F6
:10F8F8007B61BB68022B02D14FF04C037B61BB6874
:10F90800032B02D14FF044037B617B6978684FF485
:10F918000061C0F210011A464DF29173C0F603035C
:10F928009847F860FB68002B10D078684FF22D6379
:10F93800C0F6010398474FF02E00F96841F20573AD
:10F94800C0F60203984740F2426317E04FF0000305
:10F958003B6103E03B6903F101033B613B69072B12
:10F96800F8DDBB68042B07DCBB68786819464FF6DE
:10F978009113C0F6010398474FF00003184607F1AA
:10F988001807BD4680BD00BF80B485B000AF786061
:10F9980039603B68012B44DC4FF00003FB6013E047
:10F9A8007A68FB68D31803F12C034FF000021A7031
:10F9B8007A68FB68D31803F134034FF000021A7019
:10F9C800FB6803F10103FB60FB68072BE8DD7B683C
:10F9D8004FF0000262F0170283F83C204FF000025B
:10F9E80042F0030283F83D204FF0000283F83E20E6
:10F9F8004FF0000283F83F207B684FF0000262F06E
:10FA0800170283F840204FF0000242F0030283F807
:10FA180041204FF0000283F842204FF0000283F8A3
:10FA280043203B68022B29DC7B684FF0000262F020
:10FA3800170283F83C204FF0000242F0030283F8DB
:10FA48003D204FF0000283F83E204FF0000283F87B
:10FA58003F207B684FF0000262F0170283F84020D5
:10FA68004FF0000242F0030283F841204FF00002F9
:10FA780083F842204FF0000283F843203B68032BB1
:10FA880047DC7B684FF0000283F844204FF0000207
:10FA980083F845204FF0000283F846204FF000021B
:10FAA80083F847207B684FF0FF3283F848204FF0F7
:10FAB800FF3283F849204FF0FF3283F84A204FF095
:10FAC800FF3283F84B207B684FF0000242F00502BA
:10FAD80083F84C204FF0000283F84D204FF00002CD
:10FAE80083F84E204FF0000283F84F207B684FF0D8
:10FAF800000242F0050283F850204FF0000283F81C
:10FB080051204FF0000283F852204FF0000283F892
:10FB180053203B68042B00F3A8807B685B69002BAB
:10FB28000ED17B684FF0000242F001021A754FF0C7
:10FB380000025A754FF000029A754FF00002DA750C
:10FB48007B685B69012B0ED17B684FF0000242F0A5
:10FB580002021A754FF000025A754FF000029A75AA
:10FB68004FF00002DA757B689B69022B0ED17B6827
:10FB78004FF0000242F007021A764FF000025A7660
:10FB88004FF000029A764FF00002DA767B689B69A4
:10FB9800032B0ED17B684FF0000242F008021A7660
:10FBA8004FF000025A764FF000029A764FF00002AA
:10FBB800DA767B685B6A002B12D17B684FF0000213
:10FBC80042F0010283F824204FF0000283F8252038
:10FBD8004FF0000283F826204FF0000283F8272018
:10FBE8007B685B6A012B12D17B684FF0000242F000
:10FBF800020283F824204FF0000283F825204FF0FA
:10FC0800000283F826204FF0000283F827207B6843
:10FC18009B6A022B12D17B684FF0000242F0070268
:10FC280083F828204FF0000283F829204FF00002C3
:10FC380083F82A204FF0000283F82B207B689B6A08
:10FC4800032B12D17B684FF0000242F0080283F8C0
:10FC580028204FF0000283F829204FF0000283F893
:10FC68002A204FF0000283F82B204FF0000318469B
:10FC780007F11407BD4680BC704700BF90B585B03A
:10FC880000AF786078684FF40061C0F210014FF05F
:10FC980054024FF005034DF23954C0F60304A0474F
:10FCA800B860BB68002B01D0BB680BE04FF00003C5
:10FCB800FB6003E0FB6803F10103FB60FB68072BB3
:10FCC800F8DDBB68184607F11407BD4690BD00BFB4
:10FCD800B0B582B000AF786078684FF000014FF09F
:10FCE800100246F20903C0F6010398477B684FF0FB
:10FCF80000021A704FF000025A704FF000029A701A
:10FD08004FF00002DA707B684FF0000242F0010207
:10FD18001A724FF000025A724FF000029A724FF0B6
:10FD28000002DA727B684FF0000242F001021A7397
:10FD38004FF000025A734FF000029A734FF000021E
:10FD4800DA737B684FF0000242F050021A714FF0EC
:10FD580000025A714FF000029A714FF00002DA71F6
:10FD68007B684FF0000242F010021A744FF0000254
:10FD780042F00E025A744FF000029A744FF00002DB
:10FD8800DA747B684FF000021A754FF000025A755A
:10FD98004FF000029A754FF00002DA757B6803F1A4
:10FDA800180249F6FC73C0F6060315461C460FCC2C
:10FDB80028606960AA60EB6003CC286169612288C9
:10FDC800A3782A83AB764FF00003184607F108079B
:10FDD800BD46B0BD80B586B000AF78604FF0000377
:10FDE800FB6007F10C034FF44060C0F210001946A5
:10FDF8004DF2C163C0F60303984778617B69002B15
:10FE080010D078684FF6D943C0F6010398474FF0F1
:10FE18002F00796941F20573C0F60203984740F252
:10FE2800426325E04FF4CC733B613B6978684FF43B
:10FE38004061C0F210011A464DF29173C0F60303F7
:10FE4800984778617B69002B10D078684FF6D943C2
:10FE5800C0F6010398474FF02F00796941F2057306
:10FE6800C0F60203984740F2426301E04FF00003F6
:10FE7800184607F11807BD4680BD00BF90B585B08C
:10FE880000AF786078684FF44061C0F210014FF419
:10FE9800CC724FF002034DF23954C0F60304A04768
:10FEA800F860FB68002B01D0FB6800E0FB6818468F
:10FEB80007F11407BD4690BDB0B582B000AF7860B9
:10FEC80078684FF000014FF4217246F20903C0F63A
:10FED800010398477A684AF21803C0F606031546E4
:10FEE8001C460FCC28606960AA60EB602288A37862
:10FEF8002A82AB747B6803F184024AF22C03C0F6B1
:10FF0800060315461C460FCC28606960AA60EB60A2
:10FF1800206828617B6803F582724AF24003C0F6C4
:10FF2800060314461D460FCD20606160A260E360A1
:10FF380028682061AA88AB79A282A3757B6803F53B
:10FF4800C2724AF22C03C0F6060315461C460FCCB3
:10FF580028606960AA60EB60206828617B6803F507
:10FF680001724AF25803C0F60603186810601B793C
:10FF780013717B684FF0000262F0260283F880203C
:10FF88004FF0000242F05D0283F881204FF000023A
:10FF980083F882204FF0000283F883204FF000039B
:10FFA800184607F10807BD46B0BD00BF80B586B04A
:10FFB80000AF78604FF00003FB6007F10C034FF4CB
:10FFC8008050C0F2100019464DF2C163C0F6030319
:10FFD800984738613B69002B10D078684FF6C163A9
:10FFE800C0F6010398474FF03000396941F20573B4
:08FFF800C0F60203984740F235
:020000040802F0
:1000000042633CE04FF421737B61FB68012B02D11A
:100010004FF4C2737B61FB68022B02D14FF4017372
:100020007B617B6978684FF48051C0F210011A46F9
:100030004DF29173C0F60303984738613B69002B7A
:1000400010D078684FF6C163C0F6010398474FF0AF
:100050003000396941F20573C0F60203984740F257
:1000600042630CE0FB68022B07DCFB6878681946EA
:1000700040F28903C0F6020398474FF00003184688
:1000800007F11807BD4680BDB0B483B000AF7860FB
:1000900039603B68012B0FD17B6803F5C2724AF2CD
:1000A0002C03C0F6060315461C460FCC2860696079
:1000B000AA60EB60206828613B68022B0ADC7B6841
:1000C00003F501724AF25803C0F60603186810607F
:1000D0001B7913714FF00003184607F10C07BD465A
:1000E000B0BC704790B585B000AF786078684FF4C9
:1000F0008051C0F210014FF421724FF003034DF212
:100100003954C0F60304A047F860FB68002B01D007
:10011000FB6800E0FB68184607F11407BD4690BD78
:1001200080B582B000AF786078684FF000014FF082
:100130001C0246F20903C0F6010398474FF0000382
:10014000184607F10807BD4680BD00BF80B586B0E0
:1001500000AF78604FF00003FB6007F10C034FF431
:10016000A050C0F2100019464DF2C163C0F603035F
:10017000984738613B69002B10D0786840F2211312
:10018000C0F6020398474FF03100396941F2057318
:10019000C0F60203984740F2426367E04FF01C0349
:1001A0007B61FB68032B02D14FF010037B61FB687E
:1001B000022B02D14FF014037B61FB68012B02D1AB
:1001C0004FF018037B617B6978684FF4A051C0F24F
:1001D00010011A464DF29173C0F603039847386137
:1001E0003B69002B10D0786840F22113C0F602035F
:1001F00098474FF03100396941F20573C0F60203A8
:10020000984740F2426331E0FB68012B0CDC7B68CD
:100210004FF000021A744FF000025A744FF00002BF
:100220009A744FF00002DA74FB68022B0CDC7B68D6
:100230004FF000021A754FF000025A754FF000029D
:100240009A754FF00002DA75FB68032B0CDC7B68B3
:100250004FF000021A764FF000025A764FF000027B
:100260009A764FF00002DA764FF00003184607F155
:100270001807BD4680BD00BF90B585B000AF78605F
:1002800078684FF4A051C0F210014FF01C024FF0FB
:1002900004034DF23954C0F60304A047F860FB682C
:1002A000002B01D0FB6800E0FB68184607F114073B
:1002B000BD4690BD80B500AF4DF27030C2F2000077
:1002C0004FF0000140F23E5246F20903C0F601032E
:1002D00098474DF27030C2F200004DF68D63C0F6C3
:1002E000010398470F484FF21D53C0F6010398478A
:1002F0000D484FF22D63C0F6010398470B484FF6A7
:10030000D943C0F60103984709484FF6C163C0F6C8
:1003100001039847074840F22113C0F602039847AB
:1003200080BD00BFA2D3002022D4002076D40020BC
:100330000ED6002092D8002080B582B000AF786041
:100340007B68002B0AD078684FF000014FF4C1722F
:1003500046F20903C0F60103984700E000BF07F129
:100360000807BD4680BD00BF80B400AF4DF27033BA
:10037000C2F200031846BD4680BC704780B582B00B
:1003800000AF40F2B523C0F6020398474DF270303B
:10039000C2F200004DF65173C0F601039847786031
:1003A00028484FF24953C0F6010398477860264821
:1003B0004FF69903C0F601039847786023484FF63B
:1003C000DD53C0F601039847786021484FF6B573B6
:1003D000C0F60103984778601E4840F24D13C0F6FE
:1003E0000203984778607B68002B24D14DF270336C
:1003F000C2F20003D3F82235002B0FD04EF695033E
:10040000C0F60103984778607A6840F25A639A42CE
:1004100004D14EF2C573C0F6010398474DF2703314
:10042000C2F20003D3F83A35002B04D040F259430E
:10043000C0F6020398474FF00003184607F108077B
:10044000BD4680BDA2D3002022D4002076D4002057
:100450000ED6002092D8002080B59EB000AF4FF09D
:10046000FF33BB6607F1680318464FF43541C0F20D
:1004700010014DF67123C0F60303984738673B6FB0
:10048000002B01D03B6F5FE0BB6E022B02DD4FF013
:10049000000359E04FF04E03FB66BB6E012B03D106
:1004A0004FF04E03FB660DE0BB6E022B03D14FF005
:1004B0006303FB6606E04EF26933C0F6010398471A
:1004C000034641E040F26933C0F602039847034611
:1004D000D3F83A3503F1FF337B6731E03B461846EA
:1004E000796FFA6E4FF6F103C0F603039847386749
:1004F0003B6F002B05D04EF26933C0F601039847DD
:1005000021E0BB6E3A46104619464EF2ED13C0F696
:10051000010398473B461846796F4FF24573C0F682
:100520000303984738673B6F002B05D04EF26933C1
:10053000C0F60103984706E07B6F03F1FF337B674A
:100540007B6F002BCADA3B6F184607F17807BD4670
:1005500080BD00BF80B584B000AF78604FF000036D
:10056000FB607B68B3F5006F32D0B3F5006F0DDC34
:10057000202B22D0202B04DC022B1ED0102B1CD0D1
:1005800017E0402B2CD0802B2AD012E0B3F5804FFF
:1005900026D0B3F5804F06DCB3F5805F28D0B3F5E5
:1005A000005F2DD005E0B3F5004F19D0B3F5803FC3
:1005B0002ED04FF00003FB6032E04DF27030C2F2FB
:1005C00000004EF25903C0F601039847F86027E097
:1005D00016484FF2F153C0F601039847F8601FE048
:1005E00013484FF68543C0F601039847F86017E0BB
:1005F00010484FF68563C0F601039847F8600FE096
:100600000D4840F2E503C0F602039847F86007E0A2
:100610000A4840F27923C0F602039847F86000BF09
:10062000FB68184607F11007BD4680BDA2D3002025
:1006300022D4002076D400200ED6002092D80020AC
:1006400080B400AF4DF27033C2F20003D3F81E3312
:10065000002B02D14FF0000308E0064B1B78002B63
:1006600002D14FF0000301E04FF001031846BD46F0
:1006700080BC70470ED6002080B400AF4DF27033BE
:10068000C2F20003D3F80A31002B02D14FF000036D
:1006900013E04DF27033C2F20003D3F80E31002B99
:1006A00002D14FF0000308E0064B1B78002B02D16B
:1006B0004FF0000301E04FF001031846BD4680BC37
:1006C000704700BF8ED4002080B483B000AF786044
:1006D0004DF27033C2F20003D3F82A207B68134036
:1006E000184607F10C07BD4680BC704780B483B044
:1006F00000AF78607B68002B00BF07F10C07BD4698
:1007000080BC704780B483B000AF786007F10C07FD
:10071000BD4680BC704700BF80B483B000AF786036
:1007200007F10C07BD4680BC704700BF80B483B0A2
:1007300000AF786007F10C07BD4680BC704700BF72
:1007400080B483B000AF786007F10C07BD4680BC71
:10075000704700BF80B483B000AF786007F10C072A
:10076000BD4680BC704700BF80B483B000AF7860E6
:1007700007F10C07BD4680BC704700BF80B483B052
:1007800000AF78604DF6B003C2F200031A687B68D0
:100790001A434DF6B003C2F200031A604FF0000393
:1007A000184607F10C07BD4680BC704780B400AF07
:1007B0004DF6B003C2F200034FF000021A604FF092
:1007C00000031846BD4680BC704700BF80B400AF30
:1007D0004DF6B003C2F200031B68002B0CBF0023D0
:1007E0000123DBB21846BD4680BC704780B400AF21
:1007F0004DF6B003C2F200031B681846BD4680BC2C
:10080000704700BF80B582B000AF786039603B6848
:10081000002B00F044827B6840F63602934200F0E1
:10082000408140F63602934259DC40F2DE52934258
:1008300000F0C98040F2DE52934226DCB3F58A6FA5
:1008400000F00381B3F58A6F0FDC40F24E42934211
:1008500000F0E58040F24E42934200F3EB8040F21C
:100860004D42934200F0D08096E040F252429342D3
:1008700000F0018140F252429342C0F2F18040F216
:10088000DD52934200F0948086E040F26E72934213
:1008900000F0548140F26E7293420DDCB3F5BC6FF0
:1008A00000F0A780B3F5BC6FC0F2988040F26D7283
:1008B000934200F038816FE0B3F5EE6F00F05481A1
:1008C000B3F5EE6FC0F2458140F27172934200F0D1
:1008D000568140F63502934200F0D8805CE0B3F5D3
:1008E000106F00F07881B3F5106F2DDC40F63A02FE
:1008F000934200F0028140F63A0293420ADC40F64D
:100900003802934200F0E38040F63802934200F34D
:10091000E980D1E040F6FD02934200F03B8140F6D1
:10092000FD02934205DC40F63B02934200F0F0806A
:1009300032E040F6FE02934200F0378140F6FF02BB
:10094000934200F03D8127E040F60412934200F00C
:100950006E8140F6041293420ADC40F60212934282
:1009600000F04F8140F60212934200F355813DE1C1
:1009700040F60612934200F0708140F60612934250
:10098000C0F2608140F60712934200F0718140F698
:100990000812934200F0778138684AF26001C0F68D
:1009A00006017A6843F64923C0F60503984777E1C4
:1009B00038684AF27C01C0F6060143F64923C0F6C6
:1009C000050398476CE138684AF29401C0F60601C5
:1009D00043F64923C0F60503984761E138684AF2B7
:1009E000AC01C0F6060143F64923C0F6050398475B
:1009F00056E138684AF2C401C0F6060143F64923BD
:100A0000C0F6050398474BE138684AF2D801C0F6B2
:100A1000060143F64923C0F60503984740E13868CC
:100A20004AF2F401C0F6060143F64923C0F6050375
:100A3000984735E138684AF22411C0F6060143F6BA
:100A40004923C0F6050398472AE138684AF2441161
:100A5000C0F6060143F64923C0F6050398471FE197
:100A600038684AF26011C0F6060143F64923C0F621
:100A70000503984714E138684AF27C11C0F6060174
:100A800043F64923C0F60503984709E138684AF25E
:100A90009411C0F6060143F64923C0F605039847B2
:100AA000FEE038684AF2B011C0F6060143F6492369
:100AB000C0F605039847F3E038684AF2E011C0F643
:100AC000060143F64923C0F605039847E8E0386875
:100AD0004AF20021C0F6060143F64923C0F6050399
:100AE0009847DDE038684AF21C21C0F6060143F65B
:100AF0004923C0F605039847D2E038684AF2382106
:100B0000C0F6060143F64923C0F605039847C7E03F
:100B100038684AF25021C0F6060143F64923C0F670
:100B200005039847BCE038684AF27821C0F6060110
:100B300043F64923C0F605039847B1E038684AF206
:100B4000B021C0F6060143F64923C0F605039847D5
:100B5000A6E038684AF2E421C0F6060143F64923CC
:100B6000C0F6050398479BE038684AF23431C0F676
:100B7000060143F64923C0F60503984790E038681C
:100B80004AF27831C0F6060143F64923C0F6050360
:100B9000984785E038684AF2A431C0F6060143F66A
:100BA0004923C0F6050398477AE038684AF2D03105
:100BB000C0F6060143F64923C0F6050398476FE0E7
:100BC00038684AF2E431C0F6060143F64923C0F61C
:100BD0000503984764E038684AF2FC31C0F6060124
:100BE00043F64923C0F60503984759E038684AF2AE
:100BF0002041C0F6060143F64923C0F60503984795
:100C00004EE038684AF24041C0F6060143F64923F7
:100C1000C0F60503984743E038684AF26041C0F6E1
:100C2000060143F64923C0F60503984738E03868C3
:100C30004AF27441C0F6060143F64923C0F60503A3
:100C400098472DE038684AF28841C0F6060143F61D
:100C50004923C0F60503984722E038684AF2A441C8
:100C6000C0F6060143F64923C0F60503984717E08E
:100C700038684AF2C441C0F6060143F64923C0F67B
:100C8000050398470CE038684AF2E441C0F60601D3
:100C900043F64923C0F60503984700BF00E000BFB4
:100CA00007F10807BD4680BD80B582B000AF4DF6A4
:100CB000D400C2F200004FF000014FF4357246F24A
:100CC0000903C0F6010398474FF000037B604DF61F
:100CD000D403C2F200034FF00002C3F880224DF6A5
:100CE000D403C2F200034FF0FF32C3F87C224DF66A
:100CF000D403C2F200034FF000025A604DF6D40351
:100D0000C2F200034FF0FF32C3F868224DF6D4035D
:100D1000C2F200034FF0FF32C3F86C224DF6D40349
:100D2000C2F200034FF0FF0283F8AF224DF6D40366
:100D3000C2F200034FF0FF0283F8B0224DF6D40355
:100D4000C2F200034FF0FF0283F8B1224DF6D40344
:100D5000C2F200034FF0FF0283F8B2224DF6D40333
:100D6000C2F200034FF0FF0283F8B3224DF6D40322
:100D7000C2F200034FF0FF0283F8B4224DF6D40311
:100D8000C2F200034FF0FF0283F8B9224DF6D403FC
:100D9000C2F200034FF0FF0283F8AE2247F6C963A8
:100DA000C0F60203984738603B6803F1FF33052B18
:100DB0000ED801A252F823F0D10D0208D10D02087D
:100DC000D10D0208D10D0208D10D0208D10D020883
:100DD00000BF4FF2E873C1F6FF731A684DF6D403F3
:100DE000C2F20003C3F890224FF2EC73C1F6FF7316
:100DF0001A684DF6D403C2F20003C3F894224FF2EE
:100E0000F073C1F6FF731A684DF6D403C2F2000303
:100E1000C3F8982240F2B523C0F60203984747F280
:100E20007123C0F60303984741F64D63C0F60303F0
:100E300098475B4841F26143C0F60303984759481D
:100E400041F2B573C0F60303984747F26D63C0F6ED
:100E50000203984778607B68002B40F0938042F251
:100E6000C503C0F60203984740F69963C0F6040331
:100E7000984747F6C963C0F60203984702464DF605
:100E8000D403C2F200031A6047F6DD63C0F6020322
:100E9000984741F65970C0F6040044F2D103C0F6F9
:100EA00003039847404842F2E913C0F60503984708
:100EB0004DF6D403C2F200039B89B3F5FC6F30D921
:100EC0004DF6D403C2F200039B7B002B29D04DF6D4
:100ED000D403C2F200039B7B0C2B22D84DF6D40323
:100EE000C2F20003DB7B002B1BD04DF6D403C2F211
:100EF0000003DB7B1F2B14D84DF6D403C2F2000392
:100F00001B7C172B0DD84DF6D403C2F200035B7C7B
:100F10003B2B06D84DF6D403C2F200039B7C3B2B3F
:100F200031D94DF6D403C2F2000340F2E1729A8146
:100F30004DF6D403C2F200034FF001029A734DF64E
:100F4000D403C2F200034FF00102DA734DF6D4036A
:100F5000C2F200034FF000021A744DF6D403C2F23D
:100F600000034FF000025A744DF6D403C2F200039E
:100F70004FF000029A740C4842F2E103C0F60503F8
:100F8000984700E000BF786841F25523C0F602039D
:100F900098477B68184607F10807BD4680BD00BF2B
:100FA000E4D90020ECD80020E0D8002090B589B02A
:100FB00004AF4FF61133C0F603039847B8604FF6FD
:100FC0004D33C0F603039847B86049F60913C0F6DD
:100FD000020398474FF00003FB604EF27523C0F602
:100FE000030398474FF0000300934FF00003019371
:100FF0004FF0000302934FF00003039344F6156093
:10100000C0F602004FF000014FF4FA724FF00003F7
:1010100049F6BD74C0F60504A04778607B68012BD3
:1010200003D040F2DD53FB60B3E04FF000030093C8
:101030004FF0000301934FF0000302934FF00003C1
:10104000039345F26930C0F602004FF000014FF4FF
:10105000FA724FF0000349F6BD74C0F60504A047CC
:1010600078607B68012B03D040F2DF53FB6090E097
:101070004FF0000300934FF0000301934FF0000383
:1010800002934FF00003039345F20D20C0F60200D7
:101090004FF000014FF4FA724FF0000349F6BD74AF
:1010A000C0F60504A04778607B68012B03D040F2AE
:1010B000E153FB606DE04FF0000300934FF000033D
:1010C00001934FF0000302934FF00003039345F2A6
:1010D0007910C0F602004FF000014FF4FA724FF0A1
:1010E000000349F6BD74C0F60504A04778607B682C
:1010F000012B03D04FF4BC63FB604AE04FF00003C8
:1011000000934FF0000301934FF0000302934FF060
:101110000003039346F23120C0F602004FF00001B5
:101120004FF4FA724FF0000349F6BD74C0F605049F
:10113000A04778607B68012B03D040F2DE53FB6050
:1011400027E04FF0000300934FF0000301934FF0AE
:10115000000302934FF00003039345F24D40C0F6A5
:1011600002004FF000014FF4FA724FF0000349F60D
:10117000BD74C0F60504A04778607B68012B03D0DE
:1011800040F2E253FB6004E041F2B953C0F60103C0
:101190009847F86841F25523C0F602039847FB6868
:1011A000184607F11407BD4690BD00BF80B582B058
:1011B00000AF78607B68002B10DD4DF6D403C2F2DF
:1011C00000034FF0FF32C3F880224DF6D403C2F281
:1011D00000037A68C3F87C2200BF07E04FF00500E7
:1011E00047F6E953C0F602039847FEE707F1080700
:1011F000BD4680BD80B582B000AF78604DF6D403A7
:10120000C2F20003D3F88032002B1DD04DF6D40378
:10121000C2F20003D3F87C227B68D21A4DF6D403C5
:10122000C2F20003C3F87C224DF6D403C2F20003DD
:10123000D3F87C32002B08DC4FF0000041F2AD13F4
:10124000C0F60203984700E000BF07F10807BD465B
:1012500080BD00BF80B582B000AF78604DF6D4038A
:10126000C2F200037A685A607B68002B05D149F608
:101270001D43C0F60203984704E049F6ED33C0F67B
:101280000203984707F10807BD4680BD80B483B0CC
:1012900000AF78604DF6D403C2F200035B681846D5
:1012A00007F10C07BD4680BC704700BF80B483B017
:1012B00000AF78604DF6D403C2F200037A689A60FA
:1012C00007F10C07BD4680BC704700BF80B400AF7B
:1012D0004DF6D403C2F200039B681846BD4680BC9D
:1012E000704700BF80B400AF4DF6D403C2F20003D4
:1012F0001B681846BD4680BC704700BF80B584B0EF
:1013000000AF07F10403184642F2E913C0F60503E3
:10131000984707F104031846094942F2E143C0F631
:1013200005039847F8604DF6D403C2F200035B69E9
:10133000FA68D31A184607F11007BD4680BD00BFF2
:10134000E0D8002090B585B000AF786007F10803C1
:10135000184642F2E913C0F6050398474DF6D40348
:10136000C2F200035C6907F108037868194642F28B
:10137000E143C0F6050398470346E2184DF6D4034F
:10138000C2F200035A6107F11407BD4690BD00BFC9
:1013900090B583B000AF03463960FB71FB790E480E
:1013A00019464FF003023B6841F29944C0F603042A
:1013B000A047FA794DF6D403C2F20003C3F86822BD
:1013C0004DF6D403C2F200033A68C3F86C2207F169
:1013D0000C07BD4690BD00BFE4D9002090B585B094
:1013E00000AF03463960FB714DF6D403C2F200032F
:1013F000D3F86822FB799A4209D14DF6D403C2F2A0
:101400000003D3F86C223B689A4200F05B814FF0F6
:101410000003FB60FB79292B2FD14DF6D403C2F2D8
:10142000000393F8B232002B03D03B68002B00F08E
:101430004B814DF6D403C2F2000393F8B232002B75
:1014400003D13B68002B40F041813B68002B14BF67
:1014500000230123DBB21A464DF6D403C2F2000387
:1014600083F8B2224DF6D403C2F2000393F8B232ED
:10147000002B02D04FF00203FB60FB79362B2FD1FB
:101480004DF6D403C2F2000393F8B132002B03D01F
:101490003B68002B00F01C814DF6D403C2F2000320
:1014A00093F8B132002B03D13B68002B40F012813E
:1014B0003B68002B14BF00230123DBB21A464DF614
:1014C000D403C2F2000383F8B1224DF6D403C2F272
:1014D000000393F8B132002B02D04FF00203FB60FF
:1014E000FB790C2B2FD14DF6D403C2F2000393F8F5
:1014F000B032002B03D03B68002B00F0ED804DF69E
:10150000D403C2F2000393F8B032002B03D13B683E
:10151000002B40F0E3803B68002B14BF0023012325
:10152000DBB21A464DF6D403C2F2000383F8B022B0
:101530004DF6D403C2F2000393F8B032002B02D070
:101540004FF00203FB60FB794A2B2FD14DF6D403F9
:10155000C2F2000393F8AF32002B03D03B68002B9C
:1015600000F0BE804DF6D403C2F2000393F8AF3210
:10157000002B03D13B68002B40F0B4803B68002B6C
:1015800014BF00230123DBB21A464DF6D403C2F286
:10159000000383F8AF224DF6D403C2F2000393F8A0
:1015A000AF32002B02D04FF00203FB60FB79092B16
:1015B0002FD14DF6D403C2F2000393F8B932002BB9
:1015C00003D03B68002B00F08F804DF6D403C2F2AD
:1015D000000393F8B932002B03D13B68002B40F095
:1015E00085803B68002B14BF00230123DBB21A4621
:1015F0004DF6D403C2F2000383F8B9224DF6D403AA
:10160000C2F2000393F8B932002B02D04FF002036C
:10161000FB60FB794D2B1CD14DF6D403C2F20003C5
:1016200093F8B8321A463B689A4261D03B68DAB206
:101630004DF6D403C2F2000383F8B8224DF6D4036A
:10164000C2F2000393F8B832002B02D14FF002032C
:10165000FB60FB79492B1AD14DF6D403C2F200038B
:10166000D3F8BC223B689A4244D04DF6D403C2F270
:1016700000033A68C3F8BC224DF6D403C2F200035B
:10168000D3F8BC32002B02D14FF00203FB60FB68A1
:10169000DBB2FA791A4811461A463B6841F299447E
:1016A000C0F60304A047FA794DF6D403C2F2000352
:1016B000C3F868224DF6D403C2F200033A68C3F8B7
:1016C0006C2218E000BF16E000BF14E000BF12E07B
:1016D00000BF10E000BF0EE000BF0CE000BF0AE05A
:1016E00000BF08E000BF06E000BF04E000BF02E06A
:1016F00000BF00E000BF07F11407BD4690BD00BF6A
:10170000E4D9002090B585B000AF03463960FB7185
:101710004DF6D403C2F20003D3F86822FB799A4253
:1017200009D14DF6D403C2F20003D3F86C223B6812
:101730009A4200F0F0804FF00103FB60FB79432BED
:1017400033D14DF6D403C2F2000393F8B332002B29
:1017500007D13B68002B00F0E0803B68632B00F072
:10176000DC803B68002B03DD3B68622B40F3D780B5
:101770003B68002B05DD3B68622B02DC4FF0010368
:1017800001E04FF00003DAB24DF6D403C2F20003D9
:1017900083F8B3224DF6D403C2F2000393F8B332B8
:1017A000002B02D04FF00203FB60FB79402B2FD1BE
:1017B0004DF6D403C2F2000393F8B432002B03D1E8
:1017C0003B68002B40F0AD804DF6D403C2F200031D
:1017D00093F8B432002B03D03B68002B00F0A380B9
:1017E0003B68002B14BF00230123DBB21A464DF6E1
:1017F000D403C2F2000383F8B4224DF6D403C2F23C
:10180000000393F8B432002B02D04FF00203FB60C8
:10181000FB793F2B1CD14DF6D403C2F2000393F8A1
:10182000B5321A463B689A427FD03B68DAB24DF631
:10183000D403C2F2000383F8B5224DF6D403C2F2FA
:10184000000393F8B532002B02D14FF00203FB6086
:10185000FB793D2B24D14DF6D403C2F2000393F85B
:10186000B6321A463B689A4261D03B68DAB24DF60E
:10187000D403C2F2000383F8B6224DF6D403C2F2B9
:10188000000393F8B632022B07D04DF6D403C2F210
:10189000000393F8B632052B02D14FF00203FB6030
:1018A000FB793B2B1CD14DF6D403C2F2000393F815
:1018B000B7321A463B689A423BD03B68DAB24DF6E3
:1018C000D403C2F2000383F8B7224DF6D403C2F268
:1018D000000393F8B732012B02D14FF00203FB60F3
:1018E000FB68DBB2FA79154811461A463B6841F2AB
:1018F0009944C0F60304A047FA794DF6D403C2F226
:101900000003C3F868224DF6D403C2F200033A681C
:10191000C3F86C220EE000BF0CE000BF0AE000BF7D
:1019200008E000BF06E000BF04E000BF02E000BF27
:1019300000E000BF07F11407BD4690BDE4D90020C8
:1019400090B583B000AF03463960FB714DF6D40308
:10195000C2F20003D3F86822FB799A4208D14DF60F
:10196000D403C2F20003D3F86C223B689A422ED013
:10197000FB79332B11D14DF6D403C2F2000393F857
:10198000AE321A463B689A4223D03B68DAB24DF633
:10199000D403C2F2000383F8AE22FB790F48194644
:1019A0004FF002023B6841F29944C0F60304A0479D
:1019B000FA794DF6D403C2F20003C3F868224DF65B
:1019C000D403C2F200033A68C3F86C2202E000BFFD
:1019D00000E000BF07F10C07BD4690BDE4D9002030
:1019E00090B587B002AFF8607A603B600B46FB723F
:1019F000FB7A3A6800920648F9681A467B6841F615
:101A00002504C0F60304A04707F11407BD4690BDA6
:101A1000ECD8002080B483B000AF78607B68002BE6
:101A200002DB7B68032B02DD4FF0000308E04DF67C
:101A3000D403C2F200037A689B1803F5A073DB7924
:101A4000184607F10C07BD4680BC704790B58BB0B7
:101A500002AFF860B9607A603B60F86847F289339A
:101A6000C0F603039847B86140F26933C0F6020339
:101A700098470346D3F8EE30FB61FA6940F2E7334A
:101A80009A4202DC4FF47A73FB61B869F96947F650
:101A9000BD33C0F60303984778617B69002B01D002
:101AA0007B6951E0FB68002B1BD140F6F433C2F296
:101AB00000031A68BB689A420DD040F26933C0F641
:101AC000020398470346D3F82E3018464AF29D0386
:101AD000C0F60503984740F6F433C2F20003BA6833
:101AE0001A60BB68DBB23A6B00927A6B0192B869FC
:101AF00019467A683B6847F2A174C0F60304A04710
:101B00004DF6D403C2F20003FA689B1803F5A073E4
:101B10004FF00102DA71B86947F60503C0F6030316
:101B2000984778614DF6D403C2F20003FA689B1817
:101B300003F5A0734FF00002DA71B86947F63D4330
:101B4000C0F6030398477B69184607F12407BD4692
:101B500090BD00BF80B588B000AFF860B9607A6012
:101B60003B60F86847F28933C0F603039847B861D1
:101B700040F26933C0F6020398470346D3F8EE30CB
:101B8000FB61FA6940F2E7339A4202DC4FF47A7360
:101B9000FB61B869F96947F6BD33C0F6030398479E
:101BA00078617B69002B01D07B6950E0FB68002BDA
:101BB0001FD1BB681B781A4640F6F433C2F200030B
:101BC0001B689A420DD040F26933C0F60203984771
:101BD0000346D3F82E3018464AF29D03C0F605039B
:101BE0009847BB681B781A4640F6F433C2F20003EC
:101BF0001A60B869B9687A6847F65903C0F60303F2
:101C000098474DF6D403C2F20003FA689B1803F517
:101C1000A0734FF00102DA71B8693968BA6A47F601
:101C2000E103C0F60303984778614DF6D403C2F28E
:101C30000003FA689B1803F5A0734FF00002DA71F5
:101C4000B86947F63D43C0F6030398477B691846D9
:101C500007F12007BD4680BD80B588B000AFF860B1
:101C6000B9607A6049F6DD53C0F602039847F8611F
:101C700022E049F6DD53C0F602039847B861BA691D
:101C8000FB69D21A13464FEA83039B184FEA4303BA
:101C90007B617A687B699A4202D24FF4627313E0E7
:101CA00047F60963C0F6020398474FF00A004AF26C
:101CB0009D03C0F605039847FB681B781A46BB686E
:101CC0009A42D6D14FF00003184607F12007BD46CF
:101CD00080BD00BF80B400AF4DF6D403C2F2000354
:101CE000B3F870321846BD4680BC704780B400AF70
:101CF0004DF6D403C2F20003B3F872321846BD4663
:101D000080BC704780B400AF4DF6D403C2F200032C
:101D1000B3F874321846BD4680BC704780B400AF3B
:101D20004DF6D403C2F20003B3F876321846BD462E
:101D300080BC704780B400AF4DF6D403C2F20003FC
:101D4000B3F878321846BD4680BC704780B400AF07
:101D50004DF6D403C2F20003B3F87A321846BD46FA
:101D600080BC704780B400AF4DF6D403C2F20003CC
:101D7000B3F8743203F101039AB24DF6D403C2F200
:101D80000003A3F87422BD4680BC704780B400AF46
:101D90004DF6D403C2F20003B3F8763203F1010327
:101DA0009AB24DF6D403C2F20003A3F87622BD46E0
:101DB00080BC704780B400AF4DF6D403C2F200037C
:101DC000B3F8783203F101039AB24DF6D403C2F2AC
:101DD0000003A3F87822BD4680BC704780B400AFF2
:101DE0004DF6D403C2F20003B3F87A3203F10103D3
:101DF0009AB24DF6D403C2F20003A3F87A22BD468C
:101E000080BC704780B483B000AF0346FB804DF6C2
:101E1000D403C2F20003FA88A3F8742207F10C0776
:101E2000BD4680BC704700BF80B483B000AF03469E
:101E3000FB804DF6D403C2F20003FA88A3F87622A1
:101E400007F10C07BD4680BC704700BF80B483B06B
:101E500000AF0346FB804DF6D403C2F20003FA88BC
:101E6000A3F8782207F10C07BD4680BC704700BF7D
:101E700080B483B000AF0346FB804DF6D403C2F2BA
:101E80000003FA88A3F87A2207F10C07BD4680BC4C
:101E9000704700BF80B400AF4DF6D403C2F2000318
:101EA000B3F8703203F101039AB24DF6D403C2F2D3
:101EB0000003A3F87022BD4680BC704780B400AF19
:101EC0004DF6D403C2F20003B3F8723203F10103FA
:101ED0009AB24DF6D403C2F20003A3F87222BD46B3
:101EE00080BC704780B483B000AF0346FB804DF6E2
:101EF000D403C2F20003FA88A3F8702207F10C079A
:101F0000BD4680BC704700BF80B483B000AF0346BD
:101F1000FB804DF6D403C2F20003FA88A3F87222C4
:101F200007F10C07BD4680BC704700BF80B582B08A
:101F300000AF40F26933C0F6020398470346B3F995
:101F400027309BB21AB213464FEA03139B1A4FEA8B
:101F5000830318464FF000014FF25533C0F60203D9
:101F6000984778600548796842F68D53C0F60503B6
:101F7000984707F10807BD4680BD00BF58DB002029
:101F800080B500AF044842F6C553C0F60503984734
:101F90000346184680BD00BF58DB002080B483B0E4
:101FA00000AF78604DF6D403C2F20003D3F890225C
:101FB0007B681A607B6803F104024DF6D403C2F219
:101FC0000003D3F8943213607B6803F108024DF6E6
:101FD000D403C2F20003D3F89832136007F10C0760
:101FE000BD4680BC704700BF80B483B000AF78604E
:101FF0007B68582B02D14FF0010315E07B68592B09
:1020000002D14FF001030FE07B685A2B02D14FF051
:10201000010309E07A684FF6FF739A4202D14FF04C
:10202000010301E04FF00003184607F10C07BD461D
:1020300080BC704780B483B000AF78604DF6CC02AE
:10204000C2F200024AF20853C0F6060393E8030006
:1020500082E803007B68002B0BD14DF6CC02C2F264
:1020600000024AF21053C0F6060393E8030082E828
:1020700003007B68012B0BD14DF6CC02C2F20002AB
:102080004AF21853C0F6060393E8030082E80300FF
:102090007B68022B0BD14DF6CC02C2F200024AF251
:1020A0002053C0F6060393E8030082E803004DF6D0
:1020B000CC03C2F20003184607F10C07BD4680BCF2
:1020C000704700BF80B5BEB000AF42F24163C0F6BA
:1020D00003039847C7F8F4006AE047F60963C0F6BF
:1020E00002039847D7F8F43003F1FF33C7F8F43010
:1020F00007F10403D7F8F400194642F61113C0F6AD
:10210000030398474FF00003C7F8E4304FF0000393
:10211000C7F8F03034E0D7F8F0004FF27143C0F662
:1021200001039847C7F8DC004FF00003C7F8EC3014
:1021300018E0D7F8DC30D7F8EC2002F1980233F839
:1021400012309BB21A46BB881BB29A4204D14FF0A0
:102150000103C7F8E43009E0D7F8EC3003F10103DC
:10216000C7F8EC30D7F8EC30062BE2DDD7F8E430D6
:10217000002B10D1D7F8F03003F10103C7F8F0308D
:102180004EF6DD73C0F6010398470246D7F8F030EB
:102190009A42C0DC00E000BFD7F8E430002B07D142
:1021A000BB881BB2184642F2A173C0F603039847DE
:1021B000D7F8F430002B90DC42F6F513C0F6030399
:1021C0009847C7F8F40051E047F60963C0F60203E8
:1021D0009847D7F8F43003F1FF33C7F8F43007F12C
:1021E0000403D7F8F400194642F67163C0F60303FE
:1021F00098474FF00003C7F8E4304FF00003C7F8EA
:10220000F0301DE0D7F8F0004FF27143C0F6010343
:102210009847C7F8D800D7F8D830B3F900309BB248
:102220001AB2D7F806309A4204D14FF00103C7F82A
:10223000E4300FE0D7F8F03003F10103C7F8F030D5
:102240004EF6DD73C0F6010398470246D7F8F0302A
:102250009A42D7DCD7F8E430002B07D1BB881BB2F9
:10226000184642F63143C0F603039847D7F8F430D6
:10227000002BA9DC42F6F513C0F603039847C7F814
:10228000F4004FF00003C7F8F03010E147F609639F
:10229000C0F602039847D7F8F0004FF27143C0F63A
:1022A00001039847C7F8D4004FF00003C7F8E030A7
:1022B0004FF00003C7F8EC30E3E0D7F8D430D7F89C
:1022C000EC2002F1980233F812309AB24FF6FF7305
:1022D0009A424CD04FF00003C7F8E4304FF00003AF
:1022E000C7F8F43021E007F10403D7F8F4001946E9
:1022F00042F61113C0F603039847BB881AB2D7F809
:10230000D430D7F8EC1001F1980133F811309BB2BA
:102310009A4204D14FF00103C7F8E4300FE0D7F838
:10232000F43003F10103C7F8F43042F24163C0F620
:10233000030398470246D7F8F4309A42D3DCD7F823
:10234000E430002B13D1D7F8D420D7F8EC3003F1C8
:1023500098034FF0FF3102F813104FEA4303D318EC
:102360004FF0FF325A704FF00103C7F8E0304FF0E2
:102370000003C7F8E8307AE0D7F8D410D7F8EC209B
:1023800013464FEA83039B18D7F8E8209B1803F104
:1023900074034FEA4303CB185B889AB24FF6FF737E
:1023A0009A425ED04FF00003C7F8E4304FF00003CC
:1023B000C7F8F4302AE007F10403D7F8F40019460F
:1023C00042F2D523C0F603039847BB8819B2D7F869
:1023D000D400D7F8EC2013464FEA83039B18D7F8B4
:1023E000E8209B1803F174034FEA4303C3185B888A
:1023F0009BB2994204D14FF00103C7F8E4300FE0DB
:10240000D7F8F43003F10103C7F8F43041F6F5735F
:10241000C0F6030398470246D7F8F4309A42CADC64
:10242000D7F8E430002B1CD1D7F8D420D7F8EC1023
:102430000B464FEA83035B18D7F8E8105B1803F1EB
:1024400074014FEA4103D3184FF0FF3098704FEA00
:102450004103D3184FF0FF32DA704FF00103C7F891
:10246000E030D7F8E83003F10103C7F8E830D7F8D7
:10247000E830042B80DDD7F8EC3003F10103C7F816
:10248000EC30D7F8EC30062B7FF717AFD7F8E030F9
:10249000002B06D0D7F8F0004EF65103C0F601032A
:1024A0009847D7F8F03003F10103C7F8F0304EF643
:1024B000DD73C0F6010398470246D7F8F0309A4220
:1024C0003FF7E4AE4FF4803040F25553C0F60203BC
:1024D0009847C7F8D00007F1F807BD4680BD00BF98
:1024E00080B582B000AF78607A6840F203339A42D8
:1024F00010D14EF23043C2F2000303F51D5303F135
:102500001C034FF007021A6049F68D33C0F6020330
:1025100098479CE07B68B3F5407F1AD149F6BD33FC
:10252000C0F60203984749F61D43C0F602039847D8
:1025300049F67D43C0F6020398474EF23043C2F29B
:10254000000303F51D5303F11C034FF000021A6052
:102550007DE07A6845F6F7239A4211D14DF6B40032
:10256000C2F200004FF00A0142F68D53C0F6050397
:10257000984740F6F833C2F200034FF000021A60A9
:102580007A6844F6A1439A421FD140F6F833C2F26A
:1025900000031B68002B57D14DF6B400C2F20000B7
:1025A00042F6C553C0F6050398470346002B07D0F3
:1025B00040F6F833C2F200034FF001021A6046E021
:1025C00042F25963C0F6020398477A6845F6F82349
:1025D0009A4211D14DF6C000C2F200004FF00A013C
:1025E00042F68D53C0F60503984740F6FC33C2F21D
:1025F00000034FF000021A607A6844F6A2439A4240
:1026000025D140F6FC33C2F200031B68002B1DD11C
:102610004DF6C000C2F2000042F6C553C0F60503F5
:1026200098470346002B07D040F6FC33C2F2000364
:102630004FF001021A600AE04FF000004CF21973EB
:10264000C0F60403984702E000BF00E000BF07F1B6
:102650000807BD4680BD00BF80B400AF4DF6D4036F
:10266000C2F200034FF0010283F8C122BD4680BCD4
:10267000704700BF80B400AF4DF6D403C2F2000330
:1026800093F8C1321846BD4680BC704780B400AF95
:1026900040F6A863C2F200034FF001021A60BD4683
:1026A00080BC704780B400AF40F6A863C2F200035C
:1026B0001B681846BD4680BC704700BF0000000084
:1026C00090B5ADB004AF4FF00003C7F898304EF2AC
:1026D000A103C0F601039847C7F89400D7F89430D7
:1026E000002B40F3488240F60043C2F200031B680F
:1026F00003F1010240F60043C2F200031A6040F603
:102700000043C2F200031A68D7F894309A4206DBFD
:1027100040F60043C2F200034FF000021A6040F698
:102720000043C2F200031A6807F118031046194665
:102730004EF25553C0F601039847C7F89800D7F8F2
:102740009830002B40F0178207F1180318464EF21C
:102750000563C0F60103984797F83A30002B00F064
:102760000A8297F83B30022B40F08C8007F1180367
:10277000184642F68933C0F6020398470346002BF9
:1027800000F0F98107F11003184642F2E913C0F690
:102790000503984707F1100207F1180303F15C03E2
:1027A0001046194642F2E143C0F605039847C7F8C0
:1027B0009000B7F8742040F2CF739A4213D9BB8FC0
:1027C0001AB213464FEA03139B1A4FEA83031A46C1
:1027D000B7F941309BB21BB2D31803F10102D7F80D
:1027E00090309A421FDA07F11803184642F65D430B
:1027F000C0F60203984707F1180303F15C0318467B
:1028000042F2E913C0F60503984740F60043C2F2CE
:1028100000031A6807F11803104619464EF21533E3
:10282000C0F60103984707F1180303F15003184657
:1028300042F6C553C0F6050398470346002B00F047
:102840009A8107F1180303F15C03184642F2E91379
:10285000C0F60503984707F11803184642F65D4392
:10286000C0F60203984740F60043C2F200031A681C
:1028700007F11803104619464EF21533C0F601034E
:10288000984727E197F83B30012B40F02381FB8FDD
:102890001BB218464FF20D43C0F601039847C7F824
:1028A0008C00D7F88C30002B00F065814FF00003CE
:1028B000C7F89C3097F84030012B09D1D7F88C30FD
:1028C00093F87331062B03D14FF00103C7F89C3006
:1028D00097F84030022B09D1D7F88C3093F8733138
:1028E000072B03D14FF00103C7F89C3097F8403015
:1028F000032B09D1D7F88C3093F87331052B03D112
:102900004FF00103C7F89C3097F84030042B09D1F1
:10291000D7F88C3093F87331042B03D14FF00103B7
:10292000C7F89C3097F84030052B09D1D7F88C3088
:1029300093F87331032B03D14FF00103C7F89C3098
:1029400097F84030062B09D1D7F88C3093F87331C3
:10295000022B03D14FF00103C7F89C3097F84030A9
:10296000072B09D1D7F88C3093F87331012B03D1A1
:102970004FF00103C7F89C30D7F89C30002B00F0D3
:10298000FA8097F87B30002B30D0FA6F4DF6451364
:10299000C0F60103104698470146D7F88C30D3F8AB
:1029A000662113461A464DF2D973C0F60103084654
:1029B00011469847034623F00043C7F888304DF28C
:1029C000C503C0F60103D7F88800984702460B46B6
:1029D0004DF28D64C0F601041046194668A3D3E990
:1029E0000023A0470346002B40F0C58007F11803E1
:1029F000184642F68933C0F6020398470346002B77
:102A000000F0B980B7F941309BB21BB2002B61DDF9
:102A1000B7F861309AB240F2CF739A4218D807F1F2
:102A2000180303F14903184642F2E913C0F60503FF
:102A3000984740F60043C2F200031A6807F11803F2
:102A4000104619464EF21533C0F60103984792E03E
:102A500007F10803184642F2E913C0F60503984748
:102A600007F1080207F1180303F14903104619465C
:102A700042F2E143C0F605039847C7F88400B7F96E
:102A800041309BB21AB2D7F884309A4273DCB7F85F
:102A900061309AB240F2CF739A421BD907F1180302
:102AA00003F1490318464FF000014FF0070246F2C8
:102AB0000903C0F60103984740F60043C2F2000341
:102AC0001A6807F11803104619464EF21533C0F67E
:102AD0000103984797F8434040F26933C0F6020378
:102AE0009847034693F820309C4231D04FF00103C1
:102AF000C7F8803097F84330786C07F104013A4604
:102B00000090D7F88000019007F1180000F1300024
:102B100002904DF6A830C2F2000046F21964C0F6E9
:102B20000304A0477B683A4600924FF000004DF640
:102B3000A831C2F200011A464DF6B833C2F20003C2
:102B400041F65534C0F60204A047C7F8980012E0D9
:102B50007B6C1A46BB6C002B02D04FF47F4301E024
:102B60004FF000031046194646F23903C0F603033E
:102B70009847C7F8980007F1A407BD4690BD00BF6D
:102B80002D431CEBE2361A3F80B588B000AF786069
:102B900007F10C03184642F2E913C0F60503984703
:102BA0004FF00003BB814FF00003BB734FF00003F5
:102BB000FB7307F10C03184642F22143C0F60503EC
:102BC0009847F8617B684FF0000283F83B204FF094
:102BD000000283F83C207B684FF0000283F83D2020
:102BE0007B684FF0000283F83E207B6803F13B03D3
:102BF000184642F22143C0F605039847B8617B6846
:102C00004FF0000283F842204FF0000283F8432087
:102C10007B684FF0000283F844207B684FF000028D
:102C200083F845207B6803F14203184642F22143B2
:102C3000C0F6050398477861FA69BB699A4203DBDD
:102C4000FA697B699A4202DD4FF0000301E04FF020
:102C50000103184607F12007BD4680BD80B588B046
:102C600000AF78604FF00003BB617B6893F82330BE
:102C7000022B58D107F10803184642F2E913C0F6B7
:102C8000050398473B7B4FF4616202FB03F17B7BBA
:102C90001A4613464FEA03139B1A4FEA8303CA18D6
:102CA000BB7BD3187B617B6893F838304FF461624B
:102CB00002FB03F17B6893F839301A4613464FEA5A
:102CC00003139B1A4FEA8303CA187B6893F83A30C0
:102CD000D3183B617B68B3F929309BB21AB23B69C8
:102CE000D318FB610DE07B68B3F924309BB21AB2B4
:102CF00013464FEA03139B1A4FEA8303FA69D3186A
:102D0000FB61FA697B699A42EDDDFA697B69D31A46
:102D1000BB617B6803F150031846B96942F68D53D5
:102D2000C0F60503984707F12007BD4680BD00BFE8
:102D300090B591B002AFF860B9601346FB71F868C6
:102D40004FF47A7147F6BD33C0F603039847B86273
:102D5000BB6A002B01D0BB6AC1E0FB684FF00002E8
:102D60001A61FB681968FB681B691A468A18F979A9
:102D7000117003F10102FB681A6149F6DD53C0F6D8
:102D80000203984778624FF008037B634FF000031B
:102D90003B635CE049F6DD53C0F6020398473862B6
:102DA0003A6A7B6AD21A13464FEA83039B184FEAAA
:102DB0004303FB61FB69B3F57A7F00F288804FF033
:102DC0000003FB75BB689B6C07F1170210464FF0C0
:102DD00001014FF000029847B862BB6A002B07D090
:102DE0004FF00A004AF29D03C0F6050398472EE013
:102DF000FB681968FB681B691A468A18F97D11700F
:102E000003F10102FB681A61FB681A697B6B9A4245
:102E10001DD1FB681B6803F101031B78A3F10F03AD
:102E2000012B03D94FF001033B6310E0FB681B69E2
:102E3000082B08D1FB681B6803F106031B7803F11C
:102E400009037B6302E04FF001033B6300BF3B6B70
:102E5000002B9FD04FF00003FB6203E0FB6A03F1FD
:102E60000103FB62FB681A69FB6A9A42F6DCFB68A5
:102E70001968FB681A69FB681B6807F11800009065
:102E80004FF0000041F65534C0F60204A047B86286
:102E9000BB6A002B1AD14FF00003FB6203E0FB6A10
:102EA00003F10103FB62BB69FA6A9A42F7DBBB6874
:102EB000DB699847BB689B699847BB68DB6CFA681D
:102EC0001168BA6908461146984700E000BFF868E3
:102ED00047F63D43C0F6030398474FF000031846FA
:102EE00007F13C07BD4690BD90B595B002AFF860C4
:102EF000B9607A6040F6AC63C2F200031B6803F16C
:102F0000010240F6AC63C2F200031A60FB684FF0A6
:102F10000002C3F840244FF000037B6411E0FB681B
:102F2000D3F840347A6C79688A181178FA68D154E9
:102F300003F10102FB68C3F840247B6C03F1010339
:102F40007B647B6C062BEADD49F6DD53C0F6020399
:102F5000984778634FF00C03FB634FF00003BB63AB
:102F600068E049F6DD53C0F60203984738633A6BD0
:102F70007B6BD21A13464FEA83039B184FEA430335
:102F8000FB62FA6A43F698239A4200F251814FF0AD
:102F90000003FB75BB689B6C07F1170210464FF0EE
:102FA00001014FF000029847B862BB6A002B07D0BE
:102FB0004FF00A004AF29D03C0F60503984739E036
:102FC000FB68D3F84034F97DFA68D15403F101026B
:102FD000FB68C3F84024FB68D3F84024FB6B9A429B
:102FE00028D1FB68DB79A3F10F03012B03D94FF044
:102FF0000103BB631EE0FB68D3F840340C2B15D1F2
:103000004FF000037B62FB681B794FEA03237A6A67
:1030100013437B62FB685B797A6A13437B627B6A4A
:1030200003F106037B627B6AFB6302E04FF001035E
:10303000BB6300BFBB6B002B93D04FF000033B641E
:1030400003E03B6C03F101033B64FB68D3F84024CD
:103050003B6C9A42F5DCFB681B7887F82330FB68F1
:103060005B7887F822304FF000033B644FF0060393
:103070007B640FE0FA687B6CD3181A78F9683B6CB4
:10308000CB181A707B6C03F101037B643B6C03F17A
:1030900001033B64FB68D3F840247B6C9A42E9DC73
:1030A000FB68D3F84034A3F10402FB68C3F8402462
:1030B000FA68FB68D3F84034A3F1020310461946BE
:1030C00045F23913C0F603039847F861FB68D3F85B
:1030D000403403F1FF33FA694FEA1222D1B2FA68A1
:1030E000D154FB68D3F84034A3F10203FA69D1B29A
:1030F000FA68D1544FF000033B6403E03B6C03F1EA
:1031000001033B64FB68D3F840243B6C9A42F5DC36
:10311000F968FB68D3F84024FB6807F118000090B9
:103120004FF0000041F65534C0F60204A047B862E3
:10313000BB6A002B04D0BA6A40F20E739A4276D171
:103140004FF000033B6403E03B6C03F101033B647D
:10315000BB693A6C9A42F7DBBB6903F105033B6438
:10316000BB6903F1FF337B640FE0FA687B6CD31813
:103170001A78F9683B6CCB181A707B6C03F1FF333B
:103180007B643B6C03F1FF333B647B6C002BECDA1C
:103190004FF000037B6409E0FA683B6CD3184FF0F2
:1031A00000021A707B6C03F101037B647B6C052BBE
:1031B000F2DDFB6897F823201A70FB6897F822204D
:1031C0005A70FB684FF000029A70FB684FF00002E3
:1031D000DA70BB69A3F10203BB61BB6903F47F43EF
:1031E0004FEA2323DAB2FB681A71BB69DAB2FB68D3
:1031F0005A71BB6903F10603BB614FF000033B64E6
:1032000003E03B6C03F101033B64BB693A6C9A42F7
:10321000F7DBBB68DB699847BB689B699847BB686D
:10322000DB6CF968BA6908461146984700E000BFB0
:103230004FF00003184607F14C07BD4690BD00BF94
:1032400080B500AF044841F6B553C0F60303984774
:103250000346184680BD00BFECD8002080B590B072
:1032600000AF41F2F573C0F603039847F863FB6BB8
:10327000002B01DDFB6B96E043F24123C0F6020315
:10328000984778634FF00003BB633CE0484841F641
:10329000D153C0F60303984738633B6B002B07D02C
:1032A0004FF00A004AF29D03C0F60503984726E056
:1032B0003B463F48B96B1A4641F63953C0F6030303
:1032C000984738633A4841F63163C0F6030398479C
:1032D0003A6B40F286339A4219D0D7F80B30184631
:1032E0004FF20D43C0F601039847F862FB6A002BCA
:1032F00004D0FB6B03F10103FB6300E000BFBB6B79
:1033000003F10103BB63BA6B7B6B9A42BEDBFB6BC1
:10331000002B02D14FF0000345E007F120031846CF
:1033200042F2E913C0F60503984707F12003184657
:10333000204942F2E143C0F605039847B86240F2E3
:103340006933C0F6020398470346D3F82120134699
:103350004FEA03139B1A4FEA83031A46BB6A9A4249
:1033600001DAFB6B1FE007F120031846124942F215
:10337000E143C0F605039847B86240F26933C0F6EE
:10338000020398470346D3F8212013464FEA03135C
:103390009B1A4FEA83031A46BB6A9A4201DAFB6B17
:1033A00001E04FF00003184607F14007BD4680BD1D
:1033B000ECD8002074DB00207BDB002080B58AB0D5
:1033C00000AF41F60D03C0F60303984743F295435F
:1033D000C0F602039847386243F2D163C0F6020395
:1033E000984738624FF0010044F63923C0F60203D3
:1033F00098473862264841F6D153C0F603039847F0
:103400004FF000037B623B462148796A1A4641F639
:103410003953C0F60303984738623A6A40F2893359
:103420009A4228D07B7F002B02D03B7F002B04D117
:103430007B6A03F101037B62E5E7FB7E002B07D08B
:103440007B7E002B04D17B6A03F101037B62DAE708
:10345000BB7E002B07D03B7E002B04D17B6A03F19F
:1034600001037B62CFE70A48796A41F6E923C0F697
:1034700003039847C7E7064841F63163C0F60303E4
:1034800098474FF00003184607F12807BD4680BD56
:10349000ECD8002090B5C5B000AF42F6B913C0F625
:1034A00003039847C7F80001D7F8000142F291439F
:1034B000C0F60303984743F24123C0F6020398473E
:1034C000C7F8FC004FF00003C7F80C31EDE07E4870
:1034D00041F6D153C0F603039847C7F8F800D7F870
:1034E000F830002B07D04FF032004AF29D03C0F6AF
:1034F00005039847D3E007F1CC037348D7F80C11C4
:103500001A4641F63953C0F603039847C7F8F80046
:103510006D4841F63163C0F603039847D7F8F820A9
:1035200040F286339A4200F0C7806748D7F80C1102
:103530004FF0000241F6D933C0F60303984797F8DD
:10354000E430002B40F0A880D7F8D73018464FF26F
:103550000D43C0F601039847C7F8F400D7F8F430DC
:10356000002B00F09B8097F8E33003F1FF32D7F88F
:10357000F43002F1980233F812309BB2C7F8F03001
:1035800007F1CC03D7F8F000D7F80011D7F8F420F2
:1035900044F23514C0F60204A0474FF00003C7F808
:1035A000083174E097F8E33003F1FF32D7F8F410F4
:1035B00013464FEA83039B18D7F808219B1803F1A1
:1035C00074034FEA4303CB185B889BB2C7F8EC3017
:1035D000D7F8EC30002B62DDD7F8EC309BB21AB292
:1035E0003B461046194642F26923C0F6030398474A
:1035F000C7F8F800D7F8F830002B42D14FF000039D
:10360000C7F8043139E03B461846D7F8041143F6B1
:103610003D13C0F602039847C7F8F800D7F8F83012
:10362000002B23D12848D7F80C114FF0000241F6A7
:103630005D43C0F60303984743F64123C0F60203F7
:103640009847C7F8F800D7F8F830002B07D11E4884
:10365000D7F80C1141F68133C0F6030398471B4895
:1036600042F2E913C0F60503984700E000BFD7F81F
:10367000043103F10103C7F80431D7F80431012BF9
:10368000C1DDD7F8083103F10103C7F80831D7F8D5
:103690000831042B86DD02E000BF00E000BFD7F850
:1036A0000C3103F10103C7F80C31D7F80C21D7F81E
:1036B000FC309A42FFF60BAF4FF00003184607F5B7
:1036C0008A77BD4690BD00BFECD8002074DB002097
:1036D00090B5C5B000AF42F6B913C0F603039847E2
:1036E000C7F80001D7F8000142F29143C0F6030386
:1036F000984743F24123C0F602039847C7F8FC00FD
:103700004FF00003C7F80C3105E18A4841F6D15368
:10371000C0F603039847C7F8F800D7F8F830002B35
:1037200007D04FF032004AF29D03C0F605039847D8
:10373000EBE007F1CC037F48D7F80C111A4641F6AD
:103740003953C0F603039847C7F8F800794841F6A3
:103750003163C0F603039847D7F8F82040F2863368
:103760009A4200F0DF807348D7F80C114FF0010245
:1037700041F6D933C0F60303984797F8E530002B9C
:1037800040F0C080D7F8D73018464FF20D43C0F64E
:1037900001039847C7F8F400D7F8F430002B00F085
:1037A000B38097F8E33003F1FF32D7F8F43002F139
:1037B000980233F812309BB2C7F8F03007F1CC030F
:1037C000D7F8F000D7F80011D7F8F42044F23514F8
:1037D000C0F60204A04707F1CC03D7F8F40019465D
:1037E00044F2ED03C0F60203984743F60133C0F6F6
:1037F000020398474FF00003C7F8083151E097F8EB
:10380000E33003F1FF32D7F8F41013464FEA830395
:103810009B18D7F808219B1803F174034FEA430360
:10382000CB185B889BB2C7F8EC30D7F8EC30002B94
:103830003BDDD7F8EC309BB21AB23B461046194636
:1038400042F26923C0F603039847C7F8F800D7F897
:10385000F830002B1FD13B46184643F67943C0F69B
:10386000020398474FF00003C7F804310FE03148D6
:10387000D7F80C114FF0010241F65D43C0F6030387
:103880009847D7F8043103F10103C7F80431D7F89A
:103890000431012BEBDDD7F8083103F10103C7F840
:1038A0000831D7F80831042BA9DD43F6DD43C0F613
:1038B00002039847C7F8F800D7F8F830002B09D072
:1038C0004FF02A00D7F8F81041F29133C0F6020306
:1038D000984710E04FF02B00D7F8F81041F29133E1
:1038E000C0F6020398471348D7F80C1141F6E1439C
:1038F000C0F603039847104842F2E913C0F60503E7
:10390000984702E000BF00E000BFD7F80C3103F198
:103910000103C7F80C31D7F80C21D7F8FC309A42D4
:10392000FFF6F3AE4FF00003184607F58A77BD4661
:1039300090BD00BFECD800207BDB002080B58AB0B2
:1039400000AF7860396007F10803786839681A4673
:1039500042F26933C0F603039847F861FB69002B14
:1039600001D0FB6964E007F108031B78002B02D14A
:1039700040F28A335CE04FF000037B624FF00003BB
:103980003B622E484FF000014FF0140246F209034B
:10399000C0F6010398474DF6D403C2F200033A6A19
:1039A0009B1803F50A734FF02B029A703B6A03F1E0
:1039B00001033B6228E007F108027B6AD3181B78F9
:1039C0002F2B06D907F108027B6AD3181B78392BF5
:1039D00004D97B6A03F101037B6215E007F1080259
:1039E0007B6AD3181A784DF6D403C2F20003396A01
:1039F0005B1803F50A739A703B6A03F101033B629B
:103A00007B6A03F101037B6207F108027B6AD3182A
:103A10001B78002B02D03B6A132BCCDD4DF6D40370
:103A2000C2F200034FF0000283F83D224FF0000382
:103A3000184607F12807BD4680BD00BFFEDA00200A
:103A400080B584B000AF48F26143C0F602039847E6
:103A500078607B68002B02D140F6990346E04FF076
:103A60000003FB604FF00503BB600FE07B685B6DFC
:103A7000214822499847F860FB68002B13D04FF487
:103A8000FA604AF29D03C0F605039847BB686FEAE7
:103A900003034FEAD373DBB2BA6802F1FF32BA60B4
:103AA000002BE3D100E000BFFB68002B09D14FF0F1
:103AB00025004FF0000141F64113C0F6020398477C
:103AC00013E04FF02400F96841F2DD33C0F6020341
:103AD00098477B689B6D984738604FF0490039687C
:103AE00041F2DD33C0F602039847FB68184607F140
:103AF0001007BD4680BD00BFFEDA00201EDA0020A0
:103B000080B582B000AF4DF6C830C2F2000044F27A
:103B10005501C0F6020144F29D02C0F602024FF2C6
:103B20007123C0F6040398473B46184642F2E91356
:103B3000C0F6050398473B881A464DF6C833C2F2D3
:103B40000003C3F84C27BB781A464DF6C833C2F2BF
:103B50000003C3F85027FB781A464DF6C833C2F26B
:103B60000003C3F854273B791A464DF6C833C2F216
:103B70000003C3F858277B791A464DF6C833C2F2C2
:103B80000003C3F85C27BB791A464DF6C833C2F26E
:103B90000003C3F860274DF6C833C2F200034AF2AF
:103BA0002852C0F6060207CA03C31A802D4B4AF2F8
:103BB0002852C0F6060207CA03C31A804AF23453D9
:103BC000C0F606031A784DF6C833C2F2000383F834
:103BD00080204DF6C833C2F200034FF0030283F891
:103BE000C02040F26933C0F602039847034603F24F
:103BF00022431D48194646F20553C0F60103984773
:103C000040F26933C0F60203984703461748194645
:103C100046F20553C0F60103984740F26933C0F6F7
:103C200002039847034603F222331148194646F22D
:103C30000553C0F60103984740F26933C0F602030A
:103C40009847034603F2A2330A48194646F2055341
:103C5000C0F6010398474FF00003184607F1080724
:103C6000BD4680BD08DC002089DC0020C9DC0020C6
:103C70008CE20020CCE2002080B582B000AF7860FA
:103C80007B6803F166031B78002B0CD07B6803F183
:103C900066034DF6C830C2F2000019464FF2AD235C
:103CA000C0F6040398477B6803F18E031B78002B52
:103CB0000CD07B6803F18E034DF6C830C2F20000D1
:103CC00019464FF2AD23C0F6040398474FF00003A6
:103CD000184607F10807BD4680BD00BF80B5BEB0DD
:103CE00000AF40F24163C0F6020398470346002B41
:103CF00002D140F2E553A1E148F26143C0F602036C
:103D00009847C7F8D800D7F8D830002B02D140F632
:103D1000990393E14FF00003C7F8F4304FF000032C
:103D2000C7F8F0301AE0D7F8F03003F105034FEA96
:103D300083124DF6C833C2F20003D31803F1010316
:103D40001B78002B04D04FF00103C7F8F43009E0D2
:103D5000D7F8F03003F10103C7F8F030D7F8F030AE
:103D6000092BE0DDD7F8F430002B02D14FF000032F
:103D700064E107F18C0318464FF000014FF0400258
:103D800046F20903C0F60103984707F18C03184671
:103D9000AD494FF03F0246F22163C0F60103984758
:103DA00007F18C03184646F2C153C0F60103984749
:103DB0000346C7F8D4304FF00003C7F8EC3025E0D5
:103DC00007F18C02D7F8EC30D3181B780D2B07D1F4
:103DD00007F18C02D7F8EC30D3184FF020021A709C
:103DE00007F18C02D7F8EC30D3181B780A2B07D1D7
:103DF00007F18C02D7F8EC30D3184FF020021A707C
:103E0000D7F8EC3003F10103C7F8EC30D7F8EC2019
:103E1000D7F8D4309A42D3DB07F18C038B4819468C
:103E200046F20553C0F6010398478948864946F291
:103E3000DD13C0F601039847854846F2C153C0F62A
:103E400001039847034603F581624DF6C833C2F279
:103E50000003D2184AF23853C0F6060311461A4638
:103E60004FF06D03084611461A4645F67573C0F6C5
:103E7000010398474FF00003C7F8F03005E0D7F88A
:103E8000F03003F10103C7F8F030D7F8F030092B18
:103E9000F5DD4FF00003C7F88830D7F8D8309B6ABB
:103EA00007F188024FF007001146984740F2693346
:103EB000C0F602039847034603F29E2307F104026B
:103EC0001046194646F20553C0F60103984740F2E2
:103ED0006933C0F6020398470346D3F81E33C7F888
:103EE00084304FF00003C7F8E8304FF00003C7F804
:103EF000E4304FF00003C7F8E0304FF00303C7F899
:103F0000DC305AE0D7F8E830002B19D1D7F88830E8
:103F1000042B15D0D7F8D8301B699847C7F8E000B4
:103F2000D7F8E030002B07D04FF4FA604AF29D0337
:103F3000C0F60503984740E04FF00103C7F8E830AA
:103F4000D7F8E430002B18D1D7F8D830DB6B07F165
:103F5000040210469847C7F8E000D7F8E030002B7D
:103F600007D04FF4FA604AF29D03C0F60503984764
:103F700023E04FF00103C7F8E4304DF6C830C2F239
:103F800000004FF67153C0F604039847C7F8E000ED
:103F9000D7F8E030002B20D04FF04D00D7F8E010DC
:103FA00041F2DD33C0F6020398474FF4FA604AF25B
:103FB0009D03C0F6050398470FE0D7F8DC30002BCF
:103FC000D4BF00230123DBB2D7F8DC2002F1FF329B
:103FD000C7F8DC20002B95D100E000BFD7F8E43013
:103FE000002B13D0D7F8E02040F69F039A420DD063
:103FF000D7F8D8301B6C9847C7F8D000D7F8D03026
:10400000002B03D0D7F8D030C7F8E030D7F8E8302D
:10401000002B11D0D7F88830042B0DD0D7F8D8302A
:104020005B699847C7F8CC00D7F8CC30002B03D099
:10403000D7F8CC30C7F8E030D7F8E030184607F1B1
:10404000F807BD4680BD00BF1EDA002090DF0020CB
:10405000D0DF002080B584B000AF7860396048F2CE
:104060006143C0F602039847F860FB68002B02D159
:1040700040F28B330CE0FB68DB6C7868396898475A
:10408000B860BB68002B01D0BB6801E04FF00003B3
:10409000184607F11007BD4680BD00BF80B586B049
:1040A00000AF786043F698237B6148F26143C0F625
:1040B0000203984738613B69002B02D140F28B33F1
:1040C0000EE03B699B6C78684FF001017A69984774
:1040D000F860FB68002B01D0FB6801E04FF00003A3
:1040E000184607F11807BD4680BD00BF90B585B0E2
:1040F00002AF7860396040F26933C0F60203984736
:10410000034603F2A2433A6800924FF00102019283
:1041100007484FF040011A467B6844F2B114C0F6DC
:104120000204A0470346184607F10C07BD4690BDA0
:10413000BEDA002090B589B002AFF860B9607A604D
:104140003B60BB68B3F900309BB21AB2FB689A427D
:1041500013D0FB689BB21BB21846B96842F6A503A0
:10416000C0F60303984778617B69002B05D0B868D7
:1041700042F29143C0F603039847BB6803F1020380
:104180003A6800924FF00002019208484FF0A001F7
:104190001A467B6844F2B114C0F60204A0470346F5
:1041A000184607F11C07BD4690BD00BF1EDA00206F
:1041B000B0B5CEB004AF07F10C04206007F10800E1
:1041C000016007F104010A603A46136007F1080331
:1041D0001B6807F10C0210684FF000011A4646F206
:1041E0000903C0F6010398474FF00003C7F82431D4
:1041F0004FF00003C7F8203100F001BCD7F824319C
:1042000007F104021268D3181B787B2B1AD0D7F859
:10421000203107F10C021268D318D7F8242107F1D6
:10422000040109688A1812781A70D7F8203103F14E
:104230000103C7F82031D7F8243103F10103C7F88F
:104240002431DCE3D7F8243103F10103C7F824312A
:1042500007F1E40318464FF000014FF0080246F260
:104260000903C0F6010398474FF00003C7F81C315B
:1042700018E0D7F8243107F104021268D3181A782D
:1042800007F1E401D7F81C31CB181A70D7F81C31AC
:1042900003F10103C7F81C31D7F8243103F10103FE
:1042A000C7F82431D7F8243107F104021268D31873
:1042B0001B78002B0CD0D7F81C31072B08DCD7F863
:1042C000243107F104021268D3181B787D2BD0D15A
:1042D000D7F8243103F10103C7F824314FF000036C
:1042E00087F8EB3007F1E40318464AF2A851C0F60C
:1042F000060146F22933C0F6010398470346002B16
:1043000036D14FF00003C7F818311CE0D7F8203140
:1043100007F10C021268D2184DF6D403C2F2000362
:10432000D7F818115B1803F5A4739B781370D7F8AE
:10433000203103F10103C7F82031D7F8183103F118
:104340000103C7F818314DF6D403C2F20003D7F8C1
:1043500018219B1803F5A4739B78002B00F04F8362
:1043600007F10803D7F820211B689A42CEDB46E309
:1043700007F1E40318464AF2AC51C0F6060146F2D2
:104380002933C0F6010398470346002B64D107F197
:10439000DC03184642F2E913C0F6050398474DF6D0
:1043A000C833C2F200034FF0000283F8642797F885
:1043B000DE301A4697F8DF30B7F8DC100D4697F874
:1043C000E0100C4697F8E110084697F8E2100095C7
:1043D000019402900391A3484AF2B051C0F606013D
:1043E00043F64924C0F60504A0474FF00003C7F880
:1043F00014311CE0D7F8203107F10C021268D218F2
:104400004DF6C833C2F20003D7F814115B1803F558
:10441000EC631B791370D7F8203103F10103C7F85F
:104420002031D7F8143103F10103C7F814314DF6E8
:10443000C833C2F20003D7F814219B1803F5EC63CC
:104440001B79002B00F0DB8207F10803D7F820214D
:104450001B689A42CEDBD2E207F1E40318464AF227
:10446000D451C0F6060146F22933C0F6010398473D
:104470000346002B32D14FF00003C7F810311AE089
:10448000D7F8203107F10C021268D3183A461168A8
:10449000D7F810218A1802F1050212781A70D7F89D
:1044A000203103F10103C7F82031D7F8103103F1AF
:1044B0000103C7F810313B461A68D7F81031D318FA
:1044C00003F105031B78002B00F0998207F1080324
:1044D000D7F820211B689A42D2DB90E207F1E4036F
:1044E00018464AF2D851C0F6060146F22933C0F602
:1044F000010398470346002B36D14FF00003C7F85D
:104500000C311CE0D7F8203107F10C021268D418E6
:1045100040F26933C0F6020398470246D7F80C31DF
:10452000D3181B782370D7F8203103F10103C7F8A3
:104530002031D7F80C3103F10103C7F80C3140F2F8
:104540006933C0F6020398470246D7F80C31D318F6
:104550001B78002B00F0538207F10803D7F82021C5
:104560001B689A42CEDB4AE207F1E40318464AF29E
:10457000DC51C0F6060146F22933C0F60103984724
:104580000346002B70D13B461B6893F83E31002B4D
:1045900004D13B461B681B79002B1AD0D7F8383161
:1045A000D3F80F2013461A464DF67953C0F601038F
:1045B00010469847034607F1300210464AF2E05190
:1045C000C0F606011A4643F64923C0F6050398478C
:1045D00019E0D7F83831D3F8132013461A464DF2B4
:1045E000C503C0F601031046984702460B4607F183
:1045F000300108464AF2E451C0F6060143F6492468
:10460000C0F60504A0474FF00003C7F8083118E0D2
:10461000D7F8203107F10C021268D31807F13001E6
:10462000D7F808218A1812781A70D7F8203103F1C8
:104630000103C7F82031D7F8083103F10103C7F8A7
:10464000083107F13002D7F80831D3181B78002B56
:1046500000F0D58107F10803D7F820211B689A42A2
:10466000D6DBCCE12CE3002007F1E40318464AF244
:10467000EC51C0F6060146F22933C0F60103984713
:104680000346002B40F015813B461B681B79002B2D
:104690004FD03B461B68B3F900309BB21CB2D7F831
:1046A0003831D3F8132013461A464DF67953C0F625
:1046B000010310469847024607F130032046114691
:1046C0001A4642F6B173C0F603039847C7F8F400E0
:1046D000D7F8F430002B1AD0D7F83831D3F813209C
:1046E00013461A464DF2C503C0F60103104698471B
:1046F00002460B4607F1100108464AF2E451C0F6A3
:10470000060143F64924C0F60504A047A2E007F1DC
:10471000100207F1300303F10A0310464AF2F05188
:10472000C0F606011A4643F64923C0F6050398472A
:1047300090E03B461B6893F83E31002B70D03B461F
:104740001B68B3F900309BB21CB2D7F83831D3F8EC
:10475000132013461A464DF67953C0F6010310464E
:104760009847024607F13003204611461A4643F2A5
:10477000BD73C0F603039847C7F8F000D7F8F030D0
:10478000002B1AD0D7F83831D3F80F2013461A4629
:104790004DF67953C0F6010310469847034607F1DA
:1047A000100210464AF2E051C0F606011A4643F6DE
:1047B0004923C0F6050398474CE0D7F83831D3F8C1
:1047C0000F2013461A464DF67953C0F601031046E2
:1047D00098470346002B11D107F1100207F130036F
:1047E00003F1080310464AF2F051C0F606011A46DA
:1047F00043F64923C0F6050398472BE007F1100262
:1048000007F1300303F1590310464AF2F051C0F6A4
:1048100006011A4643F64923C0F60503984719E0F6
:10482000D7F83831D3F80F2013461A464DF2C50396
:10483000C0F601031046984702460B4607F11001E7
:1048400008464AF2E451C0F6060143F64924C0F690
:104850000504A0474FF00003C7F8043118E0D7F86B
:10486000203107F10C021268D31807F11001D7F8B4
:1048700004218A1812781A70D7F8203103F1010345
:10488000C7F82031D7F8043103F10103C7F8043128
:1048900007F11002D7F80431D3181B78002B00F071
:1048A000AE8007F10803D7F820211B689A42D6DBB7
:1048B000A5E007F1E40318464AF2F451C0F60601F8
:1048C00046F22933C0F6010398470346002B40F017
:1048D00096804FF00003C7F800313B461B68D3F8C1
:1048E0004D30C7F8FC303B461B689B78062B04D143
:1048F0003B461B681B6EC7F8FC30D7F8FC0046F23D
:10490000E553C0F603039847C7F8EC00D7F8EC303E
:10491000002B62D03B461B6803F13503C7F8F83023
:10492000D7F83831D3F8132013461A464DF61553ED
:10493000C0F6010310463F4998470346002B06D0B6
:104940003B461B6803F11D03C7F8F83019E018E077
:10495000D7F8203107F10C021268D318D7F80021DC
:10496000D7F8F8108A1812781A70D7F8203103F1A6
:104970000103C7F82031D7F8003103F10103C7F86C
:104980000031D7F80031D7F8F820D3181B78002B66
:1049900035D007F10803D7F820211B689A42D7DBEE
:1049A0002DE0D7F8203107F10C021268D3183A46EF
:1049B0001168D7F800218A1802F11D0212781A70C6
:1049C000D7F8203103F10103C7F82031D7F80031BF
:1049D00003F10103C7F8003100E000BF3B461A684D
:1049E000D7F80031D31803F11D031B78002B06D034
:1049F00007F10803D7F820211B689A42D1DBD7F8CA
:104A0000243107F104021268D3181B78002B09D057
:104A100007F108031B6803F1FF32D7F820319A42EF
:104A20003FF7ECAB4FF00003184607F59477BD460F
:104A3000B0BD00BF0000000090B5AFB000AF78601F
:104A400043F21023C2F201034FF00002C3F8AC237B
:104A500040F27963C0F6020398470346002B10D159
:104A6000BF4842F2E913C0F60503984743F210230A
:104A7000C2F2010340F25262C3F8AC2340F2526327
:104A8000B5E140F26933C0F6020398470346D3F814
:104A90000631002B02D14FF00003A8E140F2693348
:104AA000C0F6020398470346D3F80E31012B1AD003
:104AB00040F26933C0F6020398470346D3F8123137
:104AC000012B10D0A64842F2E913C0F6050398471F
:104AD00043F21023C2F2010340F25362C3F8AC2345
:104AE00040F2536383E148F26143C0F60203984702
:104AF000C7F8A400D7F8A430002B10D1984842F290
:104B0000E913C0F60503984743F21023C2F20103EC
:104B100040F69902C3F8AC2340F6990367E140F2EE
:104B20006933C0F602039847034603F58F731846AE
:104B30008C498D4A8D4B4FF61524C0F60204A047D0
:104B40004FF00003C7F89830D7F8A4309B6A07F1FC
:104B500098024FF007001146984707F114031846D2
:104B6000814946F20553C0F60103984740F2693384
:104B7000C0F6020398470346D3F80A31C7F89430C9
:104B80004FF00003C7F8B4304FF00003C7F8B0305F
:104B90004FF00003C7F8AC304FF01E03C7F8A83041
:104BA000CDE0D7F8B430002B19D1D7F89830042BCA
:104BB00015D0D7F8A4301B699847C7F8AC00D7F8D0
:104BC000AC30002B07D04FF4FA604AF29D03C0F6D8
:104BD00005039847B3E04FF00103C7F8B430D7F8A6
:104BE000B030002B18D1D7F8A430DB6B07F11402DA
:104BF00010469847C7F8AC00D7F8AC30002B07D068
:104C00004FF4FA604AF29D03C0F60503984796E018
:104C10004FF00103C7F8B030D7F8A4004CF2D573B9
:104C2000C0F604039847D7F8A4004CF61523C0F645
:104C300004039847D7F8A4004CF6E923C0F6040310
:104C40009847D7F8A4004CF62563C0F604039847AC
:104C50007B68012B09D1D7F8A4004DF64903C0F6B3
:104C600004039847C7F8AC0008E0D7F8A4004DF655
:104C70004143C0F604039847C7F8AC00D7F8AC30FE
:104C8000002B09D04FF05100D7F8AC1041F2DD33C2
:104C9000C0F6020398476CE0D7F8A4004CF68123D5
:104CA000C0F604039847D7F8A4004AF2F851C0F6BA
:104CB00006014EF69D03C0F604039847D7F8A400FA
:104CC0004EF2B543C0F604039847C7F8AC00D7F8D6
:104CD000AC30002B09D04FF05400D7F8AC1041F2A3
:104CE000DD33C0F60203984743E04EF62903C0F6D1
:104CF000040398470346002B3AD107F1100207F14D
:104D00000C03104619464EF66103C0F6040398479B
:104D10003B69C82B09D03B694FF05200194641F25C
:104D2000DD33C0F60203984722E0FB684FF05500E0
:104D3000194641F2DD33C0F60203984718E0D7F870
:104D4000A8306FEA03034FEAD373DBB2D7F8A82089
:104D500002F1FF32C7F8A820002B7FF422AF08E051
:104D6000143201202C32012034320120B4320120CF
:104D700000BFD7F8B030002B13D0D7F8AC2040F6E6
:104D80009F039A420DD0D7F8A4301B6C9847C7F800
:104D9000A000D7F8A030002B03D0D7F8A030C7F878
:104DA000AC30D7F8B430002B11D0D7F89830042BA2
:104DB0000DD0D7F8A4305B699847C7F89C00D7F8A6
:104DC0009C30002B03D0D7F89C30C7F8AC300A4891
:104DD00042F2E913C0F60503984743F21023C2F2EA
:104DE0000103D7F8AC20C3F8AC23D7F8AC30184691
:104DF00007F1BC07BD4690BD1432012080B400AF5E
:104E000040F60443C2F200031B681846BD4680BC4E
:104E1000704700BF90B593B000AF78604FF00003CB
:104E20007B644FF000037B6107F11403184642F6E0
:104E30005D23C0F6050398474FF000033B644FF035
:104E40000003FB6347F60963C0F602039847FB6B58
:104E5000002B0CD042F28D63C0F6020398474FF04E
:104E600064004AF29D03C0F605039847EAE74FF055
:104E700000033B6107F11003184642F65D23C0F6BC
:104E8000050398473A697B699A420CD03B697B617C
:104E90007B6C03F101037B644FF0010041F2F513D9
:104EA000C0F60203984742F2C163C0F60203984776
:104EB00042F27563C0F6020398470346002B1AD0EE
:104EC00006E04FF064004AF29D03C0F605039847E0
:104ED00040F26933C0F602039847034693F829303D
:104EE000002BEED14EF25563C0F6030398474FF006
:104EF0000103FB63A6E74FF6C563C0F603039847BB
:104F00000346D3F815203B6CD31A7B637A6B41F2CE
:104F100088339A4210D94FF6C563C0F60303984709
:104F20000346D3F815303B644FF000037B644EF228
:104F30005563C0F6030398477B6CB3F5616F1DDDC5
:104F400040F26933C0F602039847034693F82930CC
:104F5000002B13D07B6B002B10D04FF6C563C0F62F
:104F6000030398470346D3F815303B644FF0000322
:104F70007B644EF25563C0F60303984740F6CD6359
:104F8000C0F60403984740F6B063C2F200031B6802
:104F900003F1010240F6B063C2F200031A6046F268
:104FA000C113C0F60203984738633B6B0B2B14D137
:104FB00040F6B063C2F200031B6803F00103002B4C
:104FC00005D049F64D43C0F60203984734E049F650
:104FD0007D43C0F6020398472EE03B6B022B05D1C0
:104FE00049F64D43C0F60203984725E040F6B0630A
:104FF000C2F200031B68132B06D940F6B063C2F25D
:1050000000034FF000021A6040F6B063C2F20003E2
:105010001B68002B04D149F67D43C0F60203984774
:1050200040F6B063C2F200031B680A2B04D149F6B4
:105030004D43C0F60203984740F26933C0F60203BD
:1050400098470346D3F8F630002B00F08C8040F2EE
:105050006933C0F6020398470346D3F8FA30FB627F
:10506000FB6A18464FF20D43C0F601039847B86239
:10507000BB6A002B77D0BB6AD3F851307B6207F153
:105080000803184642F2E913C0F60503984740F6B4
:105090000443C2F200031B683B62BB6A03F5AA73B8
:1050A00007F108021046194642F2E143C0F6050333
:1050B0009847F8617A6AFB69D41A40F26933C0F6FE
:1050C000020398470346D3F8FE309C4207DC40F6C3
:1050D0000443C2F200034FF001021A6011E040F2F3
:1050E0006933C0F6020398470346D3F80221FB69EF
:1050F0009A4206DC40F60443C2F200034FF000027D
:105100001A6040F60443C2F200031B683A6A9A42EE
:1051100029D040F60443C2F200031B684FF062003E
:10512000194641F64113C0F6020398474FF00003B9
:10513000BB6315E0BB6BBB61BB6903F10103BB61E2
:1051400040F60443C2F200031B68B869194648F6EA
:105150006543C0F602039847BB6B03F10103BB63D1
:10516000BB6B012BE6DD4FF064004AF29D03C0F6F5
:105170000503984766E600BF80B586B000AF78604B
:105180004FF0020047F28933C0F6030398473861B5
:1051900048F2E933C0F602039847F860FB68002B39
:1051A00007D14FF47A704AF29D03C0F60503984781
:1051B000F7E74FF000037B617B69022B0ED0FB68A1
:1051C0009B699847FB68DB699847FB68DB6A4FF08F
:1051D000000098474FF002037B610FE0FB685B6BB8
:1051E0009847B860BB68002B07DD3869F96847F25B
:1051F000B133C0F60303984700E000BF4FF00A0048
:105200004AF29D03C0F605039847D5E780B58AB0FA
:1052100000AF78604FF0010047F28933C0F6030316
:105220009847F86148F21143C0F602039847B86105
:10523000BB69002B07D14FF47A704AF29D03C0F688
:1052400005039847F7E748F28943C0F602039847F9
:1052500078614FF000037B624FF0010041F61523A7
:10526000C0F6020398470346002B02D04FF0040318
:105270007B627B6A022B1BD0042B28D0BB699B6905
:105280009847BB69DB699847BB69DB6A4FF0000050
:1052900098477B699B6998477B69DB6998477B697D
:1052A000DB6A4FF0000098474FF002037B621AE080
:1052B000BB695B6B984738613B69002B12DDF8696D
:1052C000B96947F2B133C0F6030398470BE0F869B8
:1052D000B96947F66913C0F6030398474FF0000316
:1052E0007B6200E000BF7B69002B35D04DF6D40314
:1052F000C2F2000393F8C032002B2DD04FF03203DE
:1053000087F823304FF00003FB7214E07B699B6C3D
:1053100007F10B0210464FF001014FF000029847D1
:10532000F860FB68002B16D1FB7A184648F2B523CB
:10533000C0F60303984797F82330002B0CBF0023D7
:105340000123DBB297F8232002F1FF3287F82320F4
:10535000002BDBD100E000BF4FF064004AF29D0358
:10536000C0F60503984777E780B588B000AF78604E
:105370004FF0000047F28933C0F603039847B86145
:1053800048F23943C0F60203984778617B69002BE5
:1053900007D14FF47A704AF29D03C0F6050398478F
:1053A000F7E74FF00003FB614FF0000041F61523D3
:1053B000C0F6020398470346002B02D04FF00403C7
:1053C000FB61FB69022B1DD0042B2AD0B86947F67C
:1053D0009D33C0F60303984738617B699B69984702
:1053E0007B69DB6998477B69DB6A4FF0000098476F
:1053F000B86947F63D43C0F6030398474FF00203F0
:10540000FB611AE07B695B6B9847F860FB68002BD7
:1054100012DDB869796947F2B133C0F603039847E2
:105420000BE0B869796947F66913C0F6030398473A
:105430004FF00003FB6100E000BF4FF00A004AF2AA
:105440009D03C0F605039847AEE700BF90B5B5B021
:1054500002AF786040F26933C0F602039847034612
:1054600093F82630002B04D041F62D73C0F60203CA
:1054700098474FF00003C7F8BC304FF00003C7F85F
:10548000B830D7F8B830002B08D04FF064004AF29B
:105490009D03C0F60503984700F035BC4FF00A00A5
:1054A0004AF29D03C0F60503984740F26933C0F6FF
:1054B00002039847034693F82930002B00F022841A
:1054C0004DF6D403C2F20003D3F8D032002B20D023
:1054D0004DF6D403C2F20003D3F8D0320A2B0FD911
:1054E0004DF6D403C2F20003D3F8D032A3F10A027E
:1054F0004DF6D403C2F20003C3F8D02200F003BC7F
:105500004DF6D403C2F200034FF00002C3F8D022DC
:10551000F9E34FF00003C7F8BC304FF00003C7F8C1
:10552000C430D7E342F27563C0F6020398470346DE
:10553000002B0ED040F26933C0F6020398470346B1
:105540004FF0000283F829204FF00103C7F8B8306C
:10555000CDE3D7F8C4004FF27143C0F6010398477A
:10556000C7F8AC00D7F8AC30002B00F0A483D7F814
:10557000AC3093F84B31002B06D1D7F8AC304FF05C
:10558000000283F875219FE3D7F8AC309B780D2B90
:1055900000F08482D7F8AC309B780C2B1CD14FF0F4
:1055A0000103C7F8BC3048F28923C0F603039847CB
:1055B000C7F8A800D7F8A830002B06DAD7F8AC3027
:1055C0004FF0000283F875217EE3D7F8AC30D7F8AE
:1055D000A820C3F8622161E2D7F8AC309B78062B93
:1055E00040F00A814FF00003C7F8B430D7F8AC3070
:1055F00093F86430022B0BD0D7F8AC3093F86430BA
:10560000032B05D0D7F8AC3093F86430042B7AD153
:10561000D7F8AC3093F85E301946D7F8AC3093F831
:105620005F301A46D7F8AC301B6E4FF00200009086
:1056300007F1680001904FF0000041F64D24C0F6DC
:105640000204A047C7F8C000BB6EC7F8B430D7F853
:10565000C030002B40F09880D7F8AC3093F864301D
:10566000042B18D1D7F8AC3093F8653007F16802F5
:10567000104619464FF22D73C0F602039847C7F83B
:10568000A000D7F8AC00D7F8A01046F29503C0F6FA
:105690000203984778E0D7F8AC3093F86430032BD6
:1056A00018D1D7F8AC3093F8653007F1680210468E
:1056B00019464FF62503C0F602039847C7F89C0029
:1056C000D7F8AC00D7F89C1045F63573C0F6020346
:1056D000984759E0D7F8AC3093F8653007F1680285
:1056E000104619464FF61D13C0F602039847C7F837
:1056F0009800D7F8AC00D7F8981045F6D553C0F607
:105700000203984740E0D7F8AC3093F85E30194672
:10571000D7F8AC3093F85F301A46D7F8AC301B6E30
:105720004FF00100009007F1640001904FF000007D
:1057300041F64D24C0F60204A047C7F8C0007B6EB6
:10574000C7F8B430D7F8AC3093F86430002B0DD1E3
:105750007B6EA7F8A630B7F9A630D7F8AC0019468B
:1057600045F6D553C0F6020398470EE07B6EA7F8C6
:10577000A430B7F8A430D7F8AC00194645F6357315
:10578000C0F60203984700E000BFD7F8C00041F21E
:10579000AD23C0F602039847D7F8AC304FF00002B3
:1057A00083F87621D7F8C02040F20E739A4212D1C6
:1057B00041F6BD63C0F602039847D7F8B430DAB2B9
:1057C000D7F8AC3083F87621D7F8AC304FF001022F
:1057D00083F8752178E2D7F8C030002B00F05E81A5
:1057E00041F69563C0F602039847D7F8AC304FF006
:1057F000010283F8752167E2D7F8AC309B78082B5B
:1058000057D1D7F8AC30D3F84D2007F15C031046E0
:10581000194645F2B913C0F603039847C7F8C0000C
:10582000D7F8C030002B06D0D7F8AC304FF00102CB
:1058300083F8752148E2D7F8AC30D3F84D3003F146
:10584000010207F160031046194645F2B913C0F68C
:1058500003039847C7F8C000D7F8C030002B06D024
:10586000D7F8AC304FF0010283F875212CE2FB6DC4
:105870004FEA03423B6E1A43D7F8AC30C3F86221BB
:10588000D7F8AC30D3F84D30A3F51C43A3F1BA03DD
:105890004FEA5303C7F89430D7F8AC30D3F86231ED
:1058A000D7F89400194649F20163C0F602039847FD
:1058B000F4E0D7F8AC309B780B2B53D1D7F8AC3051
:1058C000D3F84D204BF22B039A424BD9D7F8AC308A
:1058D000D3F84D204BF28F039A4243D8D7F8AC301F
:1058E000D3F84D2007F154031046194645F2B91379
:1058F000C0F603039847C7F89000D7F8AC30D3F848
:105900004D3003F1010207F1540303F10403104683
:10591000194645F2B913C0F603039847C7F88C003F
:10592000D7F89030002B03D1D7F88C30002B06D05D
:10593000D7F8AC304FF0010283F87521C4E107F1CC
:10594000540318464FF003014FF22D73C0F60203C3
:105950009847C7F88800D7F8AC30D7F88820C3F844
:1059600062219BE0D7F8AC309B78052B47D1D7F864
:10597000AC30D3F84D2049F6CE439A423FD1D7F808
:10598000AC30D3F84D2007F150031046194645F2CC
:10599000B913C0F603039847C7F8C000D7F8C03062
:1059A000002B06D0D7F8AC304FF0010283F87521F8
:1059B0008AE1D7F8AC30D3F84D3003F1010207F19A
:1059C0004C031046194645F2B913C0F60303984735
:1059D000C7F8C000D7F8C030002B06D0D7F8AC30DD
:1059E0004FF0010283F875216EE1FB6C4FEA034230
:1059F0003B6D1A43D7F8AC30C3F862214EE0D7F8BC
:105A0000AC309B78002B26D14FF00003BB64D7F855
:105A1000AC30D3F84D2007F148031046194645F243
:105A2000B913C0F603039847C7F8C000D7F8C030D1
:105A3000002B06D0D7F8AC304FF0010283F8752167
:105A400042E1BB6CD7F8AC00194645F6D553C0F619
:105A50000203984722E0D7F8AC30D3F84D2007F185
:105A600044031046194645F2B913C0F6030398479C
:105A7000C7F8C000D7F8C030002B06D0D7F8AC303C
:105A80004FF0010283F875211EE17B6CA7F8863088
:105A9000B7F98620D7F8AC30C3F86221D7F8AC301C
:105AA0009B780D2B0CD1D7F8AC3093F88131022BB9
:105AB0000CD1D7F8AC304FF0020283F8752105E025
:105AC000D7F8AC304FF0020283F87521D7F8AC005C
:105AD00041F20103C0F603039847D7F8AC3093F8BE
:105AE0007830002B06D0D7F8AC0040F2C103C0F6E6
:105AF00003039847D7F8AC30DB78002B00F0DD804B
:105B000007F17003184642F2E913C0F605039847FF
:105B100040F26933C0F602039847034693F82630F3
:105B2000002B71D041F68173C0F6020398470346FB
:105B3000002B00F0C4804CF27173C0F60403984748
:105B40004EF6DD73C0F601039847C7F880004FF0AA
:105B50000003C7F8B03046E0D7F8B0004FF2714309
:105B6000C0F601039847F867FB6F93F87531022B75
:105B700033D14FF0000387F83330FB6FB3F90030B7
:105B80009BB29BB2BB86FB6FD3F86631C7F83A3045
:105B9000FB6FD3F86231C7F8363007F12C0307F1F9
:105BA000700292E80300186003F10403198003F106
:105BB00002034FEA11421A7007F1280318464EF605
:105BC000F533C0F603039847C7F8C000D7F8AC0018
:105BD00045F60D53C0F602039847D7F8B03003F1ED
:105BE0000103C7F8B030D7F8B020D7F880309A4218
:105BF000B2DB41F62D73C0F6020398474CF2A57351
